:10C00000786E0020694D02007D4D0200914D0200C6
:10C01000934D0200934D0200934D0200000000007A
:10C02000000000000000000000000000934D02002E
:10C03000934D020000000000934D0200990801009A
:10C04000934D0200934D0200934D0200934D020068
:10C05000934D0200934D0200B7100200934D020071
:10C06000BF9A0100934D0200934D0200934D0200D0
:10C07000934D0200934D0200E7480100A3C5000064
:10C08000934D020007B4010091080100934D020096
:10C09000934D0200934D0200934D02005B49010055
:10C0A000934D0200934D0200934D0200934D020008
:10C0B000934D0200934D0200934D0200934D0200F8
:10C0C000934D0200934D0200934D0200934D0200E8
:10C0D000934D0200934D0200934D02003F40020039
:10C0E000934D0200934D020000000000934D0200AA
:10C0F000934D0200934D0200934D0200934D0200B8
:10C10000934D0200934D0200CFC70000934D0200F3
:10C110000000000000000000934D0200934D02005B
:10C12000934D0200934D0200934D0200934D020087
:10C13000934D0200E3160100934D0200934D02005F
:10C1400000000000000000000000000000000000EF
:10C15000934D0200934D020045B40100934D02003F
:10C1600000000000000000000000000000000000CF
:10C1700000000000000000000000000000000000BF
:10C1800000000000000000000000000000000000AF
:10C19000000000000000000000000000000000009F
:10C1A000000000000000000000000000000000008F
:10C1B000934D0200934D0200934D0200934D0200F7
:10C1C0006FC30000934D0200934D0200934D020097
:10C1D000934D0200934D02007B440100E9440100AD
:10C1E000934D0200934D0200934D020000000000A9
:10C1F00000000000934D0200934D0200934D020099
:10C20000934D0200934D020000000000000000006A
:10C21000934D0200934D0200934D0200934D020096
:10C22000934D0200934D0200934D0200934D020086
:10C23000934D0200934D0200934D0200934D020076
:10C24000934D0200934D0200934D0200934D020066
:10C25000934D0200934D0200934D0200934D020056
:10C26000934D0200934D0200934D020080B502F001
:10C27000BBFE0421DFF8780803F0DEFF0020DFF8C2
:10C28000741808600821DFF8700803F0D5FF00205B
:10C29000DFF8681808600020DFF8641808700A20CA
:10C2A000DFF8601808700120DFF85C18086003F000
:10C2B00083F803F0D1F8002004F07CF830280FD187
:10C2C000012004F077F830280AD140F2D920DFF8B5
:10C2D0003C1808604FF42D70DFF83418086009E04E
:10C2E00040F2F320DFF82418086040F2FD20DFF868
:10C2F00020180860DFF8200A006830F01000DFF82E
:10C30000181A086003F012F9022002F0C3FD0020A1
:10C31000DFF8001808700020DFF8FC170870002014
:10C32000DFF8F81708600020DFF8F417086004F061
:10C33000DDFC002808D1DFF8E009006830F48070E7
:10C34000DFF8D419086007E0DFF8CC09006850F482
:10C350008070DFF8C419086003F07CFDDFF8B809CD
:10C36000006850F00100DFF8B019086001BD80B529
:10C370001521DFF8B00704F0DCFE04F0DBFFDFF886
:10C3800098090068C00703D4082005F019FB43E0B2
:10C39000DFF894070068012816D1DFF890070068DD
:10C3A000002809D0DFF884070068052804D0DFF8EA
:10C3B0007C070068042807D10020DFF86C170860AC
:10C3C0000020DFF83C1B086003F0D6FADFF83407E2
:10C3D0000078112808DADFF84409DFF8281709780F
:10C3E00050F82100804709E0DFF8140B006850F096
:10C3F0000800DFF80C1B086001F06AFE01F0A8FEDF
:10C4000001F002FF01F03EFF02F072F902F0BAFC07
:10C4100002F09CFD05F0B1F801BD10B4DFF8E04674
:10C420002070C0B2012802D0C0B2022809D1DFF8C2
:10C43000F0080160DFF8EC080270DFF8C80A03605A
:10C440000BE00020DFF8D81808600020DFF8D418CF
:10C4500008700020DFF8AC1A086010BC7047DFF8E5
:10C46000A80A00687047DFF8A40A00687047DFF880
:10C47000980A006852280ED0DFF88C0A00686528F8
:10C4800009D0DFF8840A0068662804D0DFF8780A4B
:10C490000068542801D1012000E0002070470120ED
:10C4A000DFF8841608607047DFF87C060068012812
:10C4B00001D1002002E0DFF8480A00687047DFF889
:10C4C0006C0600687047DFF8480A00687047DFF8BC
:10C4D000500600687047DFF8440600687047DFF8D0
:10C4E00048080068DFF830180968C1F340110029D6
:10C4F00013D1DFF824180968C1F3C011002906D050
:10C50000882148434FF4FA6190FBF1F005E0942153
:10C5100048434FF4FA6190FBF1F0704780B504F0A6
:10C52000CBFB02BDDFF8F0070068C0F34010002825
:10C530001AD1DFF8E4070068C0F3C010002809D062
:10C54000DFF8D0090168882041434FF4167091FB51
:10C55000F0F00CE0DFF8BC090168942041434FF48F
:10C56000167091FBF0F002E0DFF8A8090068704750
:10C57000DFF8A4070068C0F30020002803D1DFF82B
:10C580009C09006803E0DFF89409006840427047A6
:10C59000DFF860050068002801D0012000E00020DD
:10C5A000704738B50220DFF878190860DFF86807AF
:10C5B0000068C00740F10681DFF868090568DFF808
:10C5C00064090468DFF860090068800709D4DFF8AF
:10C5D0005C090068800704D4DFF854090068C005CE
:10C5E00023D4DFF85009006830F00200DFF8441966
:10C5F000086002E0DFF82C090068DFF83409006801
:10C60000C005F7D50121DFF82C0905F0ADFA0121AD
:10C61000DFF8200905F0AEFADFF81809006850F0DD
:10C620000200DFF810190860D0E0DFF8DC040068D1
:10C6300001285BD1DFF8DC040078002818D1DFF88E
:10C64000F80801680F2000FB0155102095FBF0F061
:10C65000DFF8E4180860DFF8E40801680F2000FB49
:10C660000144102094FBF0F0DFF8D01808602CE0B3
:10C67000DFF8A0040078042827D103F097FEDFF844
:10C68000C0180968401AB0F57A7F1ED3DFF8840815
:10C69000006805F0A9FD002817D1DFF89C080168A3
:10C6A0000F2000FB0155102095FBF0F0DFF88818F3
:10C6B0000860DFF8880801680F2000FB01441020A3
:10C6C00094FBF0F0DFF8741808600020DFF87418AD
:10C6D00008600020DFF8701808600020DFF86C1890
:10C6E00008600020DFF86818086033E0DFF85408BD
:10C6F00001680F2000FB0155102095FBF0F1DFF8D9
:10C7000044080160DFF830080068091ADFF8FC030C
:10C7100000684143642091FBF0F0DFF830180860B6
:10C72000DFF8240801680F2000FB0144102094FB6F
:10C73000F0F1DFF814080160DFF800080068091A5A
:10C74000DFF8CC0300684143642091FBF0F0DFF890
:10C7500000180860DFF8C4070068002814D4DFF868
:10C76000B8050068C0F30020002806D1DFF8DC0718
:10C770000068DFF8AC1B08601AE0DFF8D407006837
:10C78000DFF89C1B086013E0DFF88C050068C0F33D
:10C790000020002806D1DFF8B8070068DFF8801B0A
:10C7A000086005E0DFF8A4070068DFF8741B086084
:10C7B000DFF86C0B0068002808D50020DFF8601B4C
:10C7C000086003E00020DFF8581B086031BD00203E
:10C7D000DFF8801708605FF48020DFF87C170860BE
:10C7E000FF20DFF8CC1908605FF48020DFF86417C1
:10C7F00008600F20DFF80C1308700120DFF8241BFD
:10C800000860704710B50420DFF80C13087003F0BF
:10C810000FFB0400DFF89C09006805F0E5FC84428A
:10C8200004DA03F0C3FDDFF890190860DFF81C0795
:10C83000006840F29111884204DBDFF814070068B9
:10C8400000280BD4DFF80807006840F291118842F5
:10C8500009DBDFF8F8060068002804D503F0A6FD20
:10C86000DFF85419086003F0A1FDDFF84C190968DE
:10C87000401A40F2E931884208D3022002F00AFB54
:10C880000A20A04908700520A84908609C48007843
:10C89000002801D001F02CFA10BD80B55020DFF83F
:10C8A0006816086000209C490870012096490860BD
:10C8B000022002F0EFFA9248007800280DD00C20F8
:10C8C0009049087003F072FDDFF8EC18086004204E
:10C8D0009149087000208C49086001BD10B5042002
:10C8E0008D490870012002F0D5FA03F0A1FA040086
:10C8F000DFF8C008006805F077FC844204DA03F032
:10C9000055FDDFF8B418086003F050FDDFF8A818F3
:10C910000968401A40F2E931884201D301F0E8F990
:10C9200010BD80B55520DFF8E015086004207A4975
:10C93000087073480078032802D00020724908600C
:10C940006F480078002802D101F0BEF921E06C4860
:10C950000078012802D101F065FA1AE068480078F1
:10C96000042802D101F0D9F913E0654800780228C3
:10C9700002D101F007FA0CE061480078052802D1E5
:10C9800001F096FB05E05E480078062801D101F031
:10C99000F9F901BD80B55620DFF86C15086000205C
:10C9A0005D49087056480078042801D001F0A0F9CC
:10C9B00001BD80B5042058490870DFF86C09006893
:10C9C00001280DDB4FF4805006F0E6FD002807D16A
:10C9D000DFF854090068401FDFF84C19086055E083
:10C9E000DFF8340500680B2815DBDFF82C0300683E
:10C9F000C0F3401000280ED14FF4805006F0CCFD5B
:10CA0000002808D146480068012804D10120DFF839
:10CA1000FC1408603AE05120DFF8EC14086040484C
:10CA20000068002832D13D480068012824D1BA4866
:10CA30000068C0F34010002804D1DFF8DC0400686F
:10CA40000B280EDAB4480068C0F34010002813D059
:10CA50001421012003F064FADFF8BC14096888424D
:10CA60000ADADFF89C04006850F48020DFF89014A4
:10CA700008600020294908600020DFF89C14086045
:10CA8000002007F0E1FC012025490860DFF8E80BF1
:10CA90000078012802D101F0C5F926E0DFF8D80BB3
:10CAA0000078002802D101F00FF91EE0DFF8C80B72
:10CAB0000078032802D101F01BF916E0DFF8B80B6B
:10CAC0000078042802D101F028F90EE0DFF8A80B65
:10CAD0000078062802D101F011FB06E0DFF8980B80
:10CAE0000078052801D101F0E3FA01BD0000000043
:10CAF000007000401070004000400640204006409A
:10CB00006E2E00206F2E0020C02C0020782D0020DB
:10CB10007C2D0020742E0020732E0020CC2C0020B1
:10CB2000D02C002000700340C42C0020FC2C0020DE
:10CB300038B50420DFF8C0190870DFF8EC0700688A
:10CB4000012807DBDFF8E0070068401FDFF8D8178F
:10CB50000860B1E0DFF8C0030168DFF8A0090268EF
:10CB6000DFF89C090068121A463A91420FDA6A48C7
:10CB70000068C0F34010002809D1DFF88809006878
:10CB8000012804D10120DFF88413086094E05320C9
:10CB9000DFF874130860DFF86C090068002840F0C3
:10CBA0008B8004F089F8DFF86009006801282BD138
:10CBB00059480068C0F34010002807D1DFF8580337
:10CBC000046804F079F83238844212DB5248006875
:10CBD000C0F3401000286BD0DFF83C03046804F079
:10CBE0006BF805003221002003F09AF92D1AAC42AF
:10CBF0005EDAC348006850F48020C1490860002014
:10CC0000DFF80419086053E004F056F8C2490860E0
:10CC100041480068C0F30020002822D13E48006847
:10CC2000C0F34010002819D13B480068C0F3C01081
:10CC3000002809D0B84801684FF4FA6041438731B1
:10CC4000882091FBF0F031E0B34801684FF4FA60BE
:10CC500041439331942091FBF0F027E0AE48006807
:10CC600024E02D480068C0F3401000281BD12A485A
:10CC70000068C0F3C01000280AD0A74801684942E4
:10CC80004FF4FA6041438739882091FBF0F00DE0C2
:10CC9000A148016849424FF4FA6041439339942016
:10CCA00091FBF0F002E09C480068404207F0CCFBAA
:10CCB0000120DFF850180860DFF8BC090078002870
:10CCC00002D101F001F826E0DFF8AC090078032872
:10CCD00002D101F00DF81EE0DFF89C09007804286D
:10CCE00002D101F01AF816E0DFF88C09007802286A
:10CCF00002D101F047F80EE0DFF87C090078062841
:10CD000002D101F03FF806E0DFF86C090078052851
:10CD100001D101F0CDF931BDB42C0020744C0200DA
:10CD2000202D0020752E0020E42C002010B554206A
:10CD3000754908600220DFF8C0170870DFF838096D
:10CD40000078022805D0DFF830090078062840F086
:10CD5000D380DFF824090078022816D1DFF81C09F7
:10CD60000068C0F3401000280FD1DFF814090068F4
:10CD7000643069490968884207DADFF8B00500685D
:10CD800050F00070DFF8A4150860DFF87C07006839
:10CD9000002833D103F00AFBDFF8E8180968401ACD
:10CDA00040F6A171884202D300F0C3FFA7E003F070
:10CDB0003FF8DFF800140968C14219DB03F0F6FA06
:10CDC000DFF8C4180968401AB0F5FA6FC0F08C801B
:10CDD0004F480068652808DADFF85005006850F011
:10CDE0004000DFF8481508607EE000F0A2FF7BE01D
:10CDF00003F0DCFADFF89018086075E0DFF824052E
:10CE00000068012807D1DFF82405006850F04000D1
:10CE1000DFF818150860DFF8CC090168012003F07D
:10CE20007FF8040002F01AFF04193B4800688442AE
:10CE300002DB01F013F957E0DFF8AC0900780128B4
:10CE40000FD1DFF8A809006865280ADBDFF82C0895
:10CE50000068C0F34010002803D1002001F0A9F8B9
:10CE600042E003F0A3FADFF888190A68DFF8141823
:10CE70000968401A824207D2DFF878090068002862
:10CE800002D101202149086002F0D2FFDFF824130B
:10CE90000968C14223DBDFF860090068002803D17C
:10CEA000DFF84C09046801E040F6B83403F07EFA7C
:10CEB000DFF8D4170968401A844215D21448006874
:10CEC000652808DADFF86404006850F04000DFF8F5
:10CED0005C14086008E001200C49086004E003F0DD
:10CEE00065FADFF8A4170860DFF84004006800283E
:10CEF00005D001F0EDF802E0012001F05AF810BD74
:10CF0000A02D0020242D0020B02C0020BC2C0020BF
:10CF1000642D0020EC2C0020442D0020F82C002053
:10CF20000C80034068800340108003401880034059
:10CF30006C80034000800340682D00206C2D002091
:10CF40009C2D0020A82D0020AC2D0020582D002065
:10CF50005C2D0020089003400C90034038B552200F
:10CF6000964908600220DFF890150870DFF808077E
:10CF70000078012840F01781DFF800070068C0F34F
:10CF80004010002810D1DFF8A8030068DFF8F01681
:10CF900009686439884207DADFF89003006850F0C6
:10CFA0000070DFF888130860DFF858050068002873
:10CFB00032D103F0FBF9DFF8CC160968401AB0F55E
:10CFC0007A6F02D300F0C6FEF0E002F031FF79493B
:10CFD000096888421ADB03F0E9F9DFF8AC16096842
:10CFE000401AB0F5FA6FC0F0D780DFF8100800687B
:10CFF000652808DADFF83403006850F04000DFF8F5
:10D000002C130860C8E000F0A5FECFE003F0CEF9D5
:10D01000DFF874160860BFE0C2480068012805D137
:10D02000C248006850F04000C0490860DFF8B4070B
:10D030000168DFF8CC0400684118002002F070FF9E
:10D040000400BB48056802F009FEDFF8B014096867
:10D050000C1B241AA54202DB01F014F89CE0DFF857
:10D060001C060068C0F3401000280DD1DFF87807D7
:10D070000078012808D1DFF874070068652803DB11
:10D08000002000F0BDFF87E0DFF8F0050068C0F386
:10D09000401000280DD0DFF850070078012808D193
:10D0A000DFF848070068AB2803DB002000F0A8FF8A
:10D0B00072E0DFF8C8050068C0F3401000280CD10A
:10D0C000DFF824070078022807D1DFF8200700687E
:10D0D000642802DA00F024FF5EE0DFF8A0050068B3
:10D0E000C0F3401000280CD0DFF8FC0600780228BE
:10D0F00007D1DFF8F8060068AA2802DA00F010FF6E
:10D100004AE003F053F9DFF8E8160A68DFF874150F
:10D110000968401A824207D2DFF8D8060068002862
:10D1200002D101208349086002F082FE214909688A
:10D1300088422CDBDFF8C0060068002803D1DFF846
:10D14000B00604680BE0DFF834050068C0F3801017
:10D15000002802D041F2707401E040F6B83403F0C8
:10D1600025F9DFF824150968401A844214D2DFF843
:10D170008C060068652806DA6C48006850F04000AC
:10D180006A49086008E001206A49086004E003F089
:10D190000DF9DFF8F414086064480068002805D031
:10D1A00000F096FF02E0012000F02AFF31BD0000F0
:10D1B00034900340382D00208C2D0020B02C00200E
:10D1C00010B55420DFF838160860DFF8AC0400789A
:10D1D000022805D0DFF8A0040078062840F09C80E3
:10D1E0000A21012002F09CFE51490968884246DB71
:10D1F000DFF8A80A006800280DD10120DFF89C1A8A
:10D20000086003F0D3F8DFF88014086003F0CEF86C
:10D21000DFF87014086046480068002802D500F066
:10D2200088FD7CE040F6B830DFF8981A086003F01B
:10D23000BDF8DFF850140968401AB0F5FA6F02D350
:10D2400000F077FD6BE002F0F3FD0400DFF89C0ACC
:10D25000006804F0C9FF84420BDB03F0A7F8DFF895
:10D2600028140968401AB0F57A7F44D300F061FDB4
:10D2700041E003F09BF8DFF8101408603BE0002069
:10D28000DFF8181A086003F091F8DFF864150A68EF
:10D29000DFF8F0130968401A824202D201202549C2
:10D2A000086002F0C5FD0400DFF8400A006804F0E1
:10D2B0009BFF84421ADB03F079F8DFF834150A6823
:10D2C000DFF8C4130968401A824214D2DFF82C0533
:10D2D0000068652806DA1548006850F040001349D8
:10D2E000086008E001201349086004E003F05EF8DC
:10D2F000DFF8941308600B480068012805D10B483B
:10D30000006850F04000094908600848006800289B
:10D3100005D000F0DDFE02E0012000F04AFE10BD65
:10D32000602D0020B82C0020802D0020A02D002092
:10D33000442D0020BC2C002038B55220DFF8C0144A
:10D340000860DFF834030078012840F0D080DFF86F
:10D35000300A04686948056869480168002002F0DD
:10D36000DFFD2D1AAC4202DB00F0F4FCC2E06448A1
:10D3700001683231C1480068C0F3401000280AD16A
:10D38000DFF8FC0902685D4803685D4800681B1A05
:10D39000323B9A4210DAB9480068C0F340100028C6
:10D3A00058D0DFF8DC09046854480568002002F012
:10D3B000B7FD2D1AAC424DDBDFF85C0A006800288F
:10D3C0000BD10120DFF8501A086002F0EFFFAE49E0
:10D3D000086002F0EBFFAB49086040F6B830DFF8B8
:10D3E000E418086002F0E2FFA6490968401AB0F5A7
:10D3F000FA6F02D300F0AEFC7CE002F019FD0400ED
:10D400009E480068C0F34010002806D1DFF8DC0811
:10D41000006804F0E9FE84420CDA98480068C0F322
:10D420004010002811D0DFF8F409006804F0DCFE99
:10D4300084420ADB02F0BAFF93490968401AB0F54A
:10D44000FA6F40D300F086FC3DE002F0AFFF8E495A
:10D45000086038E002F0AAFFDFF894130A688949EF
:10D460000968401A824203D20120DFF8B41908602B
:10D4700002F0DEFC0400DFF87408006804F0B4FE7B
:10D4800084421CDB02F092FFDFF864130A687E49D5
:10D490000968401A824216D2DFF8600300686528E6
:10D4A00008DADFF8A40C006850F04000DFF8981CA0
:10D4B000086008E00120DFF86819086003E002F066
:10D4C00075FF71490860CF480068012807D1DFF86F
:10D4D000780C006850F04000DFF86C1C0860DFF842
:10D4E000680C0068002805D000F0F2FD02E0012081
:10D4F00000F086FD31BD0000732E0020502D00206D
:10D50000142D0020CC2C0020D02C002010B554204D
:10D51000BB49086059480068C0F34010002802D198
:10D520007FF01D0401E07FF0630402F081FC4042C3
:10D53000DFF8B8170968884212DADFF8E0090068F6
:10D54000401DDFF8D8190860DFF8D00900686528A9
:10D5500003D249480078012812D100F0C9FB0FE03E
:10D56000DFF888070068844206DA4348007801281B
:10D5700002D100F0BDFB03E00020DFF8A019086035
:10D58000A0480068012807D1DFF8BC0B006850F004
:10D590004000DFF8B41B0860DFF8AC0B006800281F
:10D5A00001D000F095FD10BD80B55220944908606F
:10D5B00002F03EFCDFF83417096881420EDADFF82A
:10D5C0005C090068401DDFF854190860DFF84C0959
:10D5D0000068652806D300F08BFB03E00020DFF82D
:10D5E0003C19086087480068012807D1DFF8580B0C
:10D5F000006850F04000DFF8501B0860DFF8480B6F
:10D600000068002801D000F063FD01BD80B5DFF89F
:10D61000480C0068012813DB572079490860DFF8BF
:10D62000380C00680A38DFF8301C0860DFF8280C76
:10D63000006800281FD50020DFF81C1C08601AE0D5
:10D64000DFF8140C0068002813D557206C490860D7
:10D65000DFF8040C00680A30DFF8FC1B0860DFF814
:10D66000F80B0068012806DB0020DFF8EC1B0860DF
:10D6700001E000F029FB01BD6E2E0020B42C00203B
:10D68000482D0020842D0020942D002080B55120AD
:10D690005B490860DFF8140A0078062840F099809A
:10D6A000DFF8280A0068C0F34010002804D1DFF832
:10D6B000D006006810280BDBDFF8100A0068C0F302
:10D6C000401000282AD0DFF8B8060068032825DAC1
:10D6D0005FF40010002104F05CF902F079F9DFF842
:10D6E000101A0860DFF8080A0068DFF8D815096822
:10D6F000884206DBDFF8F8090068DFF8C815086023
:10D7000006E0DFF8C00500681438DFF8B8150860D7
:10D7100002F04CFEDFF8DC19086061E05FF40010F5
:10D72000002104F05EF902F041FEDFF8C819096833
:10D73000401ADFF8C419884205D302F049F9DFF82E
:10D74000B01908602EE002F031FEDFF8A819096870
:10D75000401A4EF66121884212D3DFF87009006842
:10D76000C0F3C010002805D040F2DC50DFF880196B
:10D77000086017E040F6C410DFF87419086011E083
:10D78000DFF848090068C0F3C010002805D040F653
:10D79000C410DFF85C19086004E04FF47A60DFF829
:10D7A00050190860DFF81C050068DFF844190968A3
:10D7B000884206DBDFF838090068DFF808150860E2
:10D7C0000EE0DFF8000500681430DFF8F814086098
:10D7D00006E05FF40010002104F0DBF800F088FAA6
:10D7E00001BD0000102D0020752E00202C2D0020E2
:10D7F0001C2D0020D42C0020D82C0020642D0020CB
:10D80000B02C0020B82C002080B56420DFF83C1933
:10D810000860DFF8E8090068401DDFF8E0190860DB
:10D82000DFF888080078052818D0DFF8D4090068E8
:10D83000012803DB012000F0E3FB0AE0DFF8C00968
:10D840000068002803D5012000F0B3FB01E000F0E0
:10D850004FFA0020DFF8AC1908701DE2DFF8A409C8
:10D86000007800280ED0012841D0022800F09580D1
:10D87000032800F0B680052800F0E281072800F0B8
:10D880003B8101E20120DFF87C190870DFF8CC0948
:10D890000068401CDFF8C419086003F027FA00286C
:10D8A00008D1DFF82808006830F48070DFF81C1811
:10D8B000086007E0DFF81408006850F48070DFF8B3
:10D8C0000C18086002F0C6FA0020DFF894190870FE
:10D8D000012002F005F80020DFF8A4140860002001
:10D8E00006F0B2FD0020DFF87C190860D4E1652065
:10D8F000DFF8581808600220DFF86419087000206B
:10D90000DFF8F818086002F051FDDFF85C190968CB
:10D91000401A40F6A17188420AD30420DFF840196A
:10D92000087002F0A7F80220DFF8D81808702CE081
:10D93000DFF898070068C0F34010002804D1DFF832
:10D940004004006865280BDADFF880070068C0F340
:10D95000401000280CD0DFF828040068652807DB99
:10D96000DFF8E407006850F00070DFF8DC170860AB
:10D97000DFF8F8080068012807D1DFF8CC07006855
:10D9800050F04000DFF8C0170860DFF8BC070068FF
:10D99000002801D000F09CFB7EE1DFF86008006801
:10D9A00040F2D171884217DB0020DFF8B41808700C
:10D9B000DFF84808006840F6B931884210DB0320E0
:10D9C000DFF840180870002006F03EFD02F052F823
:10D9D000002001F085FF03E00420DFF884180870C0
:10D9E0005AE16620DFF8641708600220DFF870183B
:10D9F00008700020DFF80418086002F0D7FCDFF898
:10DA000068180968401A40F6A17188423FD3DFF8D0
:10DA1000BC060068C0F34010002813D0D848006846
:10DA200040F6AD51884208DBDFF81C07006850F073
:10DA30004000DFF81417086024E0D148006803F0C4
:10DA400049F91FE0CE480068C82808DADFF8F80670
:10DA5000006850F48020DFF8F016086012E0C84833
:10DA6000006840F61D41884208DBDFF8DC060068EC
:10DA700050F04000DFF8D016086003E0C0480068AE
:10DA800003F028F90720DFF87C1708702CE0DFF896
:10DA90003C060068C0F34010002804D1B848006874
:10DAA00010F1640F0BDBDFF824060068C0F34010B0
:10DAB00000280CD0B248006810F1640F07DADFF8D4
:10DAC0008806006850F00070DFF87C160860DFF808
:10DAD0009C070068012807D1DFF86C06006850F049
:10DAE0004000DFF864160860DFF85C060068002874
:10DAF00001D000F0EDFACFE04FF49670DFF8581740
:10DB0000086002F095F979490968884204DA002032
:10DB1000DFF8E81608608BE0DFF8E006006840F206
:10DB2000D171884264DB032006F039FEDFF8281744
:10DB3000096848434FF4FA61B0FBF1F1DFF83007B0
:10DB4000006801280BDB4FF47A704143DFF82007AF
:10DB5000006891FBF0F0DFF81C17086003E000207C
:10DB6000DFF810170860DFF80C070068002808D1FC
:10DB7000DFF8D405006850F04000DFF8CC150860ED
:10DB80002BE0DFF848050068C0F3C01000280ED075
:10DB9000DFF8E0060068B0F5FA6F08DADFF8A805EC
:10DBA000006850F04000DFF8A015086015E0DFF8CD
:10DBB0001C050068C0F3C01000280ED1DFF8B406C1
:10DBC000006840F69901884207DBDFF87C050068B1
:10DBD00050F04000DFF8701508600520DFF82416CB
:10DBE000087001F047FF0420DFF8741608701FE08A
:10DBF000032006F0D4FDDFF86016096848434FF4AF
:10DC0000FA61B0FBF1F1DFF87006006801280BDB68
:10DC10004FF47A704143DFF86006006891FBF0F042
:10DC2000DFF85016086003E00020DFF848160860AF
:10DC3000DFF814050068002801D000F049FA2BE055
:10DC4000DFF8B805006840F2D171884217DB002088
:10DC5000DFF80C160870DFF8A405006840F6B9314B
:10DC6000884210DB0120DFF8141608600120DFF87D
:10DC7000101608600E20DFF86C1A087003E004200C
:10DC8000DFF8DC15087007E0DFF8BC04006850F02E
:10DC90000800DFF8B414086001BD0000E02C00208B
:10DCA00080B55FF0FF30DFF8A41408600420DFF8CF
:10DCB000B0150870DFF8F4030078052801D000F0F3
:10DCC00017F801BD702D002080B501F0D3FE0B20A8
:10DCD000DFF8101A087002F069FBDFF80C1A086010
:10DCE0000420DFF87C15087001BD0000382D0020ED
:10DCF00080B50420DFF8681508700820DFF8E41903
:10DD000008700120DFF8E419086002F04FFBDFF82B
:10DD1000701A086001F0AEFE01BD80B50020DFF88A
:10DD2000401508700920DFF8BC19087001F0A2FE48
:10DD300001BD80B50420DFF8281508700020DFF849
:10DD4000A419087001F096FE4FF4C870DFF8341A79
:10DD5000086001BD80B50420DFF8041508700320B9
:10DD6000DFF88019087001F085FE0020DFF89014BC
:10DD700008604FF4C870DFF80C1A086001BD00009D
:10DD8000442D002080B501F075FE0120DFF8F81960
:10DD90000860012001F00CFCDFF8E00400680028B6
:10DDA00003D1012001F09CFD22E0DFF8E0090068CA
:10DDB000DFF8DC190860DFF8DC090078012811D1F0
:10DDC000C2480068C0F34010002805D07FF0A900C9
:10DDD000DFF82C1408600BE07FF06300DFF82014FC
:10DDE000086005E0DFF8B0090068DFF81414086087
:10DDF0000220DFF86C1408700420DFF8E8180870BF
:10DE0000DFF898090068DFF85C14086002F0CEFAC9
:10DE1000DFF88C19086001BDDC2C0020EC2C002000
:10DE2000BC2C002080B501F025FE0120DFF8581938
:10DE30000860002001F0BCFBDFF868090068642876
:10DE400004D0DFF83C040068002809D102F034FF58
:10DE5000DFF8541908606420DFF8481908600BE007
:10DE600002F02AFFDFF83C1909684843642190FB5F
:10DE7000F1F0DFF834190860DFF8040400680028C6
:10DE800003D1002001F02CFD1FE0DFF8000900683D
:10DE9000DFF8FC180860DFF8FC08007801280FD1D3
:10DEA0008A480068C0F34010002804D0AA20DFF898
:10DEB0005013086009E06420DFF84413086004E0B0
:10DEC000DFF8D4080068CE490860DFF8D808006899
:10DED00064280FD0DFF8C4080068DFF8CC180968A0
:10DEE000884207DBDFF898030068012802D1FFF7BA
:10DEF00031FF07E00220DFF8681308700120DFF827
:10DF0000E4170870DFF894080068DFF85813086019
:10DF100002F04CFADFF84C1C086001BD882D00208F
:10DF200080B50120DFF860180860162005F06CFB52
:10DF30000B2801DB0A2002E0012800DA01206349F6
:10DF40000968C1F34011002903D164214FF416720E
:10DF500002E0AA214FF4FA72521A092392FBF3F25B
:10DF6000401E00FB0210DFF830180860DFF82808B8
:10DF70000068A3490860DFF82C08006864280DD009
:10DF8000DFF818080068DFF820180968884205DB08
:10DF9000BB480068012801D1FFF7DCFEDFF8FC0771
:10DFA0000068B049086002F001FADFF8B81B0860A9
:10DFB00001BD10B5C0B2012804D101F072FEDFF836
:10DFC000EC170860DFF8D407046801F047FE241A54
:10DFD000DFF8DC070460DFF8D80700680A2803DAF6
:10DFE0000A20DFF8CC1708600720DFF8F816087061
:10DFF00002209B4908700020DFF86C1B086010BDF0
:10E0000010B5C0B2012804D101F04BFEDFF89C1717
:10E010000860DFF88807046801F020FE0419DFF8C3
:10E0200090070460DFF8800700680A38DFF880177F
:10E030000968884206DADFF8700700680A38DFF8F6
:10E04000701708600620DFF89C16087002208449CB
:10E0500008700020DFF8101B086010BD80B5052097
:10E06000DFF880160870DFF8340700687D49086023
:10E0700002F09CF9DFF8281708600020DFF8EC1A9E
:10E08000086001BD80B50220DFF858160870DFF87F
:10E090000C0700687349086002F088F9DFF8001780
:10E0A00008600020DFF8C81A086001BD6E2E00204D
:10E0B00080B504206A4908700D20DFF82816087022
:10E0C00000205049087001F0D5FC01BDB42C00209F
:10E0D00080B563480078022802D0FFF7F5FD06E01E
:10E0E00002205F4908700F20DFF8F815087001BDA5
:10E0F000B02D0020982D0020A186010080B50220BF
:10E100005749087001F0B6FC01F062FCDFF8801698
:10E110000860DFF8600A0068C0F34010002804D1EE
:10E120007FF063003649086003E0DFF84C0A3449A9
:10E13000086002F03BF9DFF8441A08601020DFF8AD
:10E14000A415087001BD0000A02D0020B02C0020F7
:10E1500080B5DFF82C0A0078012801D101F08DF894
:10E160003F480078DFF8181A097888423DD0DFF878
:10E17000040A006850F00200DFF8F8190860384817
:10E180000078042802D101F040F836E034480078E5
:10E19000002802D100F0D0FF2FE03148007803289A
:10E1A0000FD1DFF8DC090078042804D0DFF8D009AB
:10E1B0000078002802D101F004F81EE001F05DF8BB
:10E1C0001BE027480078022817D1DFF8B40900784F
:10E1D000042804D0DFF8A8090078002802D100F054
:10E1E000F0FF0AE000F0C9FF07E0DFF888090068E7
:10E1F00030F00200DFF87C19086001BD902D00208E
:10E200002C2D0020702E002080B5DFF868090068F2
:10E21000C0F34000002814D0DFF864090078042817
:10E2200007D1002300220121DFF85C0C03F031FC50
:10E2300011E0032306220121DFF84C0C03F029FC36
:10E2400009E0DFF83C090078042804D10121DFF857
:10E25000380C03F0A8FC01BDF82C0020A42D0020F0
:10E26000732E0020482D0020842D0020B82C002083
:10E27000642D0020F42C0020602D0020D02C0020E4
:10E28000CC2C002080B5DFF85C040078052840D154
:10E2900001F0D8FBDFF8F40B0168012001F040FE2B
:10E2A000DFF8F814096888421FDADFF8F01409680B
:10E2B000081ADFF8F814096800FB01F0400007F0C5
:10E2C0005FF85FF0FF314843DFF8C41B0968814203
:10E2D00002DADFF8BC0B0068DFF8BC14096888427A
:10E2E00006DADFF8B404006802E0DFF8A40B006887
:10E2F000DFF880180968C1F34011002905D101F049
:10E3000015FCDFF8401C0860EAE1DFF8381C086003
:10E31000E6E1DFF8D0030078022841D101F092FB5A
:10E32000DFF8240C0168DFF8640B00684118002056
:10E3300001F0F6FDDFF864140968DFF86C24126858
:10E34000121A914218DADFF860140968081ADFF827
:10E350004C140968401ADFF85414096800FB01F0F6
:10E36000400007F00DF8DFF830140968814206DA42
:10E37000DFF82404006802E0DFF8140B0068DFF81F
:10E38000F4170968C1F34011002905D101F0CEFB53
:10E39000DFF8B01B0860A3E1DFF8A81B08609FE16D
:10E3A000D0480078072828D101F04CFBDFF8EC03B7
:10E3B0000168DFF8FC030068081A01280BDBDFF8AE
:10E3C000EC13096800FB01F0400006F0D9FF5FF094
:10E3D000FF31484300E00020DFF898170968C1F3D7
:10E3E0004011002905D101F0A1FBDFF8581B08609E
:10E3F00076E1DFF8501B086072E1BA480078062821
:10E4000025D101F01FFBDFF8A8030168DFF88C03BA
:10E410000068081A012808DBDFF89013096800FB80
:10E4200001F0400006F0ACFF00E00020DFF84417E8
:10E430000968C1F34011002905D101F077FBDFF82D
:10E44000041B08604CE1DFF8FC1A086048E1A548AD
:10E450000078012813D0A34800780D2804D1DFF8F4
:10E46000780B007803280AD09E4800780D2840F0E9
:10E470009180DFF8640B0078072840F08B80DFF88C
:10E48000F4060068C0F34010002808D1DFF84C0BF8
:10E49000006801F04BFBDFF8481B086005E0DFF87F
:10E4A0003C0B0068DFF8381B0860002001F045FBDA
:10E4B000DFF8901A0968DFF8282B126891422EDAEB
:10E4C000DFF8201B0A68052101FB0020DFF8141B80
:10E4D0000860DFF8100B00684FF47A7190FBF1F0E0
:10E4E000DFF8601A0860DFF85C0A0068DFF8F01AED
:10E4F000096888420EDBDFF8E80A0068DFF8441A92
:10E500000860DFF8DC0A01684FF47A704143DFF8F5
:10E51000D40A01600120DFF81C1C0860E0E0DFF88D
:10E52000C01A0968DFF81C2A1268914224DADFF861
:10E53000B41A0A68052101FB1020DFF8A81A086048
:10E54000DFF8A00A00684FF47A7190FBF1F0DFF871
:10E55000F4190860DFF8EC090068012807DA0020E8
:10E56000DFF8E01908600020DFF8781A0860002062
:10E57000DFF8C01B0860B3E0DFF8640A01684FF4FD
:10E580007A704143DFF85C0A01600020DFF8A41BC9
:10E590000860A5E05348007804280DD05148007861
:10E5A0000D2804D1DFF8300A0078012804D04D4846
:10E5B0000078102840F08B80DFF8B8050068C0F3C1
:10E5C0004010002808D1DFF8140A006801F0AEFA04
:10E5D000DFF80C1A086005E0DFF8000A0068DFF8D1
:10E5E000001A0860012001F0A8FADFF8F4190968A0
:10E5F000DFF85029126891422EDADFF8E8190A682C
:10E60000052101FB1020DFF8DC190860DFF8D409D0
:10E6100000684FF47A7190FBF1F0DFF82819086078
:10E62000DFF8BC090068DFF81C19096888420EDBB6
:10E63000DFF8AC090068DFF80C190860DFF8A00902
:10E6400001684FF47A704143DFF8980901600120B6
:10E65000DFF8E01A086043E0DFF8E8180968DFF83F
:10E6600080291268914224DADFF878190A680521B6
:10E6700001FB0020DFF86C190860DFF8680900680A
:10E680004FF47A7190FBF1F0DFF8B8180860DFF80A
:10E69000B4080068002807D40020DFF8A818086034
:10E6A0000020DFF8401908600020DFF8881A0860B1
:10E6B00016E0DFF82C0901684FF47A704143DFF867
:10E6C000240901600020DFF86C1A086008E00548A2
:10E6D00000780F2802D101F0B5F901E001F0CAF984
:10E6E00001BD00006F2E00208C2D0020C02C0020CA
:10E6F00080B5DFF8DC0B00780F283FD0DFF8D00BB7
:10E7000000780D2804D1DFF8D0080078072835D02C
:10E71000DFF8BC0B0078012822D0DFF8B40B0078BA
:10E7200004281DD0DFF8A80B0078052818D0DFF8E2
:10E73000A00B0078022813D0DFF8940B007807288C
:10E740000ED0DFF88C0B0078062809D0DFF8800B9C
:10E750000078102804D0DFF8780B00780D2809D154
:10E7600000F0B8FD012802D100F00CFA06E000F03C
:10E7700021F803E00020DFF8DC1C086001BD000088
:10E780009C2D0020802D0020D82C0020182D00204A
:10E79000702D0020752E00200C2D0020442D00200F
:10E7A000942D0020202D0020502D0020042D00202D
:10E7B0004C2D002010B5DFF88C07006840F6E731DB
:10E7C000884205DB40F6E630DFF8781708600BE09A
:10E7D000DFF870070068DFF8C81B884204DADFF84A
:10E7E000C00BDFF860170860DFF8580701684FF4C6
:10E7F000FA60414340F6E63091FBF0F0DFF8A41BED
:10E800000860DFF840070168DFF89C0B0068091A10
:10E81000DFF8980B0160DFF8B80A0078012804D00F
:10E82000DFF8AC0A007804280BD101F001FBDFF817
:10E83000801B0968884208DA0020DFF8781B08602E
:10E8400003E00020DFF86C1B0860DFF8840A007822
:10E85000012822D0DFF8780A007804281DD0DFF8DC
:10E86000700A0078052818D0DFF8640A00780228BA
:10E8700013D0DFF85C0A007807280ED0DFF8500AC2
:10E880000078062809D0DFF8480A0078102804D05C
:10E89000DFF83C0A00780D2841D1B6480068C0F383
:10E8A000C000002810D1B3480068C0F380000028E1
:10E8B0000AD1DFF8E80C0168DFF8F00A00684118B7
:10E8C000DFF8D80C01602AE0AA480068C0F3800095
:10E8D00000280FD0DFF8D40A006800280AD5DFF836
:10E8E000BC0C0168DFF8C40A00684118DFF8AC0C02
:10E8F000016014E09F480068C0F3C00000280ED0FB
:10E90000DFF8A80A0068012809DBDFF8900C01682D
:10E91000DFF8980A00684118DFF8800C0160DFF822
:10E92000B009007805280ED0DFF8A4090078022885
:10E9300009D0DFF89C090078072804D0DFF8900997
:10E940000078062819D1DFF8640A006803F045FC56
:10E950000400DFF8480C006803F03FFC84420CD050
:10E96000DFF8380C0168DFF8340C0068042290FBF3
:10E97000F2F0091ADFF8240C0160DFF8280A0168B8
:10E98000DFF8280A02684FF4967042434FF47A7019
:10E9900092FBF0F04118DFF8040C026805204243B6
:10E9A0004FF47A7092FBF0F04118DFF8A80A01608A
:10E9B000DFF890050068002803D10020DFF8941AE2
:10E9C0000860DFF80C090078022835D16948006832
:10E9D000C0F3401000280FD1DFF8D4090068642884
:10E9E0000ADADFF8C0090068022190FBF1F0DFF8D5
:10E9F000641A0968814215DB5E480068C0F3401064
:10EA0000002858D0DFF8A8090068AA2853DADFF8F0
:10EA100094090068022190FBF1F0DFF8381A0968C8
:10EA2000814248DADFF87C090068022190FBF1F0AE
:10EA3000DFF8201A08603EE0DFF894080078052827
:10EA400039D14C480068C0F34010002811D1DFF8DC
:10EA50006009006810F1630F0BDBDFF848090068FC
:10EA60007FF0010190FBF1F0DFF8E81909688842B6
:10EA700017DB40480068C0F3401000281BD0DFF8C7
:10EA80003009006810F1A90F15DBDFF818090068DC
:10EA90007FF0010190FBF1F0DFF8B81909688842B6
:10EAA00009DADFF8000900687FF0010190FBF1F05E
:10EAB000DFF8A0190860DFF87C06006801281ED185
:10EAC000DFF890090068322809DADFF804080078D6
:10EAD000012804D13220DFF87C1908600FE0DFF84C
:10EAE0007409006810F1310F09DBDFF8E4070078E2
:10EAF000042804D17FF03100DFF8581908601D4860
:10EB0000006830F004001B4908601A48006830F0C3
:10EB1000080018490860DFF83C090068DFF8801A2F
:10EB200088420BDADFF8780ADFF828190860114804
:10EB3000006850F008000F49086011E0DFF8140980
:10EB4000006840F26D7188420ADB40F26C70DFF8B9
:10EB5000041908600748006850F00400054908607F
:10EB600010BD0000942D0020882D0020E02C0020F6
:10EB7000DC2C0020B42C002070FEFFFF982D00201C
:10EB8000742E002010B5DFF81C0A0068DFF8181A90
:10EB90000968884240DADFF8140A0068DFF8081ACA
:10EBA0000968884238D0DFF8000A0068DFF8F419F5
:10EBB0000968411A4FF47A704143DFF8EC090068A4
:10EBC00091FBF0F1DFF88C08006841434FF47A7054
:10EBD00091FBF0F0DFF87C180968081ADFF8741868
:10EBE0000860DFF87008006840F26D71884205DB4C
:10EBF00040F26C70DFF85C18086092E0DFF85408AF
:10EC00000068DFF89C19884280F28B80DFF8900959
:10EC1000DFF84018086084E0DFF88C090068DFF84E
:10EC200084190968B1F5C87188420FDBDFF87809EB
:10EC30000068DFF870190968884272DADFF86C0939
:10EC40000068DFF86419096888426AD1DFF858075C
:10EC5000006803F0C9FA0400BA48006803F0C4FA77
:10EC6000092148430A2190FBF1F084420CDADFF8D5
:10EC700034090168072041430A2091FBF0F0DFF8D6
:10EC800028190968814204DA0020DFF84C1C08606A
:10EC90002EE0DFF810090068DFF80C190968411A46
:10ECA0004FF47A704143DFF80009006891FBF0F1FE
:10ECB000DFF8A007006841434FF47A7091FBF0F051
:10ECC00003F092FA0A2800DA0A209E49096800290E
:10ECD00007D4DFF8801709684018DFF87817086054
:10ECE00006E0DFF870170968081ADFF8681708608F
:10ECF000DFF86007006840F26D71884205DB40F282
:10ED00006C70DFF8501708600BE0DFF84807006808
:10ED1000DFF88C18884204DADFF88408DFF834174B
:10ED20000860DFF884080068DFF880180860DFF802
:10ED3000A80B0068002824D101F038FBDFF8341C50
:10ED40000860804801684FF4FA60414340F6E630BD
:10ED500091FBF0F17B480068DFF84C261268821ABC
:10ED6000DFF8F0060068411A4FF47A7041434FF41F
:10ED7000967000FB1211052091FBF0F0DFF81C18D3
:10ED8000086010BD80B5DFF8400C007802287AD109
:10ED9000DFF8380C0068C0F30020002808D1DFF845
:10EDA000B406006810F5FA60DFF8301B086007E071
:10EDB000DFF8A0060068D0F5FA60DFF8201B0860D5
:10EDC000DFF8180B02684021DFF8A00C06F015FBF5
:10EDD000DFF8080B02688221DFF8900C06F00DFBCB
:10EDE000DFF870060068002824D4DFF8E00B006824
:10EDF000C0F3002000280ED14FF480724021DFF8CC
:10EE00006C0C06F046FB4FF400724021DFF85C0CFE
:10EE100006F039FB32E04FF400724021DFF84C0C71
:10EE200006F037FB4FF480724021DFF8400C06F00B
:10EE30002AFB23E0DFF8940B0068C0F300200028D1
:10EE40000ED14FF400724021DFF8200C06F021FBB8
:10EE50004FF480724021DFF8140C06F014FB0DE033
:10EE60004FF480724021DFF8040C06F012FB4FF4DF
:10EE700000724021DFF8F40B06F005FB0321DFF8F8
:10EE8000EC0B0160C04601BD00800340102D002046
:10EE9000082D002080B5012839D1052005F07FFC20
:10EEA00047F23051884217D24FF47F41DFF8440CCB
:10EEB00002F0CCF80221DFF8840B01F0BDF902204A
:10EEC000DFF87C1B0860DFF8040B006830F01000EE
:10EED000DFF8F81A086033E0DFF8F00A0068C0F3E2
:10EEE000001000282CD100F021FB0221DFF84C0B90
:10EEF00001F0DCF9DFF8780B01F0F0F9DFF8CC0A6B
:10EF0000006850F01000DFF8C41A086018E002280A
:10EF100016D14FF47F41DFF8DC0B02F097F80221A5
:10EF2000DFF8180B01F088F90020DFF8141B0860E7
:10EF3000DFF8980A006830F01000DFF8901A0860D7
:10EF400001BD0000302D0020142D002080B5E048C8
:10EF500000780F280ED1DFF8FC040068002804D0E8
:10EF60000420DFF8941B086034E00020DFF8881BE1
:10EF700008602FE0D648007805280BD0D4480078E8
:10EF8000022807D0D2480078072803D0D04800785C
:10EF900006281BD1032005F002FC4AF211418842E9
:10EFA00006D304220421DFF8940A01F019F911E0D4
:10EFB000032005F0F4FB4AF2280188420AD200221D
:10EFC0000421DFF8780A01F00BF903E00020DFF8F4
:10EFD000281B086001BD0000702E00202C2D002091
:10EFE000282D0020342D002080B5DFF8100B06F00E
:10EFF00079FADFF80C0B01F071F9DFF8080B01F07A
:10F000006DF9DFF8040B01F069F9DFF8000B01F08E
:10F0100065F90121DFF8F80A01F030F90221DFF883
:10F02000F00A01F02BF91021DFF8E80A01F026F9C7
:10F030002021DFF8E00A01F021F9DFF8DC2A402185
:10F04000DFF8280A06F0B6F9DFF8CC2A8021DFF8CD
:10F050001C0A06F0AFF9E020DFF8C01A0860B02003
:10F06000DFF8BC1A0860AA20DFF8B81A08604FF46D
:10F070007A624021DFF8F40906F0B2F94FF47A62BF
:10F080008021DFF8E80906F0ABF94021DFF8DC0960
:10F0900006F0B0F98021DFF8D40906F0ABF90321BE
:10F0A000DFF8C80906F0C8F95FF47020DFF8781AB5
:10F0B000086000220F21DFF8B40906F0D2F901221E
:10F0C0000F21DFF8A80906F0D5F900220F21DFF89B
:10F0D0009C0906F0B4F900220F21DFF8900906F030
:10F0E000B7F94FF4FA624021DFF8800906F085F99C
:10F0F0004FF4FA628221DFF8740906F07EF90E23DC
:10F100000E224021DFF8640906F089F90E230E2251
:10F110008021DFF8580906F082F90321DFF84C0955
:10F120000160C0464FF400724021DFF8400906F04C
:10F13000AAF901BDD42C002080B500220321DFF8FC
:10F140002C0906F07CF900220C21DFF8200906F0DA
:10F1500076F9FFF749FF0020DFF86C1808705C486B
:10F1600000780A2804D10520DFF88C1B086003E032
:10F170000020DFF8841B086001BD80B50022032158
:10F18000DFF8E80806F05BF900220C21DFF8DC0864
:10F1900006F055F9FFF728FF01220321DFF8CC081C
:10F1A00006F04DF901220C21DFF8C00806F047F9FE
:10F1B0000220DFF8141808700220DFF83C1B0860FA
:10F1C00001BD80B500220321DFF8A00806F037F961
:10F1D00000220C21DFF8940806F031F9FFF704FF54
:10F1E00001220221DFF8840806F029F90122082112
:10F1F000DFF8780806F023F90120DFF8CC17087053
:10F200000120DFF8F41A086001BD80B50022032157
:10F21000DFF8580806F013F900220C21DFF84C083B
:10F2200006F00DF90321DFF8E80801F005F83021B8
:10F23000DFF8E00801F000F800220121DFF8D00833
:10F2400000F0CEFF02220221DFF8C40800F0C8FF60
:10F2500000221021DFF8BC0800F0C2FF202220218C
:10F26000DFF8B00800F0BCFF0420DFF85C1708707E
:10F270000420DFF8841A086001BD80B5FFF7B4FEF2
:10F280004FF4FA624021DFF8E40706F0B6F84FF4D5
:10F29000FA628221DFF8D40706F0AFF80321DFF825
:10F2A000CC070160C04601220321DFF8C00706F049
:10F2B000C6F801220C21DFF8B40706F0C0F80320DD
:10F2C000DFF8041708700320DFF82C1A086001BD6E
:10F2D0006F2E002080B5DFF80006006800283ED1C0
:10F2E00001F064F8DFF88C160860DFF8100A006897
:10F2F00002280ED1DFF84C0B0068012809D1DFF895
:10F300000C0C0068012804D100F0C8FCA549086075
:10F3100004E0DFF8EC090068A249086025480068AD
:10F3200001280AD1DFF8A4060068C0F38010002885
:10F3300003D041F288309B4908609A480068012850
:10F340000BDB9848006898490968884205DA012073
:10F35000DFF884150860012020E000201EE0012075
:10F36000DFF874150860DFF8C40A0078102805D1AA
:10F37000DFF88C0900688B4908600EE0DFF87C0933
:10F380000068022804D100F089FC8649086004E086
:10F39000DFF86C09006883490860012002BD0000A5
:10F3A0001AF4FFFFB42D0020EC2C0020402D00208B
:10F3B000382D0020D82C002080B5DFF88C0A00689A
:10F3C000002807D1DFF8840A006850F00800DFF851
:10F3D0007C1A08600821DFF8780A00F005FF042194
:10F3E000DFF86C0A00F000FF0121DFF8240B02F0C7
:10F3F00035FB0121DFF8180B02F043FB0323062243
:10F400000121DFF80C0B02F044FB00230022012154
:10F41000DFF8FC0A02F067FB612301220121DFF81B
:10F42000F00A02F060FB0121DFF8E40A02F024FB9D
:10F4300000211F2006F00BFA0121DFF8D40A02F0A8
:10F4400010FB1F2006F014FA0121DFF8C40A02F0B5
:10F45000AAFB01BDF82C002080B5DFF8B80A06F041
:10F4600041F8422006F030FA0221DFF8480B02F0A2
:10F47000F5FA0221DFF83C0B02F003FB0021DFF874
:10F48000340B02F0C8FB0720DFF88C1A0860022159
:10F49000DFF8200B02F0ABFB4FF47A6340F67462A6
:10F4A0000021DFF8100B02F09AFB4FF47A6340F66C
:10F4B00074620121DFF8FC0A02F091FB41F61D5253
:10F4C0000021DFF8F00A02F084FB41F61D52012111
:10F4D000DFF8E00A02F07DFB2021DFF8D80A02F015
:10F4E00070FB03230F220221DFF8C80A02F0D1FAD1
:10F4F0005FF4002300220221DFF8B80A02F0F3FAD9
:10F50000DFF8183A01220221DFF8A80A02F0EBFA2C
:10F510000221DFF8A00A02F0AFFA422006F0A8F9B3
:10F520000221DFF8900A02F067FB01BD80B5DFF829
:10F53000880A05F0D7FF4FF47F41DFF8B80501F0E6
:10F5400085FDDFF8781ADFF8AC0501F088FDDFF8FB
:10F55000700A006830F40070DFF8641A08604FF435
:10F5600096524FF47F41DFF88C0501F0C1FD002277
:10F570004FF47F41DFF87C0501F0AEFD4FF4C86227
:10F580004FF47F41DFF86C0501F0C3FD4FF47F417C
:10F59000DFF8600501F054FD01BD00003C2D0020A6
:10F5A00094F8FFFF742D0020602D0020B82D00205E
:10F5B00010B50400E4B2002C03D1042004F024F8B8
:10F5C00002E0082004F020F8012801DA012002E01E
:10F5D0000B2800DB0A20DFF8F4130968C1F340119F
:10F5E000002919D1DFF8E4130968C1F3C01100291B
:10F5F00008D0E4B2002C02D14FF4C8720AE04FF4F4
:10F60000967207E0E4B2002C02D14FF4167201E0CA
:10F610004FF41672C82109E0E4B2002C02D141F681
:10F62000583201E040F6B8324FF44871521A401E89
:10F630004243092092FBF0F04118DFF8880901608D
:10F64000E4B2002C03D1062003F0DEFF02E00A2022
:10F6500003F0DAFF012801DA012002E00B2800DBC9
:10F660000A20DFF868130968C1F3401100290DD1A1
:10F67000DFF858130968C1F3C011002902D04FF414
:10F68000967201E04FF4C872C82103E04FF448714C
:10F6900040F6B832521A401E4243092092FBF0F065
:10F6A0004118DFF824090160E4B2002C03D11620D0
:10F6B00003F0AAFF02E0182003F0A6FF012801DAF8
:10F6C000012002E00B2800DB0A20C0490968C1F3D1
:10F6D000401100290AD1E4B2002C03D14FF4167274
:10F6E00064210DE04FF41672642109E0E4B2002CAD
:10F6F00003D14FF4FA72AA2102E04FF4C872AA2192
:10F70000521A092392FBF3F2401E00FB0211DFF8AC
:10F71000BC080160E4B2012C06D1DFF8B008006833
:10F720004042DFF8A8180860E4B2002C05D1102090
:10F7300003F06AFF0100491C04E0122003F064FF9B
:10F740000100491C002900D50021A0480068C0F331
:10F750004010002800D00A310A204143DFF8700829
:10F7600001605C2003F050FF0B2800DB0A200A2117
:10F770004843DFF860180860142006F0F5F9012806
:10F7800003D10020DFF84C180860E4B2002C03D14C
:10F79000002003F039FF02E0022003F035FF0428C7
:10F7A00001DB032002E0012800DA0120E4B2002C92
:10F7B0002BD186490968C1F34011002912D10328D1
:10F7C00004D13220DFF8101808604FE0022804D17D
:10F7D0002820DFF80418086048E01E20DFF8F8173A
:10F7E000086043E0032804D1AA20DFF8EC17086082
:10F7F0003CE0022804D19620DFF8DC17086035E0F1
:10F800008220DFF8D417086030E070490968C1F33E
:10F810004011002915D1032805D17FF03100DFF810
:10F82000B817086022E0022805D17FF02700DFF832
:10F83000A81708601AE07FF01D00DFF89C17086029
:10F8400014E0032805D17FF0A900DFF88C170860C9
:10F850000CE0022805D17FF09500DFF87C170860E6
:10F8600004E07FF08100DFF870170860E4B2002C3C
:10F8700007D10E2003F0C8FE4FF4FA6141F288323E
:10F8800006E00C2003F0C0FE4FF4FA6141F288322A
:10F890000B2801DB0A2002E0012800DA0120521ABD
:10F8A000401E4243092092FBF0F04118DFF82C077C
:10F8B0000160E4B2002C03D11C2003F0A5FE02E09D
:10F8C0001A2003F0A1FE1F2800DB1E2064214843FC
:10F8D000DFF80C17086010BDC82C0020BC2D0020DC
:10F8E0003A490968C1F3801100290ED0C0B200283E
:10F8F00005D141F28831DFF8082411600AE040F6B2
:10F90000B831DFF8FC23116004E040F6B831DFF8CD
:10F91000F0231160C0B2012811D12C480068C0F357
:10F920004010002805D07FF08100DFF8B81608608D
:10F930001FE07FF04F00DFF8AC16086019E02348A5
:10F940000068C0F34010002804D08220DFF894162D
:10F9500008600EE01D480068C0F38010002804D045
:10F960006420DFF88016086003E05020DFF874168A
:10F9700008607047842D002080B504F053FDDFF847
:10F980006816086000F0BEF9DFF860160860FCF742
:10F99000C9FDDFF85C160860FCF7A1FDDFF854161E
:10F9A000086000F004F8DFF85016086001BDDFF8C9
:10F9B0004C060168DFF840060268092000FB0211CE
:10F9C0000A2091FBF0F07047742E0020B42C002028
:10F9D00080B5042003F0E0FD00280AD05D2003F08C
:10F9E00013FE012801DA01200CE00B280ADB0A20B3
:10F9F00008E04FF4805003F0CFFD002801D00A202A
:10FA000000E00120DFF8F8150968C1F3C0110029F2
:10FA100009D0401E4FF416714843092190FBF1F0C4
:10FA200010F5167008E0401E40F24C414843092191
:10FA300090FBF1F010F52F7002BD00000070004047
:10FA4000087000400020DFF8BC1508600020DFF8D7
:10FA500094150860DFF8B0050068DFF8B01508609D
:10FA60000020DFF8AC1508607047000000800240FD
:10FA70000704030080B50020DFF888150860002027
:10FA8000DFF8601508600020DFF87C1508600020B2
:10FA9000DFF8781508600020DFF874150860002092
:10FAA000DFF87015086000F081FCDFF86C15086065
:10FAB0000020DFF8681508600020DFF86415086092
:10FAC0000020DFF8601508600020DFF85C15086092
:10FAD0000020DFF8241508600020DFF850150860CA
:10FAE00000F064FCDFF8481508600020DFF84415DA
:10FAF000086001BD00C0044010700040004000F0EC
:10FB000001000D0001040D000410010004140100A7
:10FB10000050064000500040BAAA05006080024034
:10FB2000A0800240288002401C8002404FF47A717D
:10FB30004843E32190FBF1F0704738B50400DFF84B
:10FB400084040568DFF8B8040068C0F3401000289A
:10FB500049D14FF48040002101F04CFF00220023E6
:10FB6000994201D1904205D040F2E930854201DB53
:10FB70004FF47A75DFF87C040068972802DAE4B263
:10FB8000012C0BD0DFF8B00400689638DFF864145D
:10FB90000968884208DAE4B2002C05D140F22D1041
:10FBA000854201DB4FF49675E4B2002C03D1A548E1
:10FBB0000068002807D0E4B2012C0FD1DFF84C0315
:10FBC000006800280AD1DFF838040068C0F3C010CC
:10FBD000002801D0C82501E04FF496752800FFF7F2
:10FBE000A5FF050038E04FF48040002101F002FF3E
:10FBF00000220023994201D1904202D0C92D00DB9E
:10FC0000C82509212000C0B200F08AF9DFF8E4130A
:10FC10000968884202DBE4B2012C07D0DFF8D41374
:10FC20000968814208DBE4B2002C05D140F22D10B6
:10FC3000854201DB4FF49675E4B2002C03D1814874
:10FC40000068002806D0E4B2012C05D1AF48006856
:10FC5000002801D140F26C75280032BD80B5DFF874
:10FC60009003006802F0C0FADFF894130968C1F34A
:10FC70004011002907D14043DFF84C1309684900BF
:10FC800090FBF1F009E040430A214843DFF83813C4
:10FC90000A6806214A4390FBF2F002BD40F66A2052
:10FCA000704780B5542003F0AFFC0100062901DB4A
:10FCB000052102E0012900DA0121DFF84403006890
:10FCC000C0F34010002804D14FF496704FF44872EE
:10FCD00002E0C8204FF4FA62121A491E01FB02F139
:10FCE000042291FBF2F10818B7490968884201DA49
:10FCF000B548006802BD0000FC2C0020242D002027
:10FD0000702D002080B504F06FFBDFF83013086021
:10FD1000DFF82803006844F62061884208D30020F9
:10FD2000DFF81C1308600020DFF81813087031E0BA
:10FD3000DFF814030068AC490968884208DA00203B
:10FD4000DFF8FC1208600120DFF8F812087021E0EB
:10FD5000A5480068BC490968884206DA0020B8490D
:10FD600008600220B749087014E0B5480068401CDC
:10FD7000B3490860B1480168B148026841F288306F
:10FD80004243914206D2AE48016841F28830414375
:10FD9000AA480160A9480068002805D0AB48A749D7
:10FDA0000968B0FBF1F001E040F6E630A5490978BA
:10FDB000002905D0A3490978A54A1278914201D0BB
:10FDC00000200AE09F490978012906D09D49097859
:10FDD000022901D1404200E0002001280CDB9D49AE
:10FDE0000968002916D09B4909682831814211DA37
:10FDF0009848006828300DE000280BD5954909681F
:10FE0000002907D0934909682839884202DA9148C5
:10FE1000006828388F490860734909688A4A116068
:10FE2000884909788A4A117002BD00006F2E0020AF
:10FE300073480068C0F34010002801D10A2000E098
:10FE400032207047CC2C002000C7FC43A02D00209E
:10FE500000C0054010B500F02BFF040000F042FF89
:10FE6000401E7D490860092C12D16548006830F0B9
:10FE70002000634908606248006830F04000604933
:10FE800008605F48006850F080005D4908603BE012
:10FE9000072C12D15A48006850F0200058490860D9
:10FEA0005748006830F040005549086054480068E1
:10FEB00030F080005249086026E0082C12D15048EA
:10FEC000006830F020004E4908604D48006850F04E
:10FED00040004B4908604A48006830F080004849BB
:10FEE000086011E04648006830F02000444908608E
:10FEF0004348006830F040004149086040480068CD
:10FF000030F080003E49086010BD0000D02C002079
:10FF100000800340013800F0C49F03402100090025
:10FF2000374A1268C2F34012002A40D00A2291FBDD
:10FF3000F2F2152A24DBC0B2002810D14749464806
:10FF400003685420434301EB0300006D4449424BD6
:10FF50001B6851F82310163A02FB010127E04149C2
:10FF60003D4803685420434301EB0300006D3C49C6
:10FF7000394B1B6851F82310163A02FB010116E0B9
:10FF8000C0B2002809D1354933480368542043439F
:10FF900001EB030050F8221009E032492E480368B3
:10FFA0005420434301EB030050F82210FFE7080000
:10FFB0007047000000900340025C00F0220A000439
:10FFC00004C00440002D0020042D00200C2D002032
:10FFD000102D0020142D0020082D0020182D0020A9
:10FFE0001C2D00202C2D0020E42C0020EC2C0020C7
:10FFF000382D0020442D0020642D0020602D00208D
:020000040001F9
:10000000B42C0020282D0020302D0020342D00207D
:10001000D42C0020D82C0020842D0020C82C0020B7
:100020003C2D0020402D0020F82C0020B82C002072
:10003000942D0020BC2C0020502D0020C02D00202D
:10004000C42D0020712E0020E82C0020C0270900BC
:10005000722E0020F02C0020542D0020B847020002
:10006000C84E0200B448020030B5CB4300F58064AE
:10007000D50725684CBF0D431D40256000F5846001
:10008000920747BF0268114301681940016030BD03
:1000900030B5CB4300F58164D50725684CBF0D43CF
:1000A0001D40256000F20444950725684CBF0D43B0
:1000B0001D40256000F20C44550747BF23681943D3
:1000C00021681940216000F5A760D10301684EBF87
:1000D00041F0010149084900016030BDF0B500243C
:1000E00000F6C4750126A640314211D066002F6883
:1000F0004FF0030C0CFA06FC27EA0C072F60C2F342
:100100004117D5F800C007FA06F646EA0C062E603D
:10011000641C082CE6DBCC4300F5A065D6072E68EE
:100120004CBF0E4326402E6000F2045596072E6801
:100130004CBF0E4326402E6000F5A16556072E6881
:100140004CBF0E4326402E6000F5A36516072E68AF
:100150004CBF0E4326402E6000F23C55D2062A6862
:100160004CBF0A4322402A60DD0700F20C5215689A
:100170004CBF0D432540156000F5A2629D07156830
:100180004CBF0D432540156000F214525D07156801
:100190004CBF0D432540156000F21C521D07156829
:1001A0004CBF0D432540156000F244529D05156873
:1001B0004CBF0D432540156000F5A86213F4407F45
:1001C000156814BF0D432540156000F5A560002B90
:1001D00007BF026841EA020401680C400460F0BDF8
:1001E00000EB81000260704738B501E038B50CE0E3
:1001F00004460D460022FFF737FF2946204601B08E
:10020000BDE830400023012268E704460D46022283
:10021000FFF72AFF2946204601B0BDE830400823F9
:1002200066225BE738B500F055F82946204601B054
:10023000BDE830400823E6E738B504460D460823FC
:10024000FFE70122FFF74AFF29462046BDE8384074
:10025000012209E738B500F01BF82946204601B015
:10026000BDE830400923CEE738B500F011F8294643
:10027000204601B0BDE830400823C4E738B500F09F
:1002800007F82946204601B0BDE830400823BAE708
:1002900004460D460222E7E638B5FFF7F9FF294686
:1002A000204601B0BDE830400A23ACE738B5FFF77F
:1002B000EFFF2946204601B0BDE830400823A2E701
:1002C00038B5FFF7E5FF2946204601B0BDE83040CC
:1002D000082398E704460D460022C5E610B50E4BEC
:1002E0000FF238021C68C0F30741CC40E40746BF58
:1002F00002EBC101496852F8311001F22C51020A97
:100300000B680F24944000F00F00A3439040184363
:10031000086010BD000000006CE00F40004000408D
:100320000080054000500040009005400060004003
:1003300000A005400070004000B0054000400240B1
:1003400000C005400050024000D00540006002405F
:1003500000E005400070024000F0054000D003407E
:100360000000064000100640001006400020064035
:1003700000200640003006400030064000400640A5
:100380000040064000500640005006400060064015
:100390000060064000700640007006400080064085
:1003A000008006400090064000900640DFF8F4040C
:1003B00000687047DFF8F014085C704780B5DFF81C
:1003C000EC040068C0F34000002810D1DFF8DC0422
:1003D000006850F00200DFF8D4140860FFF7E6FF71
:1003E000DFF8CC14086000F013F801F049F901BD02
:1003F000DFF8B8040068C0F340007047DFF8AC04D1
:10040000007810F001007047DFF8A804006870471A
:1004100080B50020DFF89C14086006F010FA002870
:1004200005D18021DFF88C04006806F0EFF901BDEA
:1004300080B5DFF880040068401CDFF8781408609D
:1004400006F0FDF9002805D18021DFF86804006876
:1004500006F0DCF9DFF85404006850F00200DFF821
:100460004C140860FFF7A2FFDFF84414086001F0A5
:1004700007F901BD80B505F0E3F94FF44040DFF81E
:100480003814086006F0EEF906F0F2F9DFF82C04F3
:1004900005F06CF8012005F065F8DFF8240405F09C
:1004A00021F8DFF8200405F01DF8DFF81C0405F042
:1004B00019F8DFF8180405F015F8DFF8140405F052
:1004C00011F8DFF8100405F00DF8DFF80C0405F062
:1004D00009F8DFF8080405F005F8DFF8040405F072
:1004E00001F8DFF8000404F0FDFFDFF8FC0304F07E
:1004F000F9FFDFF8F80304F0F5FFDFF8F40304F088
:10050000F1FFDFF8F00304F0EDFFDFF8EC0304F097
:10051000E9FFDFF8E80304F0E5FFDFF8E40304F0A7
:10052000E1FFDFF8E00304F0DDFF06F0F1F800285A
:1005300008D0DFF87803006840084000DFF86C134B
:10054000086007E0DFF86403006850F00100DFF89E
:100550005C13086004F0F6FF800704D50020DFF884
:100560005413086016E004228021DFF8480306F0E7
:10057000ECF8DFF84003006840F2E931884209D323
:100580000020DFF83013086004228021DFF8240304
:1005900006F0F0F8DFF8440305F0DCF8DFF830038C
:1005A00005F0D8F8DFF8600304F09CFF1E2005F08A
:1005B0008BF91F2005F088F9202005F085F921200E
:1005C00005F082F90021DFF8440301F024FB072045
:1005D000DFF83C13086005F039F84FF47A71B0FB8E
:1005E000F1F006F055F906F04DF900210F2005F065
:1005F0002EF90F2005F03CF9DFF8180304F072FF24
:10060000DFF8100304F088FF06F04AF9DFF808036A
:1006100006F05BF95FF0704004F064FF5FF080402B
:1006200006F0FCF9012803D15FF0804006F0EEF9F6
:10063000BA495FF080400160C0465FF0804006F03C
:10064000F4F95FF0804006F0D6F95FF0804006F0E4
:10065000F3F95FF0804006F0CDF95FF0804006F0DE
:10066000D0F905F0E9F801BD00B591B0AC4804F04F
:1006700039FFAC49AC4800F0F2FC01224FF6FF71A3
:10068000A94800F029FDA94AFF21A74800F030FD44
:10069000A64A4FF47F41A44800F02AFD6021702053
:1006A00005F0D5F80121A04800F03EFD702005F0CE
:1006B000DFF84FF6FF719C4800F0C2FC4022102189
:1006C000684606F042F80098452802D00098412874
:1006D0003BD10198312838D10298532805D002988F
:1006E000342802D0029878282FD103984C2802D0C1
:1006F0000398302829D10498002802D00498302883
:1007000023D10598002802D0059841281DD10698CC
:10071000002802D00698492817D10798002802D04F
:100720000798522811D1089800280ED1099800285E
:100730000BD10A98002808D10B98002805D10C98F5
:10074000002802D10D98002804D05FF4003001F099
:1007500037F903E05FF4003001F005F90E985249D3
:1007600008700F98504948704FF6FF7004F0EEFE85
:1007700011B000BD80B55FF0804006F04FF9012850
:1007800003D15FF0804006F041F969495FF0804095
:100790000160C0465FF0804006F033F95FF0004032
:1007A00001F01BF9002823D040480068C0F3400046
:1007B00000281DD106F010FA002819D108F0B2F96E
:1007C000002815D100F06AFA002811D108F032FB98
:1007D00000280DD108F0A4FD002809D102F027FF60
:1007E000002805D109F067F9002801D1FFF7E6FDDF
:1007F0002E480068C0F34000002844D0FBF72FFECD
:10080000502817D108F016FB002813D109F035FD48
:1008100000280FD10AF09BFD02280BD006F00FF83C
:10082000002807D109F047F9002803D100F036FA73
:10083000002808D0FFF7BAFD1D490968401A42F2A6
:10084000117188421AD3FFF7B1FD3A490968401A7D
:1008500065281CD304F0F4FF5FF0804006F0DEF85A
:10086000012803D15FF0804006F0D0F85FF07040BF
:1008700004F038FE304831490860FBE7FFF796FD89
:100880002C49086003E0FFF791FD2A49086001BD8B
:1008900029482A490860FBE702480068401C0149D2
:1008A000086070472C2E0020602E0020302E002083
:1008B000342E0020382E002008ED00E0800300C117
:1008C000000800F0010800F0020800F0030800F042
:1008D000040800F0050800F0060800F0070800F022
:1008E000080800F0090800F00A0800F00B0800F002
:1008F0000C0800F00D0800F00E0800F00F0800F0E2
:10090000100800F0005800F0003800F000800340AC
:10091000C48F0340000C00F0001800200008AF2F27
:10092000015C00F02222000400700340801A0600DF
:1009300000350C003C2E00200400FA050CED00E010
:1009400010B582B0DFF8DC06006840084000DFF830
:10095000D4160860202360226946DFF8CC0609F02F
:1009600010F80028F6D009F0A6F801280AD1FFF700
:100970001DFD0400FFF71AFD001B0228FAD308F042
:10098000A3FFF0E72021DFF8A00601F071F90128AC
:1009900010D1002004E00021DFF88C261154401C07
:1009A0002028F8D3DFF87C06006850F00200DFF85A
:1009B000741608602021DFF8700601F033F9002872
:1009C00003D14FF4804000F0FBFFDFF85C06007EAF
:1009D000092812D0DFF85006007E04280DD0DFF879
:1009E0004806007E082808D0DFF83C06007E07286D
:1009F00003D04FF4804000F0E3FF0020DFF82C1616
:100A00000860DFF82006006850F00100DFF81416D7
:100A1000086013BD80B5DFF80C060078C00740F110
:100A200016810BF0DFF9092880F2CF804FF4804067
:100A300000F099FF2021DFF8F00501F0F3F800281D
:100A400004D14FF4804000F0BBFF64E0DFF8D8052C
:100A5000007E092813D0DFF8D005007E04280ED0D0
:100A6000DFF8C405007E082809D0DFF8BC05007E49
:100A7000072804D04FF4804000F0A2FF4BE01E2076
:100A800002F0C2FDDFF8A015097E884204D04FF4C1
:100A9000804000F095FF3EE0DFF88C0500680028FC
:100AA00004D14FF4804000F08BFF34E0DFF878058C
:100AB0000068DFF874154968C943884204D04FF4D0
:100AC000804000F07DFF26E0DFF85C05007F032812
:100AD00004DB4FF4804000F073FF1CE0DFF84805B2
:100AE000407F022804DB4FF4804000F069FF12E0F1
:100AF000DFF83405C07E022804DB4FF4804000F0AC
:100B00005FFF08E0DFF82005807F032803DB4FF458
:100B1000804000F055FF4FF4804000F05EFF002859
:100B20004BD14FF4805000F01EFF5FF0004002F008
:100B300033FD002804D1DFF8F004C07E00280AD17C
:100B40005FF0004002F028FD002809D0DFF8D8044B
:100B5000C07E002804D14FF4805000F031FF38E00F
:100B60004FF4007002F018FD002804D1DFF8B8043B
:100B7000407F00280AD14FF4007002F00DFD0028DC
:100B800009D0DFF8A404407F002804D14FF480503E
:100B900000F016FF1DE05E2002F036FDDFF888143D
:100BA000897F884215D01E2002F02EFD072810D123
:100BB0004FF4805000F004FF0BE04FF4805000F041
:100BC000D2FE202000F0CFFE03E04FF4805000F072
:100BD000CAFEDFF850040068C0F3400000280FD0C0
:100BE00020226021DFF8400408F012FF012807D11D
:100BF000DFF83004006830F00200DFF828140860E5
:100C00000BF0F0F8C0B209281FD1FFF7F1FB012863
:100C100005D1202000F0D4FE0BF0EFF817E0DFF84C
:100C20000C040068002802D100F076F80FE0DFF82D
:100C3000FC030068012802D100F049F907E0082010
:100C400000F0BEFE0BF0D9F801E000F0DCF901BDC8
:100C5000DFF8D8030068002807D1DFF8C803006870
:100C600050F00400DFF8BC1308607047DFF8B403ED
:100C70000068C0F380007047002004E00021DFF826
:100C8000A8231154401C2028F8D3DFF898030068EB
:100C900050F00200DFF88C1308607047DFF884031F
:100CA000007810F00A0F01D0012000E0002070470A
:100CB000DFF87403007E704780B54FF4804000F089
:100CC0008CFE002803D1DFF86003006801E05FF0CC
:100CD000FF3002BDDFF850130860C043DFF848134F
:100CE00048607047DFF84003807F7047DFF83803C3
:100CF000C07E002801D1002000E00120704780B5AF
:100D00000BF0CEF9FFF752FBDFF824130860002048
:100D1000DFF81813086001BD10B580200BF0E6FD68
:100D20000BF063F804005FF40000002100F031FED6
:100D30000023002200210020FBF76FFB01200AF0B6
:100D400002FBB8480068C0F38000002813D1FFF709
:100D50002DFBB7490860E4B2012C01D10BF04DF82E
:100D60004FF4804000F039FE002800F0AF802020D2
:100D700000F0F9FDAAE0FFF719FBAD490968401A38
:100D800041F28931884234D2E4B2022C31D0E4B24B
:100D9000012C2ED0A7480EF08AFE002829D15FF042
:100DA00001500EF084FE002823D1A3480EF07FFEF0
:100DB00000281ED11E2002F027FC09280ED01E207C
:100DC00002F022FC042809D01E2002F01DFC082895
:100DD00004D01E2002F018FC07280AD14FF48040EE
:100DE000002100F007FE00220023994201D1904229
:100DF00009D08C48006830F004008A49086020203F
:100E000000F0DEFD62E0FBF72AFB50285ED185484A
:100E1000006830F00400834908605FF0FF3000F0A4
:100E2000A2FD8048006850F002007E490860002062
:100E300003E000217C4A1154401C2028F9D31E20D5
:100E400002F0E2FB784908765E2002F0DDFB76498D
:100E500088775FF0004002F09FFB002807D07248BF
:100E6000007E062803D001206F49C87602E00020EA
:100E70006D49C8764FF4007002F08EFB002807D051
:100E80006948007E062803D001206749487702E0C0
:100E9000002065494877022002F07EFB002803D13C
:100EA00002206149087702E001205F4908770022AB
:100EB0000021092007F00DFDFFF778FA5C49086072
:100EC00001200AF040FA01205849086010BD10B511
:100ED0000AF08BFF04005FF40000002100F081FDA8
:100EE000FBF7BDFA652803D181200BF0FFFC06E07B
:100EF000FBF7B5FA662802D182200BF0F7FC0AF066
:100F000026FA02280ED00AF022FA012803D15FF453
:100F1000000000F055FD0023002200210520FBF712
:100F20007CFA05E00023002200210020FBF775FA7F
:100F3000E4B2012C05D1202000F042FD0AF05DFF53
:100F400060E0E4B2022C20D03A480EF0B0FD002858
:100F50001BD15FF001500EF0AAFD002815D13648D4
:100F60000EF0A5FD002810D14FF48040002100F0C4
:100F700041FD00220023994207D1904205D1294822
:100F80000068C0F38000002805D0202000F018FD84
:100F900000F039F836E0294800F01FFD002802D0A3
:100FA00000F031F82EE0FBF75AFA10F1010F29D1C9
:100FB000022002F0F1FA002803D102201A49087732
:100FC00002E00120184908774FF4007002F0E4FABB
:100FD000002803D001201449487702E0002012497C
:100FE00048772021104800F033FE0E48006850F08A
:100FF00002000C4908605FF40000002100F0C9FC09
:101000000AF0FBFE10BD80B5FFF7D0F90849086073
:101010000020064908600348006830F004000149D8
:10102000086001BD202E00208C290020242E0020E5
:10103000282E002040000080800000405881A66AD1
:1010400050F80C3F40F20112114042E050F80C3FC2
:1010500040F20112114023EA010101607047F0B52E
:1010600000F10C03164A1C68124D144F14401C600A
:101070000A0E026000F108032E680F4A001D164098
:10108000BE4201F0FF040BD10D0905F470452C435D
:1010900044F4007404604FF2FF0000EA112004E001
:1010A00044F400740460C1F3072040F40070186039
:1010B000F0BD000000E00F400000FF7000000A10CB
:1010C000FEFEFFFF40F60C43194050F80C3F8B43E7
:1010D000114019430160704740F2022319400C305F
:1010E000002A026814BF114322EA0101016070471F
:1010F0000B061CBF00F128031A6011F47F4F18BFC4
:1011000040F82C2F7047FF290CBF28302C30006886
:1011100070470B061CBF00F130031A6011F47F4FBB
:1011200018BF40F8342F704750F8182F1143016052
:10113000704740F8241F704780B50020DFF8341650
:101140000860DFF83406DFF834160860FF20DFF8A7
:10115000301608600121DFF82C06FFF76DF8082330
:1011600001220121DFF81C06FEF7B8FF0020DFF89E
:101170001816086010215FF04020FFF75DF800208E
:10118000DFF808160860DFF8080604F0ABF9DFF8AE
:10119000000604F0C1F9DFF8FC05FFF79FF8DFF85F
:1011A000F805FFF79BF80C21DFF8F005FFF788F84A
:1011B00004F04CFA010060235FF4E132DFF8E0054F
:1011C0000FF0D2F910220221DFF8D4050FF0C8F990
:1011D000DFF8D005006830F01000DFF8C8150860AF
:1011E0001021DFF8BC050FF012FADFF8B4050FF09C
:1011F000EAF90321DFF8A8050FF017FADFF8A805D0
:1012000005F0D4FBDFF8A40505F0D0FBA0214D20AC
:1012100004F01DFB4D2004F02BFB0F21062005F0F0
:1012200057FBDFF88C15062005F065FB00F075FA1A
:101230000F21072005F04CFBDFF87815072005F09B
:101240005AFB0020DFF8701508600020DFF86C15ED
:1012500008700020DFF8641548700020DFF85C1586
:101260008870DFF85C05006850F40020DFF8501546
:101270000860DFF84C05006850F08070DFF840151A
:101280000860DFF83C05006850F48030DFF8301566
:101290000860DFF82C05006850F40010DFF8201516
:1012A00008600020DFF81C1508600020DFF8181522
:1012B00008600020DFF8141508600020DFF8101522
:1012C00008600120DFF8AC14086001BD80B5DFF8CC
:1012D000A404006800282CD04FF4007002F05CF9E0
:1012E000002818D1DFF8D8040068000C0004DFF8EB
:1012F000D01408600020DFF8CC1408600020DFF86C
:10130000B81408600020DFF8C81408605FF00060BF
:1013100000F029FB0DE0DFF8A8040068002804D0E5
:101320005FF0006000F04CFB03E05FF0006000F055
:101330001AFB01BD80B5DFF83C040068012840F0CD
:101340001B8180234FF48072DFF88814DFF8880453
:1013500005F049FD012840F0E880DFF864040068EA
:1013600030F40010DFF858140860DFF868044078A3
:10137000002824D00020DFF8441488700020DFF813
:101380003C1408700020DFF834144870DFF8300493
:10139000006850F40020DFF828140860DFF820040B
:1013A000006850F08070DFF8181408600020DFF843
:1013B000141408600020DFF800140860DCE0DFF897
:1013C00014048078C02863D10020DFF8EC13086093
:1013D000DFF80004C078872839D18720DFF8DC13D4
:1013E0008870DFF8DC03006830F40020DFF8D013E9
:1013F0000860DFF8E0034079DFF8C0130870DFF819
:10140000D4038079DFF8B4134870DFF8B0030078B4
:1014100033280CD1DFF8A4034078312807D1DFF856
:10142000A003006830F08070DFF8941308604FF478
:10143000007002F0B1F8002804D10020DFF8841316
:10144000086099E00120DFF87C13086094E0002038
:10145000DFF8681388700020DFF860130870002040
:10146000DFF858134870DFF85803006850F4002084
:10147000DFF84C130860DFF84803006850F0807014
:10148000DFF83C1308600020DFF83813086073E0D1
:10149000DFF840038078C2286ED1DFF824030068AB
:1014A000000C0004DFF818130860DFF8240300685C
:1014B000002814D1DFF808030168DFF81803007969
:1014C0000143DFF8FC020160DFF8F4020068DFF896
:1014D0000413497950EA0120DFF8E4120860DFF8CC
:1014E000E0020068800502D50020B6490860B948CE
:1014F000C078002809D10020AF490860B0480068D2
:1015000030F48070AE49086036E0AB480068401C9B
:10151000A9490860A84800680B282DD3A84800688E
:1015200050F48070A649086026E0022815D1A4482E
:10153000006830F40010A24908609F480068401C11
:101540009D4908609C4800680B2815D39C4800689A
:1015500050F480709A4908600EE097480068401C7B
:101560009549086094480068022805D394480068AB
:1015700050F400109249086001BD10B57D48006824
:10158000012871D18F480068012848D1082093496B
:101590000870002091494870C12090498870FAF77E
:1015A0008EFF8E49C870FAF7E3FF8C49087101007D
:1015B000090A8A4A51710100090C884A9171000E8A
:1015C0008649C8710024FAF7E3FF012801D154F0DD
:1015D00001047E480068012808D1FAF740FF50282E
:1015E00004D154F00204002078490860784800686B
:1015F000012808D1FAF733FF502804D154F004042D
:1016000000207349086075480472002073494872CD
:101610007349724805F061FC00F09CF827E0052052
:101620006E49087000206D494870C0206B49887071
:101630000420C0466949C8706848C078C0436749FB
:1016400008713320654948713120644988716449C3
:10165000624805F042FC00F07DF800205C4908601B
:1016600000205A49086002E0082000F0A9F910BDE6
:1016700052488078872801D0002000E00120704780
:1016800080B54E488078002809D04FF4007001F0F2
:1016900083FF002803D001204C49086002E00020AD
:1016A0004A49086001BD4549C0B2085C704780B531
:1016B0004FF4007001F070FF002801D1002001E01C
:1016C0003F48006802BD00203D49086001204049B4
:1016D0000860704780B53A48006800F0F0FAC830FA
:1016E00002BD80B501212E480EF096FF01002C4866
:1016F0000EF098FF34480068002807D1062005F056
:1017000041F9002808D100F008F805E035480068E4
:10171000800601D500F001F801BD80B500202A49FE
:101720000860062005F0C9F8002003E000212A4ADD
:101730001154401CB0F5807FF8D34FF480700090B6
:10174000254B174A0121062005F0E1F8062005F097
:10175000ACF801BD80B501211B4A11600090104B0F
:101760001F4A0121072005F0D2F8072005F09DF857
:1017700001BD0000E82A00204B434F4C2055024099
:1017800024550240005002400450024040400040B6
:10179000051800F001080800010C080000D0034003
:1017A000001001402C10014006000200070002005A
:1017B0000080000C008000C0FC2A0020F82A0020D5
:1017C000002B0020F02A0020EC2A0020F42A002020
:1017D000C42A0020D8240020801900205825002089
:1017E000801A00203C10014000209249086000202F
:1017F0000021914AC2E900010020904908600020C0
:101800008F49086000208F490860704770B589488B
:101810000068002804D0012100200FF0A6F815E090
:101820008548D0E90001884A0F2310401940002262
:101830000023994201D1904204D0022100200FF0F0
:1018400094F803E0002100200FF08FF808F038F83A
:10185000012803D15FF4002000F0A6F87548016864
:101860007A48014073480160FAF71EFE7149096821
:1018700008437049086002F0F5FD012807D1FAF726
:10188000F6FD012803D14FF4004000F099F8FEF76F
:10189000AFFD002866D1002426E066480068284293
:1018A00021D16648006828421DD0280000F0A8F821
:1018B00001000022052007F00CF8012813D15F4831
:1018C000006830EA05055D4805600CE00020020074
:1018D0003100042006F0FDFF012804D157480068BC
:1018E000054356480560641C202C1FD20125A540E5
:1018F000504800682842D0D0504800682842CCD1D7
:10190000280000F07DF806001D2E07D1FFF7E2FE4B
:10191000C82801D3C838DAE70020D8E7012ED5D18E
:101920004848006800F0CBF9401CD0E74248D0E9B5
:101930000001800311D54248006880030DD40022C5
:101940003C210C2006F0C5FF01280BD13C48006863
:1019500030F400303A49086004E03748D0E900012B
:101960003749086070BD80B539490140314A126875
:1019700032EA01012F4A116010F1010F08D1FFF77F
:10198000A2FEFAF78CFD02F074FD00202D490860DC
:1019900001BD294AD2E9002332EA000033EA0101FD
:1019A000254AC2E9000170472249096851F0100137
:1019B000204A11602349096808432249086070479A
:1019C0001C49096808431B490860704780B51D48D9
:1019D000006800F074F9401C02BD1649096808400F
:1019E0007047154AD2E9002310431943124AC2E94D
:1019F00000017047104AD2E9002310401940704797
:101A000080B500F05CF9202802D21249085C00E0A1
:101A1000002002BD80B5084AD2E9002310401940D9
:101A200000F0CFF9402802D20B49085C00E000200A
:101A300002BD0000C82B0020C82A0020CC2B0020AB
:101A4000D02B0020D42B0020FCFFFF7FBFFFFBFD2D
:101A5000F7FFFDFF7C4E0200B84C020050F8082F43
:101A600010E0012202FA01F100F10C021160CAE05B
:101A7000012202FA01F1CBE00268012303FA01F12D
:101A8000C3E00268012303FA01F122EA01010160C7
:101A90007047F0B500F1140689000F258D403468B9
:101AA000ED4302F00F0705EA040C07FA01F444EADB
:101AB0000C04346003F0030300F1200403FA01F185
:101AC00026683540BF1F2943032F21600AD8FF0035
:101AD00050F81C1F3023BB4002F030029943BA403B
:101AE0000A430260F0BD70B5490140310818920008
:101AF0000F2191400468C94303F00F050C40954045
:101B00002C430460C3F3032600F1180496402568B3
:101B10000D4035432560041DC3F3031600F01EF885
:101B200000F11C04C3F3035600F018F8012494409C
:101B300013F4702F00F110050BD050F8146FC3F39D
:101B40000243314003FA02F20A4302602868044368
:101B500002E0286820EA04042C6070BD25680D406E
:101B60009640354325607047012202FA01F140F8A2
:101B7000101F7047012202FA01F140F8181F704748
:101B800030B5490140310B1803F1080100200C3336
:101B90001C68E50506D408283EBF0C6842F8044BD3
:101BA000401CF5D330BD10B50B0C012401F00F0122
:101BB00050F8282F04FA01F141EA03411143016072
:101BC00010BD002200E0521C4908FCD140F8302F23
:101BD000704700EB810000F560600260704700EB29
:101BE000810000F5646042EA03420260704750F8E9
:101BF000082F4FF4803346E750F8082F4FF4803316
:101C000003FA01F101E050F8082F11430160704719
:101C100040F80C1F704750F8382F920841EA8201B3
:101C20000160704710B40122002302E0C45C121965
:101C30005B1C4C1EA342F9D3D243084410F8010C9C
:101C4000D2B2824201D0002000E0012010BC7047D7
:101C500010B40122002302E0C45C12195B1C4C1E6C
:101C6000A342F9D3D243084400F8012C10BC7047BA
:101C7000002200E0521CD2B28A4205D2D2B2835C6A
:101C8000FF2BF7D0002000E0012070470021C0B2F8
:101C9000B0F130010A2902D23038C0B208E0C0B237
:101CA000B0F14101062902D23738C0B200E000206D
:101CB000704710F00F00DFF8EC15085C7047002843
:101CC00001D120207CE0C10701D5002078E0810708
:101CD00001D5012074E0410701D5022070E0010721
:101CE00001D503206CE0C10601D5042068E081061F
:101CF00001D5052064E0410601D5062060E001061B
:101D000001D507205CE0C10501D5082058E0810518
:101D100001D5092054E0410501D50A2050E0010514
:101D200001D50B204CE0C10401D50C2048E0810412
:101D300001D50D2044E0410401D50E2040E001040E
:101D400001D50F203CE0C10301D5102038E081030C
:101D500001D5112034E0410301D5122030E0010308
:101D600001D513202CE0C10201D5142028E0810206
:101D700001D5152024E0410201D5162020E0010202
:101D800001D517201CE0C10101D5182018E0810100
:101D900001D5192014E0410101D51A2010E00101FC
:101DA00001D51B200CE0C10001D51C2008E08100FA
:101DB00001D51D2004E0400001D51E2000E01F20B9
:101DC000704730B400220023994203D1904201D1E0
:101DD0004020FCE10200D20701D50020F7E102001B
:101DE000920701D50120F2E10200520701D502203D
:101DF000EDE10200120701D50320E8E10200D2065E
:101E000001D50420E3E10200920601D50520DEE1C0
:101E10000200520601D50620D9E10200120601D5C2
:101E20000720D4E1C20501D50820D0E1820501D503
:101E30000920CCE1420501D50A20C8E1020501D5FF
:101E40000B20C4E1C20401D50C20C0E1820401D5FD
:101E50000D20BCE1420401D50E20B8E1020401D5F9
:101E60000F20B4E1C20301D51020B0E1820301D5F7
:101E70001120ACE1420301D51220A8E1020301D5F3
:101E80001320A4E1C20201D51420A0E1820201D5F1
:101E900015209CE1420201D5162098E1020201D5ED
:101EA000172094E1C20101D5182090E1820101D5EB
:101EB00019208CE1420101D51A2088E1020101D5E7
:101EC0001B2084E1C20001D51C2080E1820001D5E5
:101ED0001D207CE1420001D51E2078E1002801D5BB
:101EE0001F2074E110F0000211F00103002400250E
:101EF000AB4201D1A24201D0202068E110F00002E3
:101F000011F0020300240025AB4201D1A24201D00E
:101F100021205CE110F0000211F0040300240025F0
:101F2000AB4201D1A24201D0222050E110F00002C8
:101F300011F0080300240025AB4201D1A24201D0D8
:101F4000232044E110F0000211F0100300240025CA
:101F5000AB4201D1A24201D0242038E110F00002AE
:101F600011F0200300240025AB4201D1A24201D090
:101F700025202CE110F0000211F040030024002580
:101F8000AB4201D1A24201D0262020E110F0000294
:101F900011F0800300240025AB4201D1A24201D000
:101FA000272014E110F0000211F4807300240025B2
:101FB000AB4201D1A24201D0282008E110F000027A
:101FC00011F4007300240025AB4201D1A24201D0DC
:101FD0002920FCE010F0000211F4806300240025A9
:101FE000AB4201D1A24201D02A20F0E010F0000261
:101FF00011F4006300240025AB4201D1A24201D0BC
:102000002B20E4E010F0000211F48053002400259E
:10201000AB4201D1A24201D02C20D8E010F0000246
:1020200011F4005300240025AB4201D1A24201D09B
:102030002D20CCE010F0000211F480430024002594
:10204000AB4201D1A24201D02E20C0E010F000022C
:1020500011F4004300240025AB4201D1A24201D07B
:102060002F20B4E010F0000211F48033002400258A
:10207000AB4201D1A24201D03020A8E010F0000212
:1020800011F4003300240025AB4201D1A24201D05B
:1020900031209CE010F0000211F480230024002580
:1020A000AB4201D1A24201D0322090E010F00002F8
:1020B00011F4002300240025AB4201D1A24201D03B
:1020C000332084E010F0000211F480130024002576
:1020D000AB4201D1A24201D0342078E010F00002DE
:1020E00011F4001300240025AB4201D1A24201D01B
:1020F00035206CE010F0000211F48003002400256C
:10210000AB4201D1A24201D0362060E010F00002C3
:1021100011F4000300240025AB4201D1A24201D0FA
:10212000372054E010F0000211F0807300240025E5
:10213000AB4201D1A24201D0382048E010F00002A9
:1021400011F0007300240025AB4201D1A24201D05E
:1021500039203CE010F0000211F0806300240025DB
:10216000AB4201D1A24201D03A2030E010F000028F
:1021700011F0006300240025AB4201D1A24201D03E
:102180003B2024E010F0000211F0805300240025D1
:10219000AB4201D1A24201D03C2018E010F0000275
:1021A00011F0005300240025AB4201D1A24201D01E
:1021B0003D200CE010F0000011F0804100220023CF
:1021C000994201D1904201D03E2000E03F2030BC36
:1021D0007047012111FA00F07047002801D4012056
:1021E00001E05FF0FF307047002801D54042FFE773
:1021F0007047C0B230380A2801D2012000E0002028
:10220000704730B43C22B0FBF2F33C2202FB1300D7
:1022100008603C20B3FBF0F43C2000FB14334B601F
:102220001820B4FBF0F2182000FB12448C60101D43
:102230000723B0FBF3F403FB1400886102F2DB22F6
:1022400040F2B550B2FBF0F340F2B55000FB132062
:102250003C2802D35B1C0C2400E00224D01A40F27C
:102260006D15B0FBF5F0443048614D69443D40F2D6
:102270006D1000FB1522D21A002000E0401CA04285
:1022800004D2094B53F820309A42F7D2431E0B6117
:10229000054B03EB800050F8040C121A521CCA6064
:1022A00030BC7047B84E0200384D020070B58AB09D
:1022B00005005FF000465FF0804469463000FFF79C
:1022C000A0FF6946280000F01BF80DE0361B02E075
:1022D0000128FBDBA619640869463000FFF791FF6F
:1022E0006946280000F00CF8002801D0002CEFD13E
:1022F000002801D1300001E05FF0FF300AB070BD6E
:102300004A6943699A4201DA012048E042694B690F
:102310009A4202DA5FF0FF3041E00A6903699A42AB
:1023200001DA01203BE002690B699A4202DA5FF0B0
:10233000FF3034E0CA68C3689A4201DA01202EE017
:10234000C268CB689A4202DA5FF0FF3027E08A6801
:1023500083689A4201DA012021E082688B689A4200
:1023600002DA5FF0FF301AE04A6843689A4201DA05
:10237000012014E042684B689A4202DA5FF0FF30B5
:102380000DE00A6803689A4201DA012007E000685C
:102390000968884202DA5FF0FF3000E000207047F1
:1023A00080B5DFF80008006840084000DFF8F41747
:1023B0000860DFF8F007006830F00200DFF8E4178B
:1023C0000860DFF8E007006830F00400DFF8D41799
:1023D0000860DFF8D007006830F00800DFF8C417A5
:1023E00008600020DFF8C01708600020DFF8BC1785
:1023F00008600020DFF8B8170860DFF8A807006859
:1024000030F00200DFF89C170860DFF898070068DA
:1024100030F00400DFF88C170860DFF888070068E8
:1024200030F00800DFF87C170860DFF878070068F4
:1024300030F01000DFF86C170860DFF868070068FC
:1024400030F02000DFF85C170860DFF858070068FC
:1024500030F04000DFF84C17086020234FF4807202
:10246000DFF84417DFF8940907F08BFA0028F4D05E
:1024700007F021FB012802D107F026FAF8E7202314
:102480004FF49072DFF82417DFF8280707F079FA85
:102490000028F4D007F00FFB012802D107F014FA4E
:1024A000F8E720234FF4A072DFF80417DFF80807DD
:1024B00007F067FA0028F4D007F0FDFA012802D1EE
:1024C00007F002FAF8E76021DFF83009FFF7D0FBE8
:1024D000012808D1002200211E2001F02EF9012040
:1024E00001F004F8B4E02021DFF81009FFF79AFBAF
:1024F000002804D15FF40010FFF762FAA8E0202161
:10250000DFF8B006FFF78EFB002804D15FF400105F
:10251000FFF756FA9CE02021DFF89C06FFF782FBCC
:10252000002804D15FF40010FFF74AFA90E01E2063
:1025300001F06AF809281FD01E2001F065F8042870
:102540001AD01E2001F060F8082815D01E2001F0D6
:102550005BF8072810D05FF40010FFF731FA002273
:1025600009211E2001F0E9F8002000F0BFFF012240
:1025700000211E2001F0E1F8542001F045F8062862
:1025800003D30121542000F01BFB562001F03CF83E
:10259000032803D30121562000F012FB572001F03D
:1025A00033F8102803D30121572000F009FB5820ED
:1025B00001F02AF8022808D0582001F025F8012857
:1025C00003D00121582000F0FBFA5D2001F01CF837
:1025D0000B2804D25D2001F017F8002803D1012157
:1025E0005D2000F0EDFA5E2001F00EF8032803D321
:1025F00001215E2000F0E4FA5C2001F005F80B28D0
:1026000003D301215C2000F0DBFA0021DFF8EC07A6
:1026100001F0F8FA002804D15FF40010FFF7D0F9B8
:1026200016E02021DFF88C0501F0ECFA002804D137
:102630005FF40010FFF7C4F90AE04021DFF87805E5
:1026400001F0E0FA002803D15FF40010FFF7B8F9B9
:10265000DFF85005006850F00100DFF84815086009
:1026600001BD80B5DFF83C050078C0073DD51E20D0
:1026700000F0CAFF092812D01E2000F0C5FF042870
:102680000DD01E2000F0C0FF082808D01E2000F04A
:10269000BBFF072803D05FF40010FFF791F901F0AA
:1026A00076F9002803D14FF40060FFF77DF901F0BF
:1026B000B9F9002803D14FF40060FFF775F91E2027
:1026C00000F0A2FF01F038FA002805D15FF00040C9
:1026D0000021FFF786F904E05FF000400021FFF7DA
:1026E00058F901F0E3F901F03EFA01BD10B504001C
:1026F0001E2000F089FF042801D1012108E00828EC
:1027000001D1022104E0072801D1032100E00021CA
:10271000E4B2002C05D1DFF8A42460204143505CD2
:102720003EE2E4B2022C07D1DFF89024602041435E
:1027300002EB0100807833E2E4B2042C07D1DFF829
:102740007C246020414302EB0100007928E2E4B2DE
:10275000062C07D1DFF864246020414302EB01001E
:1027600080791DE2E4B2082C07D1DFF85024602004
:10277000414302EB0100007A12E2E4B20A2C07D1D5
:10278000DFF838246020414302EB0100807A07E241
:10279000E4B20C2C07D1DFF824246020414302EB83
:1027A0000100007BFCE1E4B20E2C07D1DFF80C2421
:1027B0006020414302EB0100807BF1E1E4B2102C88
:1027C00007D1DFF8F8236020414302EB0100007CD1
:1027D000E6E1E4B2122C07D1DFF8E02360204143A8
:1027E00002EB0100807CDBE1E4B2142C07D1DFF8BE
:1027F000CC236020414302EB0100007DD0E1E4B234
:10280000162C07D1DFF8B4236020414302EB01000E
:10281000807DC5E1E4B2182C07D1DFF8A023602049
:10282000414302EB0100007EBAE1E4B21A2C07D169
:10283000DFF888236020414302EB0100807EAFE196
:10284000E4B21C2C07D1DFF874236020414302EB73
:102850000100007FA4E1E4B21E2C07D1DFF85C2365
:102860006020414302EB0100807F99E1E4B2202C1B
:1028700008D1DFF848236020414302EB010090F8C3
:1028800020008DE1E4B2222C08D1DFF83023602053
:10289000414302EB010090F8220081E1E4B2242CD4
:1028A00008D1DFF818236020414302EB010090F8C3
:1028B000240075E1E4B2262C08D1DFF80023602063
:1028C000414302EB010090F8260069E1E4B2282CB4
:1028D00007D1BA4A6020414302EB010090F828007A
:1028E0005EE1E4B22A2C07D1B44A6020414302EBF6
:1028F000010090F82A0053E1E4B22C2C07D1AF4A32
:102900006020414302EB010090F82C0048E1E4B262
:102910002E2C07D1A94A6020414302EB010090F818
:102920002E003DE1E4B2302C07D1A44A602041439F
:1029300002EB010090F8300032E1E4B2322C07D112
:102940009E4A6020414302EB010090F8320027E1EB
:10295000E4B2342C07D1994A6020414302EB0100D4
:1029600090F834001CE1E4B2362C07D1934A602081
:10297000414302EB010090F8360011E1E4B2382C3B
:1029800007D18E4A6020414302EB010090F83800E5
:1029900006E1E4B2392C07D1884A6020414302EBBA
:1029A000010090F83900FBE0E4B23A2C07D1834AE9
:1029B0006020414302EB010090F83A00F0E0E4B2FD
:1029C0003B2C07D17D4A6020414302EB010090F887
:1029D0003B00E5E0E4B23C2C07D1784A602041435B
:1029E00002EB010090F83C00DAE0E4B23D2C07D1A4
:1029F000724A6020414302EB010090F83D00CFE0B5
:102A0000E4B2402C06D16D4A6020414302EB010044
:102A1000006CC5E0E4B2442C06D1684A6020414312
:102A200002EB0100406CBBE0E4B2482C07D1634AE2
:102A30006020414302EB010090F84800B0E0E4B2AE
:102A4000492C07D15D4A6020414302EB010090F818
:102A50004900A5E0E4B24A2C07D1584A602041431E
:102A600002EB010090F84A009AE0E4B24B2C07D147
:102A7000524A6020414302EB010090F84B008FE086
:102A8000E4B24D2C07D14D4A6020414302EB0100D6
:102A900090F84D0084E0E4B24E2C07D1474A602004
:102AA000414302EB010090F84E0079E0E4B24F2C74
:102AB00007D1424A6020414302EB010090F84F00E9
:102AC0006EE0E4B2502C07D13C4A6020414302EB57
:102AD000010090F8500063E0E4B2512C07D1374A6E
:102AE0006020414302EB010090F8510058E0E4B24D
:102AF000522C07D1314A6020414302EB010090F88B
:102B000052004DE0E4B2542C07D12C4A60204143DE
:102B100002EB010090F8540042E0E4B2562C07D1D9
:102B2000264A6020414302EB010090F8560037E04E
:102B3000E4B2572C07D1214A6020414302EB010047
:102B400090F857002CE0E4B2582C07D11B4A6020C3
:102B5000414302EB010090F8580021E0E4B25C2C04
:102B600007D1164A6020414302EB010090F85C0057
:102B700016E0E4B25D2C07D1104A6020414302EB1D
:102B8000010090F85D000BE0E4B25E2C07D10B4A27
:102B90006020414302EB010090F85E0000E000205D
:102BA00010BD0000102B0020142B0020182B00203B
:102BB0001C2B002088270020A82700203846020070
:102BC00038B505000C001E2000F01EFD042801D1C0
:102BD000012108E0082801D1022104E0072801D1E1
:102BE000032100E00021EDB2002D12D1DFF8140C1A
:102BF000602202FB01F2805C804A1070DFF8042C36
:102C00006020414302EB010040787C49487000F0AD
:102C100034BCEDB2022D13D1DFF8E80B602202FBC9
:102C200001F210448078754A9070DFF8D82B60204C
:102C3000414302EB0100C0787049C87000F01DBC30
:102C4000EDB2042D13D1DFF8BC0B602202FB01F2C0
:102C500010440079694A1071DFF8A82B60204143C5
:102C600002EB010040796549487100F006BCEDB205
:102C7000062D12D1DFF88C0B602202FB01F210440A
:102C800080795E4A9071DFF87C2B6020414302EB33
:102C90000100C0795949C871EFE3EDB2082D12D196
:102CA000DFF8600B602202FB01F21044007A534A05
:102CB0001072DFF8502B6020414302EB0100407A94
:102CC0004E494872D9E3EDB20A2D12D1DFF8340B28
:102CD000602202FB01F21044807A484A9072DFF8C9
:102CE000242B6020414302EB0100C07A4349C872A3
:102CF000C3E3EDB20C2D12D1DFF8080B602202FB0A
:102D000001F21044007B3D4A1073DFF8F82A60207E
:102D1000414302EB0100407B38494873ADE3EDB21B
:102D20000E2D12D1DFF8DC0A602202FB01F2104402
:102D3000807B324A9073DFF8CC2A6020414302EB5B
:102D40000100C07B2D49C87397E3EDB2102D12D15D
:102D5000DFF8B00A602202FB01F21044007C274A2F
:102D60001074DFF8A02A6020414302EB0100407C90
:102D70002249487481E3EDB2122D12D1DFF8840AA2
:102D8000602202FB01F21044807C1C4A9074DFF840
:102D9000742A6020414302EB0100C07C1749C874CB
:102DA0006BE3EDB2142D12D1DFF8580A602202FB5A
:102DB00001F21044007D114A1075DFF8482A6020A6
:102DC000414302EB0100407D0C49487555E3EDB2EB
:102DD000162D15D1DFF82C0A602202FB01F21044F7
:102DE000807D064A9075DFF81C2A6020414302EB83
:102DF0000100C07D0149C8753FE300BF682700207E
:102E0000EDB2182D14D1DFF8FC09602202FB01F2AB
:102E10001044007EDFF8082C1076DFF8E8296020E7
:102E2000414302EB0100407EDFF8F41B487624E3C7
:102E3000EDB21A2D14D1DFF8CC09602202FB01F2A9
:102E40001044807EDFF8D82B9076DFF8B829602018
:102E5000414302EB0100C07EDFF8C41BC8760CE3DF
:102E6000EDB21C2D14D1DFF89C09602202FB01F2A7
:102E70001044007FDFF8A82B1077DFF88829602046
:102E8000414302EB0100407FDFF8941B4877F4E2F6
:102E9000EDB21E2D0AD1DFF86C296020414302EB10
:102EA0000100807FDFF8781B8877E6E2EDB2202D05
:102EB00018D1DFF85009602202FB01F2104490F8AB
:102EC0002000DFF85C2B82F82000DFF83829602032
:102ED000414302EB010090F82100DFF8441B81F828
:102EE0002100CAE2EDB2222D18D1DFF818096022C4
:102EF00002FB01F2104490F82200DFF8242B82F844
:102F00002200DFF800296020414302EB010090F825
:102F10002300DFF80C1B81F82300AEE2EDB2242D74
:102F200018D1DFF8E008602202FB01F2104490F8AB
:102F30002400DFF8EC2A82F82400DFF8C82860209B
:102F4000414302EB010090F82500DFF8D41A81F824
:102F5000250092E2EDB2262D18D1DFF8A8086022F4
:102F600002FB01F2104490F82600DFF8B42A82F840
:102F70002600DFF890286020414302EB010090F822
:102F80002700DFF89C1A81F8270076E2EDB2282DA1
:102F900018D1DFF87008602202FB01F2104490F8AB
:102FA0002800DFF87C2A82F82800DFF85828602003
:102FB000414302EB010090F82900DFF8641A81F820
:102FC00029005AE2EDB22A2D18D1DFF83808602224
:102FD00002FB01F2104490F82A00DFF8442A82F83C
:102FE0002A00DFF820286020414302EB010090F81E
:102FF0002B00DFF82C1A81F82B003EE2EDB22C2DCD
:1030000018D1DFF80008602202FB01F2104490F8AA
:103010002C00DFF80C2A82F82C00DFF8E82760206B
:10302000414302EB010090F82D00DFF8F41981F81C
:103030002D0022E2EDB22E2D18D1DFF8C807602254
:1030400002FB01F2104490F82E00DFF8D42982F838
:103050002E00DFF8B0276020414302EB010090F81A
:103060002F00DFF8BC1981F82F0006E2EDB2302DF9
:1030700018D1DFF89007602202FB01F2104490F8AB
:103080003000DFF89C2982F83000DFF878276020D4
:10309000414302EB010090F83100DFF8841981F818
:1030A0003100EAE1EDB2322D18D1DFF85807602285
:1030B00002FB01F2104490F83200DFF8642982F834
:1030C0003200DFF840276020414302EB010090F816
:1030D0003300DFF84C1981F83300CEE1EDB2342D26
:1030E00018D1DFF82007602202FB01F2104490F8AB
:1030F0003400DFF82C2982F83400DFF8082760203C
:10310000414302EB010090F83500DFF8141981F813
:103110003500B2E1EDB2362D18D1DFF8E8066022B5
:1031200002FB01F2104490F83600DFF8F42882F830
:103130003600DFF8D0266020414302EB010090F812
:103140003700DFF8DC1881F8370096E1EDB2382D52
:103150000CD1DFF8B0266020414302EB010090F86B
:103160003800DFF8BC1881F8380086E1EDB2392D5F
:103170000CD1DFF890266020414302EB010090F86B
:103180003900DFF89C1881F8390076E1EDB23A2D6C
:103190000CD1DFF870266020414302EB010090F86B
:1031A0003A00DFF87C1881F83A0066E1EDB23B2D79
:1031B0000CD1DFF850266020414302EB010090F86B
:1031C0003B00DFF85C1881F83B0056E1EDB23C2D86
:1031D0000CD1DFF830266020414302EB010090F86B
:1031E0003C00DFF83C1881F83C0046E1EDB23D2D93
:1031F0000CD1DFF810266020414302EB010090F86B
:103200003D00DFF81C1881F83D0036E1EDB2402D9D
:103210000AD1DFF8F0256020414302EB0100006C89
:10322000DFF8FC17086428E1EDB2442D0AD1DFF87D
:10323000D4256020414302EB0100406CDFF8E01729
:1032400048641AE1EDB2482D0CD1DFF8B8256020B2
:10325000414302EB010090F84800DFF8C41781F801
:1032600048000AE1EDB2492D0CD1DFF89825602025
:10327000414302EB010090F84900DFF8A41781F800
:103280004900FAE0EDB24A2D0CD1DFF87825602034
:10329000414302EB010090F84A00DFF8841781F8FF
:1032A0004A00EAE0EDB24B2D0CD1DFF85825602042
:1032B000414302EB010090F84B00DFF8641781F8FE
:1032C0004B00DAE0EDB24D2D0CD1DFF8382560204F
:1032D000414302EB010090F84D00DFF8441781F8FC
:1032E0004D00CAE0EDB24E2D0CD1DFF8182560205C
:1032F000414302EB010090F84E00DFF8241781F8FB
:103300004E00BAE0EDB24F2D0CD1DFF8F82460206A
:10331000414302EB010090F84F00DFF8041781F8F9
:103320004F00AAE0EDB2502D0CD1DFF8D824602078
:10333000414302EB010090F85000DFF8E41681F8F9
:1033400050009AE0EDB2512D0CD1DFF8B824602086
:10335000414302EB010090F85100DFF8C41681F8F8
:1033600051008AE0EDB2522D0CD1DFF89824602094
:10337000414302EB010090F85200DFF8A41681F8F7
:1033800052007AE0EDB2542D18D1DFF878046022B3
:1033900002FB01F2104490F85400DFF8842682F812
:1033A0005400DFF860246020414302EB010090F8F4
:1033B0005500DFF86C1681F855005EE0EDB2562D31
:1033C0000CD1DFF840246020414302EB010090F86B
:1033D0005600DFF84C1681F856004EE0EDB2572D3E
:1033E0000CD1DFF820246020414302EB010090F86B
:1033F0005700DFF82C1681F857003EE0EDB2582D4B
:103400000CD1DFF800246020414302EB010090F86A
:103410005800DFF80C1681F858002EE0EDB25C2D54
:103420000CD1DFF8E0236020414302EB010090F86B
:103430005C00DFF8EC1581F85C001EE0EDB25D2D5C
:103440000CD1DFF8C0236020414302EB010090F86B
:103450005D00DFF8CC1581F85D000EE0EDB25E2D69
:103460000BD1DFF8A0236020414302EB010090F86C
:103470005E00DFF8AC1581F85E00EDB21F2D10DAAA
:103480002021DFF89C05FEF7E3FBE4B2002C2CD0F2
:10349000DFF85407006850F00200DFF84C170860AE
:1034A00023E0EDB23F2D10DA2021DFF84007FEF7D0
:1034B000CFFBE4B2002C18D0DFF82C07006850F0E6
:1034C0000400DFF8241708600FE02021DFF8200750
:1034D000FEF7BEFBE4B2002C07D0DFF80C07006853
:1034E00050F00800DFF80017086031BD10B5040087
:1034F000DFF82C05807F092806D1DFF82405C149B3
:1035000060220DF06BFC1CE0042807D1DFF81005E9
:10351000DFF8E01660220DF061FC12E0082807D108
:10352000DFF8FC04DFF8D01660220DF057FC08E04D
:10353000072806D1DFF8E804DFF8C01660220DF096
:103540004DFC2021DFF8D804FEF782FB2021DFF8B4
:103550009C06FEF77DFB2021DFF89406FEF778FB42
:10356000E4B2002C17D0DFF88006006850F00200AB
:10357000DFF874160860DFF87006006850F0040089
:10358000DFF864160860DFF86006006850F0080095
:10359000DFF85416086010BDDFF88414496C084049
:1035A000704780B5DFF87824526C1043DFF8702440
:1035B0005064C9B200290CD02021DFF83406FEF790
:1035C00047FBDFF82406006850F00800DFF8181603
:1035D000086001BD80B5DFF84824526C32EA000073
:1035E000DFF83C245064C9B200290CD02021DFF858
:1035F0000006FEF72DFBDFF8F005006850F008002C
:10360000DFF8E415086001BDC0B2442803D1DFF83B
:103610001004406C0AE0C0B2402803D1DFF8000477
:10362000006C03E0DFF8F813C0B2085C7047DFF805
:10363000B805007810F00E0F01D0012000E0002046
:10364000704710B504002820FFF7DEFF10F03F00A0
:10365000E4B2A04201D101206EE02A20FFF7D4FF9E
:1036600010F03F00E4B2A04201D1012064E02C2020
:10367000FFF7CAFF10F03F00E4B2A04201D10120E1
:103680005AE02E20FFF7C0FF10F03F00E4B2A04246
:1036900001D1012050E02020FFF7B6FF10F03F00DD
:1036A000E4B2A04201D1012046E02220FFF7ACFFA6
:1036B00010F03F00E4B2A04201D101203CE0242000
:1036C000FFF7A2FF10F03F00E4B2A04201D10120B9
:1036D00032E02620FFF798FF10F03F00E4B2A0424E
:1036E00001D1012028E03020FFF78EFF10F03F00CD
:1036F000E4B2A04201D101201EE03220FFF784FF96
:1037000010F03F00E4B2A04201D1012014E03420C7
:10371000FFF77AFF10F03F00E4B2A04201D1012090
:103720000AE03620FFF770FF10F03F00E4B2A0423D
:1037300001D1012000E0002010BD80B5C0B260289A
:103740005ADAC0B238280BDAC0B21E2808D0B44BFF
:10375000C0B21954401CC943B14BC0B219541AE04D
:10376000C0B2542808D1AE4BC0B21954401CC94352
:10377000AB4BC0B219540EE0C0B2442802D1A84BE2
:10378000596408E0C0B2402802D1A54B196402E098
:10379000A34BC0B21954D2B2002A2DD0C0B22028F7
:1037A0000CD220219E48FEF753FADFF83C04006853
:1037B00050F00200DFF8301408601DE0C0B240286D
:1037C0000DD22021DFF82404FEF742FADFF81804B6
:1037D000006850F00400DFF8101408600CE02021AD
:1037E000DFF80C04FEF734FADFF8FC03006850F051
:1037F0000800DFF8F413086001BDDFF8B82A0818E4
:10380000105C70473846020038B505000C002100F6
:10381000280000F0F7F9002800F08180402C3BD10F
:1038200028787F49095D884211D168787C49214414
:10383000497888420BD1A87879492144897888420F
:1038400005D1E87876492144C978884204D000221D
:103850000021082005F03DF8287C71492144097CAD
:1038600088420BD1687C6E492144497C884205D14D
:10387000A87C6B492144897C884204D00022002125
:10388000072005F026F8287D062803DB052028758B
:10389000FA20687500201DE0002CFBD1A87F60494C
:1038A000897F8842F6D0A97F092906D0042904D04F
:1038B000082902D0072900D0002100221E20FFF78E
:1038C0003CFF0120FFF712FE29E0295C544A03194E
:1038D000D154401C1F28F8D3202151482044FEF722
:1038E000B7F9002C08D1DFF80003006850F002009F
:1038F000DFF8F412086012E0202C08D1DFF8E802AB
:10390000006850F00400DFF8E012086007E0DFF81C
:10391000D802006850F00800DFF8CC12086031BD12
:1039200080B520213E48FEF793F92021AF48FEF7ED
:103930008FF92021AE48FEF78BF9AB48006850F0B4
:103940000200A9490860A848006850F00400A64990
:103950000860A548006850F00800A34908605FF4BB
:103960000010FEF700F801BD9F48006850F080008D
:103970009D4908609C48006850F480709A4908602E
:103980009948006850F4007097490860704780B506
:1039900008F0A4FF022840D15FF40010FEF71DF8E4
:1039A00000283AD1DFF81009006800280DD18E48B0
:1039B0000068C0F3C010002807D120211848FEF786
:1039C00031F9002801D1002028E0DFF8F008006874
:1039D00000280DD184480068C0F30020002807D1DA
:1039E00020218248FEF71EF9002801D1002015E0B1
:1039F000DFF8CC08006800280DD17B480068C0F3D0
:103A00004020002807D120217948FEF70BF9002833
:103A100001D1002002E0012000E0012002BD0000F1
:103A20006827002080B55FF40010FDF7D6FF00285E
:103A30003AD1DFF88408006800280DD16A48006890
:103A4000C0F3C010002807D100216D4800F0DAF85B
:103A5000002801D1002028E0DFF860080068002875
:103A60000DD161480068C0F30020002807D1202153
:103A70005E4800F0C7F8002801D1002015E0DFF80B
:103A80004008006800280DD157480068C0F3402066
:103A9000002807D14021564800F0B4F8002801D191
:103AA000002002E0012000E0012002BD80B54E4868
:103AB0000068C0F3C010002810D020234FF480729B
:103AC000DFF8F4174E4805F05CFF012833D1464873
:103AD000006830F08000444908602CE042480068EB
:103AE000C0F30020002810D020234FF49072DFF89C
:103AF000CC173E4805F045FF01281CD13A48006824
:103B000030F480703849086015E037480068C0F329
:103B1000402000280FD020234FF4A072DFF8A01718
:103B2000334805F02EFF012805D12F48006830F4F6
:103B300000702D49086001BD80B5042801D1012025
:103B400008E0082801D1022004E0072801D1032061
:103B500000E00020C0B200F084F8012801D101206B
:103B600000E0002002BD80B51F480068C0F340009F
:103B700000280ED020224FF48071214805F048FF24
:103B800001282FD11848006830F00200164908605B
:103B900028E015480068C0F3800000280ED02022DD
:103BA0004FF49071114805F033FF01281AD10E48E7
:103BB000006830F004000C49086013E00A4800680F
:103BC000C0F3C00000280DD020224FF4A071084897
:103BD00005F01EFF012805D10348006830F00800F9
:103BE0000149086001BD0000102B0020882700203B
:103BF000A827002098460200F84602005847020015
:103C00006827002010B40200012000290ED10024F2
:103C10001D2C24D2115D02EB04035B7873F0FF03CB
:103C2000DB43994200D00020A41CF1E720290ED1EB
:103C30000024172C13D2115D02EB04035B7873F0A0
:103C4000FF03DB43994200D00020A41CF1E7117D63
:103C5000527D72F0FF02D243914200D0002010BC8E
:103C6000704710B504005FF000400021FDF7B9FE79
:103C7000DFF840060078DFF84C16E4B2602202FB61
:103C800004F2895C884201D0002011E3DFF82406A9
:103C90008078DFF83016E4B2602202FB04F21144AF
:103CA0008978884201D0002002E3DFF80806007915
:103CB000DFF81016E4B2602202FB04F21144097925
:103CC000884201D00020F3E2DFF8E8058079DFF8D0
:103CD000F415E4B2602202FB04F2114489798842AF
:103CE00001D00020E4E2DFF8CC05007ADFF8D4153B
:103CF000E4B2602202FB04F21144097A884201D046
:103D00000020D5E2DFF8AC05807ADFF8B815E4B220
:103D1000602202FB04F21144897A884201D000201B
:103D2000C6E2DFF89005007BDFF89815E4B2602268
:103D300002FB04F21144097B884201D00020B7E263
:103D4000DFF87005807BDFF87C15E4B2602202FBAF
:103D500004F21144897B884201D00020A8E2DFF8F8
:103D60005405007CDFF85C15E4B2602202FB04F22B
:103D70001144097C884201D0002099E2DFF8340523
:103D8000807CDFF84015E4B2602202FB04F21144AB
:103D9000897C884201D000208AE2DFF81805007D86
:103DA000DFF82015E4B2602202FB04F21144097D21
:103DB000884201D000207BE2DFF8F804807DDFF844
:103DC0000415E4B2602202FB04F21144897D8842AA
:103DD00001D000206CE2DFF8DC04007EDFF8E414A0
:103DE000E4B2602202FB04F21144097E884201D051
:103DF00000205DE2DFF8BC04807EDFF8C814E4B286
:103E0000602202FB04F21144897E884201D0002026
:103E10004EE2DFF8A004007FDFF8A814E4B26022CD
:103E200002FB04F21144097F884201D000203FE2E6
:103E3000DFF8800490F82000DFF88814E4B26022F4
:103E400002FB04F2114491F82010884201D00020B6
:103E50002EE2DFF8600490F82200DFF86814E4B284
:103E6000602202FB04F2114491F82210884201D032
:103E700000201DE2DFF83C0490F82400DFF8441431
:103E8000E4B2602202FB04F2114491F8241088424B
:103E900001D000200CE2DFF81C0490F82600DFF8C7
:103EA0002414E4B2602202FB04F2114491F82610BB
:103EB000884201D00020FBE1DFF8F80390F82800E9
:103EC000DFF80014E4B2602202FB04F2114491F81E
:103ED0002810884201D00020EAE1DFF8D80390F8EA
:103EE0002A00DFF8E013E4B2602202FB04F211447E
:103EF00091F82A10884201D00020D9E1DFF8B403FC
:103F000090F82C00DFF8BC13E4B2602202FB04F24C
:103F1000114491F82C10884201D00020C8E1DFF84C
:103F2000940390F82E00DFF89C13E4B2602202FBA9
:103F300004F2114491F82E10884201D00020B7E11C
:103F4000DFF8700390F83000DFF87813E4B26022F5
:103F500002FB04F2114491F83010884201D0002095
:103F6000A6E1DFF8500390F83200DFF85813E4B20E
:103F7000602202FB04F2114491F83210884201D011
:103F8000002095E1DFF82C0390F83400DFF83413BB
:103F9000E4B2602202FB04F2114491F8341088422A
:103FA00001D0002084E1DFF80C0390F83600DFF840
:103FB0001413E4B2602202FB04F2114491F83610AB
:103FC000884201D0002073E1BA4890F83800BD491A
:103FD000E4B2602202FB04F2114491F838108842E6
:103FE00001D0002064E1B34890F83900B549E4B24B
:103FF000602202FB04F2114491F83910884201D08A
:10400000002055E1AB4890F83A00AE49E4B2602296
:1040100002FB04F2114491F83A10884201D00020CA
:1040200046E1A44890F83B00A649E4B2602202FBB6
:1040300004F2114491F83B10884201D0002037E18E
:104040009C4890F83C009F49E4B2602202FB04F2D5
:10405000114491F83C10884201D0002028E1954895
:1040600090F83D009749E4B2602202FB04F211444B
:1040700091F83D10884201D0002019E18D48006C74
:104080009049E4B2602202FB04F21144096C8842B8
:1040900001D000200CE18748406C8A49E4B26022DC
:1040A00002FB04F21144496C884201D00020FFE079
:1040B000804890F848008349E4B2602202FB04F291
:1040C000114491F84810884201D00020F0E079486E
:1040D00090F849007B49E4B2602202FB04F21144EB
:1040E00091F84910884201D00020E1E0714890F831
:1040F0004A007449E4B2602202FB04F2114491F8D0
:104100004A10884201D00020D2E06A4890F84B0063
:104110006C49E4B2602202FB04F2114491F84B10A6
:10412000884201D00020C3E0624890F84D00654904
:10413000E4B2602202FB04F2114491F84D1088426F
:1041400001D00020B4E05B4890F84E005D49E4B235
:10415000602202FB04F2114491F84E10884201D013
:104160000020A5E0534890F84F005649E4B2602281
:1041700002FB04F2114491F84F10884201D0002054
:1041800096E04C4890F850004E49E4B2602202FBA1
:1041900004F2114491F85010884201D0002087E0C9
:1041A000444890F851004749E4B2602202FB04F20F
:1041B000114491F85110884201D0002078E03D4828
:1041C00090F852003F49E4B2602202FB04F211442D
:1041D00091F85210884201D0002069E0354890F8EB
:1041E00054003849E4B2602202FB04F2114491F811
:1041F0005410884201D000205AE02E4890F8560012
:104200003049E4B2602202FB04F2114491F85610E6
:10421000884201D000204BE0264890F857002949F9
:10422000E4B2602202FB04F2114491F85710884274
:1042300001D000203CE01F4890F858002149E4B22A
:10424000602202FB04F2114491F85810884201D018
:1042500000202DE0174890F85C001A49E4B2602273
:1042600002FB04F2114491F85C10884201D0002056
:104270001EE0104890F85D001249E4B2602202FB93
:1042800004F2114491F85D10884201D000200FE043
:10429000084890F85E100B4AE4B26020444302EBF9
:1042A000040090F85E00814201D0002000E001206F
:1042B00010BD000068270020142B0020182B0020C0
:1042C0001C2B00203846020070B5954C954E2046B8
:1042D00001F008F9204601F01FF9934C1021204607
:1042E000FBF7A0FF20212046FBF79CFF082120467A
:1042F000FBF798FF40212046FBF794FF8B48FBF724
:10430000EDFF40212046FBF7D1FF10212046FBF7AF
:10431000C3FF20212046FBF7BFFF85494FF47220E1
:1043200008600D464FF0FF32002128460CF087FD53
:1043300028460CF07FFD7F48FBF7D0FF7E48FBF757
:10434000CDFF304601F0CEF8304601F0E5F87B4E67
:10435000304601F0C7F8304601F0DEF8784E794972
:104360003046FCF77CFE40F20442FF213046FCF769
:10437000A9FE4FF0FF32FF213046FCF7B9FE724A2A
:104380004FF47F413046FCF7B3FE04213046FCF782
:10439000CBFE4FF480713046FCF7C6FE202176201C
:1043A00001F055FA4021772001F051FA762001F012
:1043B0005FFA772001F05CFA4FF6FF713046FCF7A8
:1043C0003FFE012208212046FBF762FE5F4C0120E0
:1043D0006060FCF78BFC002128460CF038FD0020C3
:1043E00060610120206070BD30B581B001F028FA15
:1043F00056484168012905D101F01EFA4FF0FF30FF
:1044000001B030BDC4680569514801680C1B01F05A
:1044100013FAA54238BF25464E4AA5FB022188095A
:1044200001B030BD10B54949086810B900242046D4
:1044300010BD3F48083000680446FCF757FC0128CF
:1044400008BF6442204610BD10B50446FCF74EFC80
:1044500000281CBF002C64422146BDE810403448AF
:104460000CF0F5BC3948416915298041C043C00FA3
:104470007047364901208860704710B4364881B0D3
:104480000421016000210163304A416A90680128DB
:1044900002D10023536193605068304BA0B91C686F
:1044A000200703D45069401C506101E0002454618E
:1044B000D068081AB0F5FA5F28BF10610AD2082048
:1044C000986001B010BC70474FF0FF3010610020C1
:1044D00050615060D1600820986001B010BC4FF46A
:1044E00080711748FCF725BE00B581B04FF480718C
:1044F0001348FCF71EFE15480121416017490A6860
:10450000130706D40023436183600820886001B04C
:1045100000BD4269521C42610820886001B000BDA4
:10452000004400F0000400F000F005400718070008
:1045300000C002400510070005140700045C00F0ED
:1045400000E004401732000400D43000042A0020A8
:1045500050E00440CDCCCCCC24E0044014F4054021
:1045600080B58021DFF8F00AFBF766FE8020DFF8D7
:10457000EC1A08600421DFF8E00AFBF75DFE00207A
:10458000DFF8DC1A08601021DFF8D80AFBF754FEC8
:104590002021DFF8D00AFBF74FFE0020DFF8441C93
:1045A00008602020DFF8001C08601021DFF8FC0BF9
:1045B000FBF742FE1020DFF8301C08604021DFF8D6
:1045C000A80AFBF739FE0020DFF8A01A08601021C6
:1045D000DFF8940AFBF730FE0020DFF8D41B0860F8
:1045E0002021DFF8840AFBF727FE0020DFF8C41B38
:1045F0000860DFF8C40B00F075FF2221DFF8BC0B68
:10460000FCF72DFD0122FF21DFF8B00BFCF764FD64
:104610008021272001F01BF9DFF8D02BFF21DFF8E4
:104620009C0BFCF765FD0121DFF8900BFCF77CFD8E
:104630000121DFF8880BFCF77CFD272001F018F939
:10464000FF21DFF8780BFCF7FBFC0020DFF8A01B54
:104650000860DFF8A00B00F045FF7121DFF8980B30
:10466000FBF7C2FD0321DFF8440BFBF7BDFD012181
:10467000DFF8880BFBF7B8FD012300220021DFF8EB
:10468000800BFDF706FA052300220021DFF8700BEE
:10469000FDF729FA062301220021DFF8640BFDF75C
:1046A00022FA072302220021DFF8540BFDF71BFA40
:1046B000032303220021DFF8480BFDF714FA02233D
:1046C00004220021DFF8380BFDF70DFA6F230522D5
:1046D0000021DFF82C0BFDF706FA0021DFF8200B94
:1046E000FDF7CAF90021DFF8180BFDF7C1F9002129
:1046F000DFF80C0BFDF7B5F9E0211E2001F0A7F85B
:104700001E2001F0B5F8DFF8580C0078C007FAD584
:10471000FBF74CFEDFF84C1C0862FBF747FEDFF8A6
:10472000441CC861DFF8380C006830F02000DFF866
:10473000301C0860FBF73AFEDFF8A41B0860FBF7AB
:1047400035FEDFF8A01B0860FBF730FEDFF8981B92
:104750000860FBF72BFEDFF8941B0860022000F0D6
:10476000C7FD46F6605188420ED24E20FEF74CFF40
:10477000C00706D44FF48070FDF722F900F04DFA1F
:104780000CE000F0FAF909E000F047FADFF8D00B8E
:10479000006850F01000DFF8C81B086001BD80B54C
:1047A000C0B2042803D0C0B200F0A2FD02E0DFF8DE
:1047B000B40B006802BD80B54FF480400021FDF7C6
:1047C00019F900220023994201D190421AD00E20FB
:1047D000FEF737FF002815D14FF40060FEF7DCFE2E
:1047E00000280FD007F001FB012803D007F0FDFAE5
:1047F000022807D1DFF8680B006850F02000DFF8CE
:10480000601B086001BDDFF8580B006830F0200025
:10481000DFF84C1B0860704780B5DFF8440B007868
:10482000C00719D5DFF8380B0068C0F34000002836
:1048300002D000F09EF801E000F04DFA00F0E2FC3A
:1048400000F016FCDFF8180B006810F4407F03D06E
:104850004FF40070FDF7A8F801BD80B54FF480401B
:104860000021FDF7C7F800220023994206D19042AB
:1048700004D18020DFF8E417086003E00020DFF8AF
:10488000DC17086001BD80B5DFF8D007006800289C
:104890000AD14FF480400021FDF7ACF8002200233C
:1048A000994201D190420FD0DFF8B007006800288C
:1048B0000CD04FF480400021FDF79CF8002200232B
:1048C000994201D1904201D0002000E0012002BDB8
:1048D000DFF88C0A0068C0F38000002801D10120B5
:1048E00000E00020704780B50021DFF81409FDF7D3
:1048F000BFF8DFF8742A0021DFF80409FDF740F95A
:1049000000210FE0DFF8642ADFF8E40803681820CC
:10491000434302EB0300DFF8502A52F8212040F80D
:104920002120491C0629EDD3DFF8C4080068401C8B
:10493000DFF8BC180860DFF8B808006806280BD359
:104940000020DFF8AC180860DFF8140A006850F0A7
:104950000100DFF80C1A086001BD80B50121DFF805
:104960005C08FCF7E6FB0021DFF89408FDF71BF973
:1049700001BD80B54FF480400021FDF70AF85FF0DB
:1049800000500021FDF705F8DFF8D409006830F089
:104990002000DFF8CC190860FBF708FDDFF8D0191C
:1049A0000860DFF8BC09006830F48060DFF8B019F7
:1049B0000860022000F09CFCDFF8A8194860DFF8CE
:1049C000A409406846F6605188420FD2FBF7EEFC1E
:1049D000DFF80C190968401A652807D34E20FEF746
:1049E00013FEC00702D500F0C8F8C5E0DFF874096F
:1049F000406846F66051884215D25FF08040FCF76F
:104A0000B2FFFBF7D3FCDFF8D8180968401A652815
:104A10002ED34E20FEF7F8FDC00729D44FF4807046
:104A2000FCF7CEFF24E0DFF83C0940684AF6C97184
:104A3000884210D34FF48070FCF795FFFBF7B6FC6B
:104A4000DFF89C180968401A652811D35FF0804090
:104A5000FCF7B6FF0CE0FBF7A9FCDFF88418086050
:104A60005FF08040FCF77FFF4FF48070FCF77BFF26
:104A700000F0F3F900F05FFA052000F039FCDFF8F0
:104A8000E4188860DFF8DC084168DFF8D80880683F
:104A9000081A41F27171884212DBFBF787FCDFF8DC
:104AA00048180968401A40F2D171884215D3DFF8DE
:104AB000B008006850F40070DFF8A41808600CE03B
:104AC000FBF774FCDFF820180860DFF89408006832
:104AD00030F40070DFF8881808604E20FEF794FD6F
:104AE000C0070DD44FF40070FCF73DFF5FF080402D
:104AF0000021FCF74EFF0020DFF8681808603BE05B
:104B0000DFF85C080068C0F30010002834D1FBF720
:104B10004DFCDFF850188969401A4EF66121884231
:104B200008D3DFF83C08006850F01000DFF83018B8
:104B3000086021E0042000F0DBFB47F619118842F1
:104B400006D3DFF81C180968C1F3C011002909D089
:104B5000DFF80C180968C1F3C01100290CD0B0F5BA
:104B6000FA6F09D25FF080400021FCF73AFFFBF7B3
:104B70001DFCDFF8F017886101BD80B52020DFF84B
:104B800028160860FBF712FCDFF8D8170862DFF878
:104B9000D007006850F00400DFF8C4170860FBF786
:104BA00005FCDFF8C017C861DFF8B407006830F013
:104BB0000200DFF8AC17086000F002FBFBF7F6FB21
:104BC000DFF81C170860FBF7F1FBDFF81817086027
:104BD000FBF7ECFBDFF814170860DFF884070068C8
:104BE00030F40070DFF8781708605FF08040002133
:104BF000FCF7CFFE4FF480400021FCF7F2FE5FF09F
:104C00008040FCF7B0FE4FF40070FCF7ACFE0022D1
:104C100001210F2003F05DFE01BD80B54FF400704F
:104C2000FCF7DBFE002802D0FBF7C8FB52E00020B7
:104C3000DFF8B01508601020DFF8AC150860FBF74E
:104C4000B5FBDFF820170862DFF81407006850F0A2
:104C50000400DFF80C170860FBF7A8FBDFF8041767
:104C6000C861DFF8FC06006850F00200DFF8F016BB
:104C70000860FBF79BFBDFF868160860FBF796FB04
:104C8000DFF860160860FBF791FBDFF8601608603C
:104C9000FBF78CFBDFF850160860FBF787FBDFF8AB
:104CA000C41688614FF40070FCF75DFE5FF0804031
:104CB0000021FCF76EFE4FF480400021FCF769FEF6
:104CC0005FF000500021FCF764FE002200210F205D
:104CD00003F0FFFD01BD80B500F072FA022000F084
:104CE00007FBDFF880164860DFF87806406847F277
:104CF000315188420AD3FBF759FBDFF8781609686F
:104D0000401A652802D3FFF788FFA5E0DFF85406B4
:104D1000406847F23151884204D2FBF747FBDFF885
:104D20005416086007F064F801284CD14FF4007065
:104D3000FCF746FE0020DFF8701408601020DFF852
:104D4000A41408600020DFF8A0140860DFF8100643
:104D50000068C0F3802000281BD1002102200BF046
:104D600004FEFBF723FBDFF808160968401A40F63B
:104D7000B831884270D3FBF719FBDFF8F4150860EF
:104D8000DFF8DC05006850F48060DFF8D4150860B7
:104D900062E0012102200BF0E8FDFBF707FBDFF8E2
:104DA000D0150968401AC82856D3FBF7FFFADFF878
:104DB000C0150860DFF8A805006830F48060DFF8EF
:104DC000A015086048E02020DFF8DC130860FBF73E
:104DD000EDFADFF89C150860DFF88405006830F410
:104DE0008060DFF87C150860022102200BF0BDFD19
:104DF0005FF000500021FCF7FDFD002200239942E6
:104E000001D1904207D0DFF85805006850F020002B
:104E1000DFF84C150860042000F06AFADFF844154A
:104E2000086006F0DFFF062803D006F0DBFF052848
:104E300002D144F6206001E045F2F050DFF824157D
:104E40000968814204D25FF080400021FCF7C9FD6F
:104E500000F003F800F06FF801BD80B5012000F00C
:104E600047FADFF80015C860FBF7A0FADFF8F41482
:104E7000096A401AC92850D3DFF8E404006830F00A
:104E80000400DFF8DC140860DFF8D4040068C0F325
:104E90004000002804D11020DFF84813086002E029
:104EA0000020C14908605FF080400021FCF7A2FDAE
:104EB00000220023994201D1904206D0DFF8A004DD
:104EC0000068C0F34000002834D0DFF89804C068C0
:104ED00042F6E061884212D2FBF768FADFF8041468
:104EE0000968401A40F2D171884223D3DFF8700478
:104EF000006850F48070DFF8681408601AE0FBF76F
:104F000055FADFF8E0130860DFF85404006830F465
:104F10008070DFF84C1408600CE0DFF8440400688F
:104F200050F00400DFF838140860FBF73FFADFF8B0
:104F3000B413086001BD80B5DFF824040068C0F335
:104F40004000002807D0DFF81804006830F0200087
:104F5000DFF80C140860002000F0CAF9DFF8041430
:104F60000861DFF8FC030068C0F3401000285CD142
:104F700010209D490860FBF719FADFF8E813C969AA
:104F8000401A40F2D17188420DD3DFF8D403006893
:104F900030F00800DFF8C81308605FF000700021EF
:104FA000FCF7F7FC07E0DFF8B803006850F00800F2
:104FB000DFF8AC130860DFF8A803007810F00C0FDE
:104FC0002ED15FF080400021FCF714FD0022002369
:104FD000994201D1904206D0DFF884030068C0F303
:104FE000400000281CD0DFF87C030069DFF8741350
:104FF000C968B1F57A7188420AD2FBF7D7F9BB4983
:105000000968401AC92825D30420FCF7D9FC21E0FF
:10501000FBF7CCF9B54908600420FCF7A4FC19E0C3
:10502000FBF7C4F9B149086014E05FF0007000219B
:10503000FCF7D7FCFBF7BAF9DFF82813C861DFF8F3
:105040002003006850F00800DFF814130860002007
:105050006549086001BD000000F0054000F2054010
:1050600010F0054000300640004006400041064078
:1050700010B5042000F03CF904004FF480400021FA
:10508000FCF7B8FC00220023994229D1904227D195
:1050900045480068002823D1B1480068C0F30010DB
:1050A00000281DD1AF48407D002819D1FBF7A0F999
:1050B000012815D0AA480068C0F3C02000280FD1ED
:1050C0004E20FEF7A1FAC0070AD55FF400200021A8
:1050D000FCF790FC00220023994201D1904213D0AA
:1050E00000203449086000203149086003209D49B0
:1050F0000875002101200BF038FC9948006850F039
:105100008000974908604DE09548006830F08000C5
:10511000934908601020264908609248006846F6C6
:10512000615188420FD35FF080400021FCF762FCA0
:1051300000220023994206D1904204D1012101208E
:105140000BF013FC03E0022101200BF00EFC85485C
:10515000007D401C834908758248007D042802DBDD
:105160000120804908757F48007D012803D1202057
:105170001049086016E07B48007D02280BD144F6F8
:105180002160844203D320200A4908600AE00020FD
:105190000849086006E07348007D032802D100201A
:1051A0000449086010BD00008030064000C0054082
:1051B0004040064080400640020400F000200340CA
:1051C00080B500206C4908606548006830F0100028
:1051D00063490860002063494875FBF7E7F86149B7
:1051E000886101BD4030064040C0054000710200AA
:1051F000F82D0020003800F000700040001006403C
:105200000080034080B55748407D002815D15448A0
:105210000068C0F30010002860D04E20FEF7F4F9BB
:10522000C0075BD5FBF7C2F85449086001204D491F
:10523000487540205049086050E04A48407D0128A8
:1052400040D1FBF7B3F84D490968401A652845D3AA
:10525000002044494875FBF7A9F8424988610420B9
:1052600000F046F83F4908600020434908603C4888
:10527000006830F010003A4908603A48006845F686
:10528000D811884205D25FF080400021FCF7A9FBCD
:1052900004E05FF080400021FCF77BFB31480068B0
:1052A00047F61911884206D32D48006850F4006073
:1052B0002B49086012E02A48006830F40060284951
:1052C00008600BE02648006830F0100024490860B0
:1052D00000202449487500202749086001BD0000CE
:1052E000082E0020002E0020FC2D0020042E00207F
:1052F00010B504002000C0B200F01CF8E4B2002C8D
:1053000008D0022C0DD005D3042C03D009D3052CD2
:1053100007D00DE040F2763148436421B0FBF1F054
:1053200007E04FF49E6148436421B0FBF1F000E0D8
:10533000002010BD10B40022002309E00B491824FE
:1053400004FB03F42144C0B251F820108A185B1CFE
:10535000062BF3D30620B2FBF0F010BC7047000020
:10536000F42D0020B82800201C2A0020482400200A
:105370000C2E0020082E002000410640102E002098
:1053800010B401000022002000230EE0401E0BE0BC
:10539000400014000A00920F12EB84028900401CA6
:1053A0008242F3D3121A401C5B1C102BF0D340082E
:1053B00010BC7047401801686FF35201114301603F
:1053C00000F124012030920704D5B02202604FF48E
:1053D000306003E08C22026040F60C0008607047E9
:1053E000401800F11001006883074CBF5208521E9C
:1053F0000A607047081801681AE010B58B0900EBC5
:10540000831003689C0700F1100348BF52081B6813
:105410009A1AC9074CBF1C301830026010BD4018E2
:1054200000F12C010A6000F130010B6050F8281FD8
:1054300041F001010160704740F8041F70470830D7
:10544000012A02680CBF114322EA01010160704782
:105450000C30012A02680CBF114322EA01010160ED
:1054600070472430012A02680CBF114322EA01016F
:10547000016070471030012A02680CBF114322EA14
:10548000010101607047081850F8041F0A430260C8
:105490007047081850F8041F21EA020202607047A2
:1054A00018B58100DFF8C422C0F3072301F47F712F
:1054B000D31841EA431343F0844301241C600023C2
:1054C000009302E0009C641C0094009B102BF9D315
:1054D000C0F30720121841EA421141F08441002034
:1054E000086011BDC0F30722DFF8841280008A181B
:1054F00000F47F7040EA421040F0844001210160D6
:10550000704780008A1800F47F7040EA421040F033
:105510008440002101607047C0F30722DFF8541275
:10552000EFE7C0F30722DFF85012DFE7C0F30722EE
:10553000DFF84412E5E7DFF8441208B188687047E5
:1055400008687047DFF8380200687047DFF83012EB
:105550000A6822EA00000860704700000138FDD1A7
:1055600070477047DFF81C120860704770B5DFF8AD
:105570000C221369146A014623F4800301F001052B
:1055800043F4006303F0010085F0010544F4006476
:105590001361284214620ED061F0010003404FF401
:1055A0008070906013614FF400201568EE054AD4B6
:1055B000401EFAD170BD080960F30A13DFF8D40168
:1055C00013610440DFF8D00108400443C80000F034
:1055D000400004431462480B60F34D3360F34D34D4
:1055E00040209060002C47BF146213611361146265
:1055F000DFF8A8010340DFF8A80108400343C80D05
:1056000060F3DC54480008D5DFF8980124F48004E6
:10561000084043F48003044301E024F0804408057B
:105620000BD44FF4004060490D68EE0701D4401ED2
:10563000FAD123F4006324F400641361146210208F
:10564000BDE870408AE70028B5D170BDF0B5574974
:105650000A6D0B6E002B4CBF03F0700002F030009F
:1056600040B1102847D0202847D0302847D0702894
:1056700048D04AE00FF25410C2F3841450F824507A
:105680004B4C04EA0306B6F1004F4FF0FF3003D055
:10569000002B41D416053FD43C4E37687668096824
:1056A000C6F3042C06F01F060CF1010C761C16FB49
:1056B0000CF67600B5FBF6F5C7F30906C7F38927A4
:1056C0006F4301F47041BF0AB1F5005F06FB057539
:1056D00042F480020DD0B1F5405F18D0B1F5804F93
:1056E00017D0B1F5E04F16D0B1F5104F08BF3148D3
:1056F00012E0314810E0244DC2E7304DC0E747F2D8
:105700003055BDE74FF40045BAE70020F0BD2C4806
:1057100002E02C4800E01E48510217D5002B10D59E
:1057200059000BD51C40B4F1004F03D0002B05D419
:10573000110503D46D00C3F3865104E0C3F3C551D2
:1057400001E0C2F3C351491CB5FBF1F5A84288BF83
:105750002846F0BD1C4901230A6800F00F0003FA37
:1057600000F000E00A6810430860704700E50F4051
:1057700000E60F4000E70F4000E80F4050E00F4008
:105780005CE00F407CE00F400024F40060E10F403B
:1057900040787D018FFFFF7F30000080FEFF3FF8E3
:1057A0000100C0070000404068E10F4010E00F40DA
:1057B00000080080002D310100B4C40400093D0040
:1057C00080F0FA02005A62026CE00F4040420F0083
:1057D00000201C0080841E0000802500999E360059
:1057E0000040380000093D0000803E0000004B00F2
:1057F000404B4C0000204E00808D5B0000C05D00DF
:105800000080700000127A0000007D0080969800F1
:10581000001BB7000080BB00C0E8CE00647ADA004D
:105820000024F4000000FA0080A81201002D3101CC
:1058300000366E0140787D0180B50BF00FFB02E071
:1058400080B50BF007FB00B10120C0B202BD10B55E
:105850000FF2D402830852F823201368C00000F02E
:105860001800FF248440A34381401943116010BDF8
:1058700004282B4903D1086840F480300BE0052848
:1058800004D10A6842F400320A607047062804D145
:10589000086840F48020086070470F2805D121482F
:1058A000016841F00201016070470CD90FF2141336
:1058B000A0F110011038400953F82000012201F036
:1058C0001F018A40026070470428154903D1086807
:1058D00020F480300BE0052804D10A6822F400325D
:1058E0000A607047062804D1086820F48020086008
:1058F00070470F2805D10B48016821F002010160B3
:1059000070470CD90FF2D003A0F1100110384009F4
:1059100053F82000012201F01F018A400260704705
:1059200024ED00E010E000E00000000018ED00E0D1
:105930001CED00E020ED00E000E400E004E400E005
:1059400008E400E00CE400E010E400E014E400E00F
:1059500018E400E01CE400E020E400E024E400E0BF
:1059600028E400E02CE400E030E400E034E400E06F
:1059700038E400E03CE400E040E400E044E400E01F
:1059800048E400E04CE400E050E400E054E400E0CF
:1059900058E400E05CE400E060E400E064E400E07F
:1059A00068E400E06CE400E070E400E074E400E02F
:1059B00078E400E07CE400E080E400E084E400E0DF
:1059C00088E400E000E100E004E100E008E100E03C
:1059D0000CE100E010E100E080E100E084E100E0A3
:1059E00088E100E08CE100E090E100E080B5DFF8C4
:1059F000440B006840084000DFF8381B0860FAF7E5
:105A0000FDFC00280CD10820FBF7DAFF0020DFF8AE
:105A1000281B08605FF0FF30DFF8201B086039E0CA
:105A200000F00DFF0028FBD1002000F098FADFF80D
:105A3000081B0860012000F092FADFF8001B0860E4
:105A4000DFF8F40A0068DFF8F41A0968C9438842ED
:105A500018D00020DFF8E01A08605FF0FF30DFF8B0
:105A6000DC1A0860DFF8D40A0068DFF8CC1A09787D
:105A700001F0FF0151EA002100910422042168464F
:105A800000F078FEDFF8AC0A006850F00100DFF8A3
:105A9000A41A086001BD10B5DFF8980A0078C007A5
:105AA00056D5DFF8940A0068DFF8901A0968C943F0
:105AB000884206D000F03BFC5FF08070FBF774FF7B
:105AC00046E0DFF8740A006800F070FA04001E2057
:105AD000FDF79AFD062802D134F0500406E01E209E
:105AE000FDF792FD072801D134F00404DFF8480ADD
:105AF0000068844213D0DFF8400A0460E443DFF812
:105B00003C0A0460DFF8300A006800F08DFD0100F7
:105B1000DFF82C0A0278C9B2032002F0DAFE00F0A6
:105B20008EFE002814D1002000F019FADFF8081AC0
:105B3000096888420CD0DFF8040A0168DFF8F80928
:105B4000007800F0FF0050EA0120042100F05EFE22
:105B500010BDDFF8E8090168DFF8DC09007800F023
:105B6000FF0050EA01207047C0B20A2808D1DFF8D0
:105B7000C8090078800701D5012041E100203FE1FC
:105B8000C0B211280AD1DFF8B009007810F0630024
:105B9000402801D1012033E1002031E1C0B20B28BF
:105BA0000AD1DFF89409007810F07F00402801D175
:105BB000012025E1002023E1C0B20E280AD1DFF840
:105BC0007809007810F07F00442801D1012017E106
:105BD000002015E1C0B20D280AD1DFF85C09007879
:105BE00010F07F00502801D1012009E1002007E1D9
:105BF000C0B210280AD1DFF84009007810F07F0009
:105C0000542801D10120FBE00020F9E0C0B20C28AB
:105C10000AD1DFF82409007810F07F00482801D16C
:105C20000120EDE00020EBE0C0B20F280AD1DFF840
:105C30000809007810F07F004C2801D10120DFE036
:105C40000020DDE0C0B212280AD1DFF8EC080078AD
:105C500010F00300012801D10120D1E00020CFE0A5
:105C6000C0B213280AD1DFF8D008007810F0630022
:105C7000202801D10120C3E00020C1E0C0B21428D7
:105C80000AD1DFF8B408007810F00600042801D12A
:105C90000120B5E00020B3E0C0B2152809D1DFF83B
:105CA0009808007810F03B0F01D10120A8E00020F7
:105CB000A6E0C0B216280AD1DFF87C08007810F000
:105CC0003B00082801D101209AE0002098E0C0B2F2
:105CD00017280AD1DFF86008007810F03B00102880
:105CE00001D101208CE000208AE0C0B208280AD14E
:105CF000DFF84408007810F00700012801D10120E6
:105D00007EE000207CE0C0B209280AD1DFF8280834
:105D1000007810F00700052801D1012070E0002074
:105D20006EE0C0B2002808D1DFF80C080068002837
:105D300001D1012064E0002062E0C0B206280AD14F
:105D4000DFF8F407007810F07F00202801D101204F
:105D500056E0002054E0C0B207280AD1DFF8D80787
:105D6000007810F07F00242801D1012048E00020B5
:105D700046E0C0B201280AD1DFF8BC07007810F075
:105D80007F00042801D101203AE0002038E0C0B2B1
:105D900002280AD1DFF8A007007810F07F00082859
:105DA00001D101202CE000202AE0C0B203280AD152
:105DB000DFF88407007810F07F000C2801D1012063
:105DC0001EE000201CE0C0B204280AD1DFF86807FA
:105DD000007810F07F00102801D1012010E0002091
:105DE0000EE0C0B205280AD1DFF84C07007810F0A9
:105DF0007F00142801D1012002E0002000E00020F3
:105E0000704780B500F093FA01BD10B5040056202C
:105E1000FDF7FAFB002804D05720FDF7F5FB012819
:105E200032D1DFF81407007880072DD42000C0B2EB
:105E300000F092FB040060060DD534F020045620DB
:105E4000FDF7E2FB800704D55720FDF7DDFB0128B5
:105E500001D07FF04004DFF8E006006884420BD0F8
:105E6000DFF8D006006850F01000DFF8C8160860B0
:105E7000DFF8D006046007E0DFF8B806006830F00D
:105E80001000DFF8B016086010BD10F07F00DFF8DA
:105E9000A816096888420BD0DFF89816096851F0F7
:105EA0000401DFF890261160DFF89C16086007E017
:105EB000DFF88006006830F00400DFF8781608602C
:105EC000704710B5040014F07F04DFF86C0600681A
:105ED000844211D05FF00050FDF75EFB00280BD12B
:105EE000DFF85006006850F00200DFF8481608603E
:105EF000DFF85806046007E0DFF83806006830F085
:105F00000200DFF83016086010BD10B504005620FE
:105F1000FDF77AFB002821D05720FDF775FB0128FB
:105F20001CD014F07F0460060DD55620FDF76CFBE5
:105F3000800707D55720FDF767FB032802D134F00F
:105F4000200400E00024DFF8EC05006850F00800B1
:105F5000DFF8E0150860DFF8F805046010BD10B543
:105F600082B00400FAF74AFA012815D100F067FC64
:105F7000002811D104220421684600F0E6FB002C21
:105F800004D1009800F0FF0000900DE00098000A96
:105F900070F0FF00009007E0002C02D1002000907C
:105FA00002E05FF0FF300090009816BD10B50400CD
:105FB00000F0D7F9DFF87C050068C0F3C0000028C6
:105FC00025D000200821FBF715FD0022002399426F
:105FD0001DD190421BD1DFF8780504680520DFF859
:105FE000601508705FF480200021FBF703FD00229C
:105FF0000023994202D1904200F08581DFF83405F8
:10600000006830F00800DFF82C1508607BE1DFF84D
:1060100024050068C0F30010002800F0AC80DFF811
:1060200024050078800707D5DFF8180504680320E9
:10603000DFF80C15087066E1DFF8F8040068C0F3BB
:106040004010C0070CD5DFF80C050078800707D595
:10605000DFF8000504680120DFF8E414087052E15D
:10606000DFF8D0040068C0F38000C0070AD5DFF86D
:10607000D8040078800705D502240220DFF8C01478
:10608000087040E1DFF8AC040068C0F34000C007CE
:106090000AD5DFF8B8040078800705D5022404206B
:1060A000DFF89C1408702EE1A0075CD5DFF890049F
:1060B0000078022809D0DFF888040078042804D08A
:1060C000DFF87C04007801284DD1DFF874040078F3
:1060D000012813D1DFF85C040068C0F34010C0074A
:1060E0000CD5DFF870040078800707D4DFF864046B
:1060F00004680120DFF84814087004E1DFF8400468
:106100000078022813D1DFF82C040068C0F3800067
:10611000C0070CD5DFF830040078800707D4DFF81B
:10612000280404680220DFF818140870EBE0DFF898
:1061300010040078042840F0E680DFF8F8030068D7
:10614000C0F34000C00740F1DE80DFF800040078B3
:10615000800700F1D880DFF8F40304680420DFF83A
:10616000E0130870CFE0DFF8DC0304680320DFF8F9
:10617000D0130870C7E0DFF8BC030068C0F340101C
:10618000002876D0DFF8CC030078800707D5DFF849
:10619000C40304680120DFF8A8130870B3E0DFF837
:1061A00094030068C0F38000C0070AD5DFF89803A5
:1061B0000078800705D502240220DFF884130870D8
:1061C000A1E0DFF870030068C0F34000C0070AD503
:1061D000DFF878030078800705D502240420DFF873
:1061E000601308708FE0A0073BD5DFF854030078F8
:1061F000022804D0DFF848030078042831D1DFF802
:1062000040030078022813D1DFF828030068C0F3A8
:106210008000C0070CD5DFF830030078800707D472
:10622000DFF8240304680220DFF8141308706AE022
:10623000DFF80C030078042865D1DFF8F802006865
:10624000C0F34000C0075ED5DFF800030078800788
:1062500059D4DFF8F80204680420DFF8E41208706B
:1062600051E0DFF8F00204680120DFF8D412087072
:1062700049E0B0480068C0F38000002838D0B24838
:106280000078800705D5B04804680220AC49087042
:1062900039E0A8480068C0F34000C00708D5AB4803
:1062A0000078800704D502240420A54908702AE05C
:1062B000A00717D5A2480078042813D1A048007879
:1062C000042820D19B480068C0F34000C0071AD5BD
:1062D0009E480078800716D49C480468042098499A
:1062E000087010E0984804680220954908700AE098
:1062F00090480068C0F34000002804D09348046828
:1063000004208F4908708B48006830F010008949DC
:1063100008608848006830F00400864908608548B5
:10632000006830F0020083490860200010BD80B58D
:1063300000208149086080480068C0437F490860A8
:1063400000F07DFA10F0290F0AD17C4801687A48E4
:10635000007800F0FF0050EA0120042100F056FA16
:1063600001BD80B55FF4802009F0A1FB002809D0B1
:106370000220784908606F48006850F020006D499D
:106380000860D5E05FF4802009F09BFB002809D06D
:106390000020704908606748006850F02000654997
:1063A0000860C5E05FF4003009F081FB002809D0E7
:1063B0000120684908605F48006850F020005D498E
:1063C0000860B5E05FF4003009F07BFB002809D0DD
:1063D0000020604908605748006850F02000554987
:1063E0000860A5E04FF4805009F061FB002809D057
:1063F0004020584908604F48006850F020004D493F
:10640000086095E04FF4805009F05BFB002809D04C
:106410000020504908604748006850F02000454976
:10642000086085E05FF4803009F041FB002809D066
:106430002020484908603F48006850F020003D494E
:10644000086075E05FF4803009F03BFB002809D05C
:106450000020404908603748006850F02000354966
:10646000086065E04FF4004009F021FB002809D0E6
:106470000820384908602F48006850F020002D4956
:10648000086055E04FF4004009F01BFB002809D0DC
:106490000020304908602748006850F02000254956
:1064A000086045E04FF4804009F001FB002809D066
:1064B0001020284908601F48006850F020001D493E
:1064C000086035E04FF4804009F0FBFA002809D05D
:1064D0000020204908601748006850F02000154946
:1064E000086025E04FF4005009F0E1FA002809D0D7
:1064F0000420184908600F48006850F020000D493A
:10650000086015E04FF4005009F0DBFA002809D0CC
:106510000020104908600748006850F02000054935
:10652000086005E00348006830F020000149086079
:1065300001BD0000982C0020902C0020942C0020FD
:106540006D2E0020A02C0020A42C00209C2C0020CC
:10655000A82C0020AC2C002001000020C9B20A2980
:1065600001D102205FE0C9B2112902D0C9B20B29C2
:1065700001D1402057E0C9B20E2901D1442052E098
:10658000C9B20D2901D150204DE0C9B2102901D165
:10659000542048E0C9B20C2901D1482043E0C9B2D7
:1065A0000F2901D14C203EE0C9B2122902D0C9B254
:1065B000082901D1012036E0C9B2092901D10520FD
:1065C00031E0C9B2132902D0C9B2062902D150F074
:1065D000200028E0C9B2072901D1242023E0C9B254
:1065E000022902D0C9B2162902D150F008001AE0DF
:1065F000C9B2032901D10C2015E0C9B2042902D087
:10660000C9B2172902D150F010000CE0C9B2052917
:1066100001D1142007E0C9B2012902D0C9B214295E
:1066200001D150F004007047810701D50A203CE0F9
:10663000C10705D5400701D5092036E0082034E020
:10664000410615D5010705D5400701D50F202CE0DF
:106650000C202AE0C10605D5400701D5102024E012
:106660000D2022E0400701D50E201EE00B201CE08B
:10667000810605D5400701D5072016E0062014E065
:10668000010705D5400701D503200EE002200CE0EC
:10669000C10605D5400701D5052006E0052004E028
:1066A000400701D5012000E00020C0B27047000083
:1066B00038B5044600F029F8624D0321296000F046
:1066C00024F80120E40900FA04F45F48E44304607C
:1066D00000F01BF8002028600A20BDE83240FEF7D9
:1066E0003DBF10B500F011F8564C0321216000F0B9
:1066F0000CF855490020086000F007F800202060E1
:106700000A20BDE81040FEF729BF0A20FEF726BF89
:1067100010B50220FEF722FF4C4C2168C807FCD4BC
:10672000606810F00C0F0CD14948FEF7B9FE02204A
:10673000FEF714FF2068C107FCD4606810F00C0F4E
:1067400001D0022010BD002010BD10B5414B8C09B6
:106750001C60C1F38301920859600AD004E05968B3
:1067600011B91C68641C1C60521E196940F8041B96
:10677000F5D110BD2DE9F84F81468A46354D68693F
:10678000C007FCD4DFF8D080344F354E4FEA9A1062
:1067900028609408CAF38300686005D12AE068681D
:1067A00010B92968491C296030683840404505D136
:1067B0003068010404BF5046FFF77AFFD9F80000A3
:1067C0002861FFF7A2FFD5F814B05FEACB70FAD4C6
:1067D0005FEACB600AD530680740474504D130688E
:1067E000010408BFFFF77DFF58460DE0641E09F164
:1067F0000409D4D130680740474504D1306801040A
:1068000008BFFFF76EFF6869BDE8F28F38B50D4627
:106810001349114B0A680446104802409A4205D1B8
:106820000968080404BF2846FFF742FF0948A90980
:106830000160C5F3830141600461406932BD0348D2
:1068400000687047FCD00F40C0E20A4018F00A40D0
:10685000005800F004F00A40000005100000FF702E
:1068600000E00F400548016841F470010160704785
:106870000348016841F040410160704788ED00E045
:1068800034EF00E00448016841F005010160704701
:106890000249401E0860704710E000E014E000E08C
:1068A0004C49FFE7012008607047012100F01F00FC
:1068B00001FA00F0484908607047012100F01F000C
:1068C00001FA00F045490860704745490860704783
:1068D00000F01F00012202FA00F0424ACB0748BF35
:1068E00010608B0748BF90614B0748BF10620907D3
:1068F00048BF906070473A4A126800F03F0002EBD0
:106900000012394893680340194391607047F0B50D
:10691000334C2568354C00F03F0005EB0016B76896
:106920002740840604D5042914BF062941F001013B
:10693000DDF814C0ACF1010E41EA0E14274307F054
:106940004064B4F1406F04D0A40E0CFA04F4A21811
:10695000521E326007F04042B2F1404F0FD004297E
:1069600018BF062906D140F0200005EB001000F109
:106970000C0304E0920F0CFA02F003445B1E7360F8
:10698000B760F0BD1649096800F03F0001EB001048
:10699000806800F007004108490004291EBF420832
:1069A0005200062A04BF40084000704700F0FF0173
:1069B00010B5CB080E4A02EB8302890001F01C01DE
:1069C00013680F248C40000CA343884018431060C8
:1069D00010BD000004F00F4028F00F402CF00F40D5
:1069E00008F00F401CF00F40F73FFC0008C0FFFF0D
:1069F00010F50F401AE050F8081F41F00201016045
:106A0000704700F5406001210160704700F540606B
:106A1000014901607047000051E5CC1A00F5406063
:106A20000068012818BF0020704700BF50F8081FF9
:106A300041F001010160704700F58360016841F495
:106A4000807101607047000080B500200090DFF881
:106A5000380C006840084000DFF82C1C0860042354
:106A6000E0226946DFF8240C02F08BFF0028F6D004
:106A700000980128FCD00423E4226946DFF8980C32
:106A800002F07FFF0028F6D000980128FCD0DFF844
:106A9000FC0B0078FBF7ADFB002814D0DFF8EC0B03
:106AA0004078FBF7A6FB00280DD0DFF8E00B8078DC
:106AB000FBF79FFB002806D0DFF8D00BC078FBF770
:106AC00098FB00280AD1022001F029FADFF8B80B60
:106AD000006850F00200DFF8B01B0860DFF8380CE7
:106AE0000078FBF786FB002814D0DFF82C0C4078E8
:106AF000FBF77FFB00280DD0DFF81C0C8078FBF73C
:106B000078FB002806D0DFF8100CC078FBF771FB8B
:106B100000280AD1012001F002FADFF86C0B0068AE
:106B200050F00400DFF8601B0860DFF85C0B0068C1
:106B300050F00100DFF8501B086001BD80B5DFF8A0
:106B4000480B0078C0072ED5DFF83C0B0068C0F377
:106B50004000002810D00422E021DFF8300B02F0C2
:106B600057FF01281FD1DFF8200B006830F002002A
:106B7000DFF8141B086016E0DFF80C0B0068C0F3A8
:106B8000800000280FD00422E421DFF88C0B02F0F3
:106B90003FFF012807D1DFF8F00A006830F0040059
:106BA000DFF8E41A086001BD80B5022001F0B7F9F2
:106BB000012001F0B4F9DFF8D00A006850F00400B9
:106BC000DFF8C41A0860DFF8C00A006850F002005D
:106BD000DFF8B41A086001BDDFF8AC0A007810F0E5
:106BE000060F01D0012000E00020704770B50D00B5
:106BF00014001A00DFF8241B802606FB04F631443B
:106C000000F0F1F8012840F0DA80DFF8100B802165
:106C100001FB04F108444078BB2811D12300002275
:106C20000021FF2001F0E1F8002C00F0BE80012CD3
:106C300040F0BB800022002100200AF0E5F9B4E01A
:106C4000DFF8D80A802101FB04F108448078DFF8DE
:106C5000D01A08600020DFF8CC1A802202FB04F270
:106C600011444870DFF8B80A0068012832D00228C1
:106C700035D0032838D006286AD007286CD00828D9
:106C800037D00A287CD00B2876D00D283DD00E288E
:106C90007AD00F2868D010282FD02F2850D0522813
:106CA00014D081283DD0822840D0832843D0852825
:106CB0005ED0872848D088282FD08F2850D09028A1
:106CC0001FD09D2825D0A22862D068E0200000F0C7
:106CD0003DF96AE00021200000F0C2F965E00121E1
:106CE000200000F0BDF960E00221200000F0B8F9BA
:106CF0005BE0200001F068FC57E0200000F0B7FAEC
:106D000053E0200000F008FB4FE0200000F0E1FA23
:106D10004BE0200000F072FB47E0200000F0B8FCE0
:106D200043E00021200000F024FA3EE00121200091
:106D300000F01FFA39E00221200000F01AFA34E0D6
:106D4000200000F013FE30E0200000F0EDFC2CE00D
:106D5000200000F044FE28E0200000F05AFE24E06D
:106D6000200000F0DDFE20E0200000F050FF1CE0DD
:106D7000200000F0B2FF18E0200000F09BFB14E0C0
:106D8000200000F057FC10E0200000F059FE0CE05D
:106D900023000022A221F02001F027F805E02300C3
:106DA00000220021FF2001F020F82900DFF87429DB
:106DB0008020444302EB040000F08FF812E0022828
:106DC0000FD1230000220021FF2001F00EF829003E
:106DD000DFF850298020444302EB040000F07DF8E6
:106DE00000E0002070BD2DE9F84305000E000024EE
:106DF000002000E0401C904205D2295C0329F9D113
:106E0000002129540400904201D2002C01D100201D
:106E100061E0671E00E07F1E002F5BD4E85D022862
:106E2000F9D10020E855E41B641C092C01D2022092
:106E300051E0083CE00701D502204CE06408002C3A
:106E400001D07D2C01D3022045E0D81EA04201D301
:106E5000032B01D203203EE0781C411C695C285CB6
:106E600000F0F2FF30703078844201D0022032E02E
:106E70005FF00108F81C411C695C285C00F0E4FF2D
:106E80007070707818EB00085FF0000913E017EBE2
:106E90004900401D411C695C285C00F0D5FF06EBF1
:106EA00009018870A14504D206EB0900807858FAE0
:106EB00080F819F101094C45E9D27FEA080808F089
:106EC000FF0806EB04008078804501D0022002E034
:106ED000012000E00020BDE8F283F8B505000E00B7
:106EE000012702203070002413E0285D0009FAF722
:106EF000E0FE06EB44014870285D10F00F00FAF741
:106F0000D8FE06EB44018870002C01D0285D3F18A4
:106F1000641C2878801C8442E7D3FF4307F0FF07F6
:106F200038000009FAF7C5FE06EB4401487017F077
:106F30000F073800FAF7BDFE06EB44018870032006
:106F400006EB4401C8706000001DF2BD10B582B0B0
:106F50000400DFF8C807802101FB04F10844C07871
:106F60008DF80000DFF8B407802101FB04F108442C
:106F700000798DF80100DFF8A407802101FB04F1FE
:106F8000084440798DF80200DFF89007802101FB6A
:106F900004F1084480798DF80300684600F063FF2F
:106FA00000280BD1684600F080FF002806D123009E
:106FB00000225221F82000F018FF50E0DFF85C07B3
:106FC000802101FB04F10844007AC04300F0FF0077
:106FD000DFF84817802202FB04F21144C979884285
:106FE00006D0230000225221FF2000F0FEFE36E0F2
:106FF000012C18D10AF057F8002806D123000022EE
:107000005221F92000F0F1FE29E00AF04FF80028A3
:107010001FD1DFF80807802101FB04F10844C07983
:10702000FEF733FF15E0022C13D10AF07DF900289A
:1070300006D1230000225221F92000F0D6FE0EE0F6
:10704000DFF8D806802101FB04F10844C079FEF77F
:1070500038FF230000225221F02000F0C6FE13BDAD
:10706000F8B505000C00002C01D1012604E0012C2C
:1070700001D1022600E00326012D0AD10AF013F8FF
:1070800000281ED12B0000223100F92000F0ADFEB7
:107090006EE0022D0AD10AF047F9002811D12B0029
:1070A00000223100F92000F0A0FE61E0FAF7E0FADA
:1070B000002806D12B0000223100F92000F095FEB7
:1070C00056E02120DFF85C16802202FB05F288548E
:1070D000002C08D18120DFF84C16802202FB05F23B
:1070E0001144887012E0012C08D18220DFF8341698
:1070F000802202FB05F21144887007E08320DFF84C
:107100002416802202FB05F21144887000261DE03F
:10711000DFF81006802101FB05F1084400EB0607AB
:1071200040213000FCF769FBF8700EE0012CEFD134
:10713000DFF8F005802101FB05F1084400EB0607AC
:1071400020213000FCF759FBF870761C202E0FD25E
:10715000002CEBD1DFF8CC05802101FB05F10844C0
:1071600000EB060700213000FCF747FBF870ECE766
:10717000F1BD70B58AB005000C00DFF8A0058021D4
:1071800001FB05F10844C0788DF80000DFF88C059C
:10719000802101FB05F1084400798DF80100DFF83A
:1071A0007C05802101FB05F1084440798DF802003F
:1071B000DFF86805802101FB05F1084480798DF82E
:1071C0000300002C01D1812604E0012C01D182268C
:1071D00000E08326684600F068FE002806D12B00F8
:1071E00000223100F82000F000FE3EE0012D36D1F3
:1071F00009F059FF002806D12B0000223100F920A8
:1072000000F0F3FD31E009F051FF002820D100200B
:107210000AE0DFF80815802202FB05F21144014460
:10722000C97901AA1154401C2028F2D3002C04D1A2
:10723000002101A8FCF7E8FA0AE0012C04D1202182
:1072400001A8FCF7E1FA03E0402101A8FCF7DCFA11
:107250002B0000223100F02000F0C7FD05E02B00DC
:1072600000223100F92000F0C0FD0AB070BDF8B571
:107270000400DFF8A804802101FB04F10844C5796B
:107280002220DFF8A014802202FB04F28854902010
:10729000DFF89014802202FB04F211448870DFF8BA
:1072A0008404802101FB04F10844C57000260DE030
:1072B000DFF87004802101FB04F1084400EB0607AD
:1072C0003100280002F04CF83871761C202EEFD3E4
:1072D000F1BD70B504002120DFF84814802202FBC4
:1072E00004F288549D20DFF83C14802202FB04F253
:1072F0001144887000250CE0DFF82804802101FB90
:1073000004F1084400EB0506280002F035F8F0709F
:107310006D1C202DF0D370BD70B582B00400DFF875
:10732000FC03802101FB04F10844C0788DF80000C3
:10733000DFF8E803802101FB04F1084400798DF8AF
:107340000100DFF8D803802101FB04F108444079F3
:107350008DF80200DFF8C403802101FB04F108442A
:1073600080798DF80300684600F09FFD002806D163
:10737000230000229021F82000F037FD3DE0012C91
:1073800035D109F090FE002806D12300002290217B
:10739000F92000F02AFD30E0DFF88003802101FBB6
:1073A00004F10844C579082D06D32300002290215A
:1073B000FF2000F01AFD20E009F078FE00280FD130
:1073C00000260BE0D548802101FB04F1084430443D
:1073D000027A3100280001F0D7FF761C202EF1D36D
:1073E00023002A009021F02000F0FFFC05E023009C
:1073F00000229021FF2000F0F8FC73BD38B5040096
:10740000C648802101FB04F10844C0788DF80000D3
:10741000C248802101FB04F1084400798DF8010085
:10742000BE48802101FB04F1084440798DF8020038
:10743000BA48802101FB04F1084480798DF80300EB
:10744000684600F032FD002806D1230000229D216D
:10745000F82000F0CAFC2CE0012C24D109F023FE16
:10746000002806D1230000229D21F92000F0BDFC58
:107470001FE009F01BFE00280ED100250AE0A748F6
:10748000802101FB04F108442844C179280001F05F
:10749000A2FF6D1C202DF2D3230000229D21F0209D
:1074A00000F0A3FC05E0230000229D21F92000F05C
:1074B0009CFC31BD70B504009848802101FB04F1AB
:1074C0000844C57813209749802202FB04F28854AF
:1074D0008B209449802202FB04F211448870914869
:1074E000802101FB04F10844C570280002F03BFE36
:1074F0008C49802202FB04F211440871280002F03A
:10750000F7FD8849802202FB04F211444871010012
:10751000090A844A802303FB04F31A449171010091
:10752000090C804A802303FB04F31A44D171000E36
:107530007C49802202FB04F211440872280002F008
:10754000F4FD784A802303FB04F31A4450720200CE
:1075500092B2120A734B802606FB04F633449A72E9
:107560000200120C6F4B802606FB04F63344DA72DD
:107570000200120E6B4B802606FB04F633441A738E
:10758000684A802303FB04F31A44517402000B0081
:107590001A0A0023634B802606FB04F633449A74D0
:1075A00002000B001A0C00235E4B802606FB04F63B
:1075B0003344DA74880D00215A49802202FB04F218
:1075C00011440875280002F0EBFD5649802202FBA9
:1075D00004F2114448730100090A524A802303FB54
:1075E00004F31A4491730100090C4E4A802303FBF3
:1075F00004F31A44D173000E4A49802202FB04F2BC
:107600001144087402F00CFE06002800FAF7E1FDB0
:10761000304207D00121434A8020444302EB04005A
:10762000417406E000213F4A8020444302EB0400FD
:10763000417470BD10B504003848802101FB04F18D
:107640000844C0783549802202FB04F211440979CC
:1076500050EA012002F0ECFD3048802101FB04F1EA
:10766000084440792D49802202FB04F211448979B3
:1076700050EA012002F0E0FD230000220A21F02060
:1076800000F0B3FB10BD0000F42B0020EC2B002019
:1076900010B504002148802101FB04F10844807DDD
:1076A0001E49802202FB04F21144C97D71F0FF01E2
:1076B000C943884206D0230000228821FF2000F021
:1076C00094FB27E0012C10D11449802202FB04F224
:1076D000114491F823201149802303FB04F319443A
:1076E00091F8221009F090FC11E0022C0FD10B4907
:1076F000802202FB04F2114491F8232007498023E1
:1077000003FB04F3194491F8221009F0F5FD200061
:1077100000F05AFF10BD0000F02B00209C1200204A
:10772000F82B00201C14002010B582B00400DFF8F4
:10773000FC0B802101FB04F10844C0788DF80000A7
:10774000DFF8E80B802101FB04F1084400798DF893
:107750000100DFF8D80B802101FB04F108444079D7
:107760008DF80200DFF8C40B802101FB04F108440E
:1077700080798DF80300012C40F0F18009F093FC32
:10778000002800F0EC80684600F08FFB012840F0F4
:107790008F80DFF8980B802101FB04F10844C07949
:1077A00001283AD109F082FC00282FD1DFF87C0BA8
:1077B000802101FB04F10844007ADFF8741B087093
:1077C000DFF8680B802101FB04F10844407ADFF800
:1077D000601B4870DFF8540B802101FB04F1084462
:1077E000807ADFF84C1B8870DFF8400B802101FBAA
:1077F00004F10844C07ADFF8381BC870DFF8BC0D0C
:10780000006850F00400DFF8B41D08602300002277
:107810008721F02000F0E9FAA7E0DFF8100B8021C3
:1078200001FB04F10844C07902283AD109F03EFC7A
:1078300000282FD1DFF8F40A802101FB04F108446D
:10784000007ADFF87C1D0870DFF8E00A802101FB78
:1078500004F10844407ADFF8681D4870DFF8CC0A6C
:10786000802101FB04F10844807ADFF8541D887000
:10787000DFF8B80A802101FB04F10844C07ADFF880
:10788000401DC870DFF8340D006850F00200DFF8CA
:107890002C1D0860230000228721F02000F0A5FAAB
:1078A00063E0230000228721F82000F09EFA5CE0CC
:1078B000684600F0D8FA01284AD1DFF8700A802122
:1078C00001FB04F10844C07902283AD109F0EEFB2B
:1078D00000282FD1DFF8540A802101FB04F108446D
:1078E000007ADFF8DC1C0870DFF8400A802101FB19
:1078F00004F10844407ADFF8C81C4870DFF82C0A0D
:10790000802101FB04F10844807ADFF8B41C887000
:10791000DFF8180A802101FB04F10844C07ADFF87F
:10792000A01CC870DFF8940C006850F00200DFF86B
:107930008C1C0860230000228721F02000F055FAFB
:1079400013E0230000228721F82000F04EFA0CE01B
:10795000230000228721F82000F047FA05E02300E9
:1079600000228721F92000F040FA13BD80B5030002
:10797000012B2ED10920DFF84C1C802202FB03F2E0
:107980008854A120DFF83C1C802202FB03F2114442
:10799000887000200BE0DFF82C1C802202FB03F231
:1079A00011440144DFF88829125CCA70401C042885
:1079B000F1D30020042811D2DFF8081C802202FB3A
:1079C00003F211440144DFF8F82B125CCA71401C29
:1079D000F0E700222F21F92000F007FA01BD10B5D1
:1079E0000400012C0ED109F05EFB002803D020001A
:1079F00000F0C9FA0CE0230000220621F92000F073
:107A0000F4F905E0230000220621F82000F0EDF94A
:107A100010BD10B50400012C0ED109F044FB8428E0
:107A200003D1200000F086FC09E02300002207219A
:107A3000F92000F0DAF902E0200000F07BFC10BD34
:107A400010B50400012C64D109F02DFB002860D092
:107A50000A20DFF8701B802202FB04F28854912078
:107A6000DFF8601B802202FB04F2114488700220C0
:107A7000F9F719FEDFF84C1B802202FB04F21144D7
:107A8000C870F9F714FEDFF83C1B802202FB04F2F9
:107A9000114408710100090ADFF8282B802303FB39
:107AA00004F31A4451710100090CDFF8182B8023EC
:107AB00003FB04F31A449171800BDFF8081B80224A
:107AC00002FB04F21144C87100200020C046DFF818
:107AD000F41A802202FB04F2114408720100090A20
:107AE000DFF8E02A802303FB04F31A4451720100FB
:107AF000090CDFF8D02A802303FB04F31A449172A7
:107B0000800BDFF8C02A80214C4302EB0401C872CD
:107B100005E0230000220E21F92000F066F910BDD7
:107B200010B582B00400DFF80408802101FB04F1E5
:107B30000844C0788DF80000DFF8F007802101FBD1
:107B400004F1084400798DF80100DFF8E007802196
:107B500001FB04F1084440798DF80200DFF8CC07FE
:107B6000802101FB04F1084480798DF80300684608
:107B700000F079F9012804D0684600F096F9012850
:107B80003ED109F093FA002831D1DFF8A007802117
:107B900001FB04F10844C179012009F0D5FCDFF8AC
:107BA0008C07802101FB04F10844017A022009F0CE
:107BB000CBFCDFF87807802101FB04F10844417A0F
:107BC000032009F0C1FCDFF86407802101FB04F108
:107BD0000844C17A042009F0B7FCDFF8500780217F
:107BE00001FB04F10844017B052009F0ADFC2300F2
:107BF0000022DFF8E40B0168F02000F0F6F805E061
:107C0000230000228F21F82000F0EFF813BD10B5FB
:107C100004000A20DFF8AC19802202FB04F2885429
:107C20007820DFF8A019802202FB04F2114488704A
:107C30000220F9F738FDDFF88C19802202FB04F2EC
:107C40001144C8700020F9F72EFDDFF87819802262
:107C500002FB04F2114408710120F9F724FDDFF85A
:107C60006419802202FB04F211444871022009F0D9
:107C700015FADFF85019802202FB04F211448871D2
:107C8000002009F00BFADFF83C19802202FB04F215
:107C90001144C871012009F001FADFF82819802287
:107CA00002FB04F2114408720020DFF81819802248
:107CB00002FB04F2114448720020DFF80819802208
:107CC00002FB04F2114488720021DFF8F8288020BA
:107CD000444302EB0400C17210BD10B582B0040031
:107CE000DFF84806802101FB04F10844C0788DF8D4
:107CF0000000DFF83806802101FB04F10844007918
:107D00008DF80100DFF82406802101FB04F108440E
:107D100040798DF80200DFF81406802101FB04F1A0
:107D2000084480798DF80300684600F0BEF800280A
:107D300006D1230000228521F82000F056F853E0F8
:107D4000DFF8E805802101FB04F10844C079000652
:107D5000DFF8D815802202FB04F21144097A10EBF7
:107D60000140DFF8C815802202FB04F21144497A71
:107D700010EB0120DFF8B415802202FB04F211445D
:107D8000897A50FA81F0C10704D5F8F717FB02F0A1
:107D900057FA23E0810702D5F8F75AFF1EE0810168
:107DA00002D501F018F819E0410703D50120FBF7CF
:107DB0009DFB13E0002805D501214FF40050FBF78F
:107DC000F0FB0BE0410005D501214FF40050FBF71B
:107DD00001FC03E0400601D502F0FFF92300002278
:107DE0008521F02000F001F813BD70B40424DFF801
:107DF000D457802606FB03F6AC550024DFF8C457A1
:107E0000802606FB03F635446C70DFF8B847802502
:107E100005FB03F52C44A070DFF8A807802404FBC1
:107E200003F42044C170DFF89C07802101FB03F1BB
:107E300008440271120ADFF88C178020434301EBDB
:107E40000300427170BC704738B50C00C0B2F9F73E
:107E50001DFF05002D012000C0B2F9F717FF4519DD
:107E60002800C0B232BD0178DFF854271278914261
:107E700001D0002018E04178DFF844275278914281
:107E800001D0002010E08178DFF834279278914209
:107E900001D0002008E0C078DFF82417C9788842B4
:107EA00001D0002000E0012070470178DFF8802435
:107EB0001278914201D0002118E04178DFF8702457
:107EC0005278914201D0002110E08178DFF86024DF
:107ED0009278914201D0002108E0C178DFF8502467
:107EE000D278914201D0002100E00121002914D173
:107EF0000178332901D000210FE04178312901D0E8
:107F000000210AE08178302901D0002105E0C07805
:107F1000312801D0002100E001210800704702282B
:107F200018D13020DFF8981608703020DFF890164E
:107F300048703020DFF8881688703020DFF880160F
:107F4000C870DFF87806006850F00200DFF86C16A1
:107F5000086017E03020DFF8D81308703020DFF811
:107F6000D01348703020DFF8C81388703020DFF855
:107F7000C013C870DFF84406006850F00400DFF852
:107F80003C160860704738B504002720DFF8341627
:107F9000802202FB04F288548620DFF82816802213
:107FA00002FB04F2114488705FF0FF30F9F715FD11
:107FB0000100090EDFF80C26802303FB04F31A44AA
:107FC000D1700100090CDFF8FC25802303FB04F3CA
:107FD0001A4411710100090ADFF8E825802303FB28
:107FE00004F31A445171DFF8DC15802202FB04F21D
:107FF000114488710025002008F0CAFC012801D135
:1080000055F00105012008F0C3FC012801D155F00D
:108010000205DFF8B005802101FB04F10844C571B9
:108020005FF0FF30F9F7D9FC002809D0F9F7E8FC38
:10803000DFF89015802202FB04F21144087207E079
:108040000020DFF88015802202FB04F21144087240
:108050005FF0FF300F21F9F7CDFC0100090EDFF8CA
:108060006425802303FB04F31A4451720100090CB8
:10807000DFF85025802303FB04F31A4491720100BA
:10808000090ADFF84025802303FB04F31A44D17268
:10809000DFF83015802202FB04F211440873002C33
:1080A0001AD14FF48040F9F798FC002802D1F4F778
:1080B00035FA00E000200100090ADFF808258023D6
:1080C00003FB04F31A445173DFF8F814802202FB17
:1080D00004F21144887316E05FF0FF300F21F9F7C6
:1080E00089FC02000B001A0A0023DFF8D83480252F
:1080F00005FB04F52B445A73DFF8C804802202FB09
:1081000004F2104481735FF0FF3007F0D0FC0100EF
:10811000090EDFF8B024802303FB04F31A44D17363
:108120000100090CDFF89C24802303FB04F31A44AC
:1081300011740100090ADFF88C24802303FB04F387
:108140001A445174DFF87C14802202FB04F21144BB
:1081500088747FF0704007F0A0FC0100090EDFF882
:108160006424802303FB04F31A44D1740100090C36
:10817000DFF85024802303FB04F31A441175010037
:10818000090ADFF84024802303FB04F31A445175E5
:10819000DFF83014802202FB04F21144887500F0ED
:1081A000DCFD0100090EDFF81C24802303FB04F32F
:1081B0001A44D1750100090CDFF80824802303FB61
:1081C00004F31A4411760100090ADFF8F82380232A
:1081D00003FB04F31A445176DFF8E813802202FB14
:1081E00004F211448876FDF7B4FCDFF8D81380223E
:1081F00002FB04F21144C876000ADFF8C81380229B
:1082000002FB04F21144087704F074FBDFF8B413A6
:10821000802202FB04F211444877002C13D108207D
:10822000F9F7CEFB0020DFF89C13802202FB04F25A
:10823000114488770020DFF88C13802202FB04F2BF
:108240001144C8770FE01E20FBF7DEF9DD498022DC
:1082500002FB04F2114488770020DA49802202FBF5
:1082600004F21144C877F9F7B1FBD649802202FB2A
:1082700004F2114481F820004FF48040F9F7ADFB7F
:10828000002803D1F4F74AF9C04301E05FF0FF3062
:108290000100090ACB4A802303FB04F31A4482F845
:1082A0002110C849802202FB04F2114481F8220007
:1082B000012009F023F9C349802202FB04F2114492
:1082C00081F82300022009F019F9BE49802202FB3F
:1082D00004F2114481F82400032009F00FF9B94990
:1082E000802202FB04F2114481F82500062009F0E7
:1082F00005F9B449802202FB04F2114481F82600FA
:10830000042009F0FBF8AF49802202FB04F211447B
:1083100081F82700052009F0F1F8AA4A80214C4392
:1083200002EB040181F8280031BD00009C120020FE
:10833000F02B002038B504002720A249802202FB40
:1083400004F2885477209F49802202FB04F21144F2
:1083500088700320FCF723FA9A49802202FB04F27A
:108360001144C870000A9749802202FB04F21144AC
:1083700008710420FCF713FA9249802202FB04F2F0
:1083800011444871000A8F49802202FB04F2114413
:1083900088710120FCF703FA8A49802202FB04F26B
:1083A0001144C871000A8749802202FB04F211447B
:1083B00008720020FCF7F3F98249802202FB04F2E4
:1083C00011444872000A7F49802202FB04F21144E2
:1083D000887200207B49802202FB04F21144C8729B
:1083E00000207849802202FB04F211440873022025
:1083F000FCF7D5F97349802202FB04F2114448735B
:10840000000A7049802202FB04F211448873F4F7D9
:1084100066F80500002D02D46D046D0C03E06D04B8
:108420006D0C55F400456748802101FB04F10844B8
:10843000C5732800000A6349802202FB04F211443C
:108440000874F4F76BF864214D43B5FBF0F05D4917
:10845000802202FB04F21144487400205949802212
:1084600002FB04F21144887400205649802202FB6A
:1084700004F21144C87400205249802202FB04F225
:108480001144087500204F49802202FB04F2114478
:10849000487500204B49802202FB04F21144887584
:1084A000F4F711F84749802202FB04F21144C87521
:1084B000000A4449802202FB04F21144087600209D
:1084C0004049802202FB04F21144487600203D49D5
:1084D000802202FB04F21144887601F094FE3949AF
:1084E000802202FB04F21144C876000A354980223A
:1084F00002FB04F21144087701F078FE3149802232
:1085000002FB04F211444877000A2E49802202FB44
:1085100004F21144887701F0BFFE2A49802202FB51
:1085200004F21144C877000A2649802202FB04F2B3
:10853000114481F8200001F073FE2249802202FBE1
:1085400004F2114481F82100000A1E49802202FB36
:1085500004F2114481F8220001F066FE19498022DC
:1085600002FB04F2114481F82300000A154980221D
:1085700002FB04F2114481F82400002011498022FA
:1085800002FB04F2114481F8250000200D498022ED
:1085900002FB04F2114481F82600002009498022E0
:1085A00002FB04F2114481F827000021054A8020D3
:1085B000444302EB040080F8281031BDF42B002066
:1085C000EC2B00201C14002010B504002920834946
:1085D000802202FB04F2885488208049802202FB1A
:1085E00004F21144887045207C49802202FB04F289
:1085F0001144C87031207949802202FB04F21144F1
:10860000087153207549802202FB04F2114448711D
:108610004C207249802202FB04F211448871002030
:108620006E49802202FB04F21144C87100206B499C
:10863000802202FB04F21144087200206749802264
:1086400002FB04F21144487200206449802202FBBC
:1086500004F21144887200206049802202FB04F277
:108660001144C87200205D49802202FB04F21144CB
:10867000087300205949802202FB04F21144487318
:1086800000205649802202FB04F211448873002026
:108690005249802202FB04F21144C87300204F4962
:1086A000802202FB04F2114408740020F7F782FED6
:1086B0004A49802202FB04F2114448740120F7F772
:1086C00079FE4649802202FB04F211448874FF209F
:1086D0004249802202FB04F21144C874FF203F4942
:1086E000802202FB04F211440875FF203B498022DE
:1086F00002FB04F2114448750420C0463749802229
:1087000002FB04F2114488753448802101FB04F116
:108710000844807DC0433149802202FB04F21144A9
:10872000C875002008E02D49802202FB04F21144A4
:108730000144FF220A76401C0A28F4D3332027493B
:10874000802202FB04F2114481F8220031202349E7
:10875000802202FB04F2114481F8230000201F490B
:10876000802202FB04F2114481F8240000201B49FE
:10877000802202FB04F2114481F8250000201749F1
:10878000802202FB04F2114481F8260000F0E8FA8E
:108790000100090E114A802303FB04F31A4482F8F6
:1087A00027100100090C0D4A802303FB04F31A442F
:1087B00082F828100100090A084A802303FB04F309
:1087C0001A4482F82910054A80214C4302EB040127
:1087D00081F82A0010BD0000F82B00201C14002096
:1087E00038B5DFF82C04006840084000DFF820149A
:1087F0000860002400E0641CB4F5007F4AD208231E
:10880000E20012F580526946DFF8080400EBC4006C
:1088100001F0B7F80028F2D001F04DF901280AD193
:10882000F7F7C4FD0500F7F7C1FD401B0228FAD396
:1088300001F04AF8F0E70821DFF8D80300EBC400A4
:10884000F9F716FA0128D6D1002006E00021DFF85A
:10885000C42302EBC4021154401C0828F6D308229A
:10886000E10011F58051DFF8AC0300EBC40001F02A
:10887000CFF80028F3D001F01EF90128BBD1F7F79B
:1088800095FD0500F7F792FD401B0228FAD301F091
:108890001BF8F0E700F060F900F06EF9DFF87813EC
:1088A0000860DFF86C03006850F00100DFF8601327
:1088B0000860FCF747FEC00605D5312233210220AF
:1088C00000F007F804E031223321012000F001F824
:1088D00031BD70B504000D001600DFF834030078D8
:1088E000C00701D4002078E001200021F9F782F8C8
:1088F0000022002399426FD190426DD1DFF810031E
:10890000007810F00E0F67D15FF00040F9F765F8BE
:10891000002861D1DFF80403006812285AD2DFF87A
:10892000F8020068401CBC490860BB480068B0F50C
:10893000007F02D30020B8490860052008F0DEFD62
:10894000B449B54A126801F83200042008F0D6FD97
:10895000B049B14A126801EBC2014870032008F027
:10896000CDFDAC49AC4A126801EBC201887002200F
:1089700008F0C4FDA749A84A126801EBC201C870FB
:10898000012008F0BBFDA349A34A126801EBC20114
:108990000871A048A049096800EBC10044719D48D6
:1089A0009D49096800EBC10085719A489A49096898
:1089B00000EBC100C67198480068401C9849974A6E
:1089C000126841F8220095480068401C93490860ED
:1089D000012002E0002000E0002070BD80B58C483E
:1089E0000078C00740F19D8089480068C0F34000CE
:1089F000002820D008228B480068C10011F5805162
:108A00008448884B1B6800EBC30001F001F8012883
:108A100040F0878083480068401C82490860814894
:108A20000068B0F5007F7CD37948006830F0020020
:108A30007749086075E076480068C0F3C0000028F8
:108A400029D0002108E00022724B03EBC1031A5425
:108A5000401C0828F7D3491CB1F5007F01D2002043
:108A6000F7E700F079F808224FF48051694800F0E8
:108A7000CFFF012855D16648006830F008006449EE
:108A800008606348006850F00200614908600120F6
:108A90006449086045E05E480068C0F38000002833
:108AA00018D0002108E000225A4B03EBC1031A54EE
:108AB000401C0828F7D3491CB1F5007F01D20020E3
:108AC000F7E700F049F85248006830F004005049D8
:108AD000086026E052480068002822D0504800680C
:108AE000401E0822C10011F580514A4B03EBC00023
:108AF00000F08EFF012814D1012008E0484951F808
:108B00002010474A02EB800242F8041C401C122845
:108B1000F4D300204249486440480068401E3F4961
:108B2000086001BD3A48007810F00A0F01D001201A
:108B300000E000207047C0B2012806D13448006828
:108B400050F008003249086005E03148006850F0F4
:108B500004002F490860704700202F49086000205A
:108B60002E490860002004E000212D4A42F8201020
:108B7000401C1228F8D3704730B593B0002401256B
:108B80003FE0244810F8340064300E90214800EB98
:108B9000C4004078401E0D901E4800EBC400807851
:108BA0000C901C4800EBC400C0780B90194800EBF7
:108BB000C40000790A9000200990164810F835008A
:108BC00064300590134800EBC5004078401E0490C7
:108BD000104800EBC500807803900E4800EBC500FC
:108BE000C07802900B4800EBC5000079019000208E
:108BF000009009A96846F9F783FB002800D42C00EF
:108C00006D1CB5F5007FBCD3200013B030BD000053
:108C1000802C00201C000020782C00207C2C0020C0
:108C2000C8270020842C002080B500207C490860E3
:108C30007C497D4808F090FD7A4800687B490860CF
:108C400001207749086001BD70B5754800680128AA
:108C500040F0828073480068152801D2012000E0AE
:108C6000142070490968714A12688018814209D33A
:108C70006C4801686C48006808F0F6FD69480068B7
:108C80006A490860674801686748006808F03BFE69
:108C90005FF400300021F8F77CFE01200021F8F796
:108CA000A9FE00220023994246D1904244D150208F
:108CB000FAF7AAFC00283FD05120FAF7A5FC0028BB
:108CC0003AD05220FAF7A0FC002835D0032008F053
:108CD00015FC0400042008F011FC0500052008F034
:108CE0000DFC06005220FAF78FFCB04205D25FF46B
:108CF00000300021F8F775FE1EE05220FAF784FCE0
:108D0000864219D15120FAF77FFCA84205D25FF4C0
:108D100000300021F8F765FE0EE05120FAF774FCF0
:108D2000854209D15020FAF76FFC844204D35FF4E6
:108D300000300021F8F755FE4020FAF765FC3C4969
:108D4000884200D33A4837490968814204D35FF426
:108D500000300021F8F745FE70BD324800687047CA
:108D600031480068704780B52E48006810F1010F47
:108D700004D02C480068401C2A4908602A48006832
:108D800010F1010F04D028480068401C26490860F3
:108D9000244801682448006808F0D3FD01BD80B56F
:108DA00000202149086000201E4908601D48006815
:108DB0001E4908605FF400300021F8F7EAFD5FF417
:108DC00080100021F8F7E5FD164801681648006894
:108DD00008F04AFD01BD80B5002012490860114825
:108DE0000068124908605FF400300021F8F7D1FDF7
:108DF0005FF480100021F8F7CCFD0A4801680A48AA
:108E0000006808F031FD01BD80B5064800680749DB
:108E10000860044801680448006808F025FD01BDA9
:108E20002C2B0020242B0020202B0020282B00207E
:108E300040420F0080B508F08BFD02BD38B500241C
:108E400000E0641C082C6DD22023620112F5D07260
:108E50006946DFF8140A6501284400F092FD0028F5
:108E6000F2D000F028FE01280AD1F7F79FFA05009A
:108E7000F7F79CFA401B0228FAD300F025FDF0E733
:108E80002021DFF8E40962011044F8F7F1FE01281F
:108E900025D1002006E00021DFF8CC2963011A4427
:108EA0001154401C2028F6D32022610111F5D07105
:108EB000DFF8B4096301184400F0AAFD0028F3D0DC
:108EC00000F0F9FD0128BCD1F7F770FA0500F7F7BB
:108ED0006DFA401B0228FAD300F0F6FCF0E7DFF849
:108EE00088096101084400F078FB0028A9D12022FC
:108EF000610111F5D071DFF870096301184400F0C9
:108F000087FD0028F3D000F0D6FD012899D1F7F7AE
:108F10004DFA0500F7F74AFA401B0228FAD300F091
:108F2000D3FCF0E71C234FF438726946DFF83C09A4
:108F300000F027FD0028F5D000F0BDFD01280AD182
:108F4000F7F734FA0400F7F731FA001B0228FAD3D6
:108F500000F0BAFCF0E71C21DFF81009F8F788FEF2
:108F6000012820D1002004E00021DFF8002911545D
:108F7000401C1C28F8D31C224FF43871DFF8EC0891
:108F800000F046FD0128F6D000F095FD01280AD139
:108F9000F7F70CFA0400F7F709FA001B0228FAD3D6
:108FA00000F092FCF0E7DFF8C808406850F00100DC
:108FB000DFF8BC18486031BD70B5DFF8B40800793F
:108FC000C00740F18381DFF8A8084068C0F3800043
:108FD000002825D0DFF89808406830F00400DFF85A
:108FE00090184860002009E00022DFF87C38440136
:108FF00023441A54491C2029F6D3401C082801D2C6
:109000000021F8E7002404E00021200000F0E3F94B
:10901000641C1C2CF8D3DFF85C08DFF854180860D7
:10902000DFF84C080068002830D0DFF844080068FA
:10903000F8F745FE0400082C17D22022610111F533
:10904000D071DFF824086301184400F0E1FC012826
:109050001CD12000F9F7BDF8DFF81418096831EACF
:109060000000DFF80C18086010E01C224FF4387183
:10907000DFF8F80700F0CCFC012807D1DFF8F00793
:10908000006830F08050DFF8E81708605FF080502B
:109090000021F8F77EFC10200021F8F77AFC00F0A0
:1090A00016F9002814D1DFF8C8074068C0F3C000E3
:1090B000002804D0002200210E20FFF70AFCDFF870
:1090C000B007406830F00800DFF8A4174860FDE002
:1090D000DFF89C074068C0F3C000002804D10022DC
:1090E00001210E20FFF7F5FBDFF88407406850F000
:1090F0000800DFF87C1748605FF080500021F8F727
:1091000070FC01200021F8F775FC00220023994231
:1091100001D1904200D0D9E00020062008F0EEF9FD
:10912000050000240CE0200000F076FB012806D1A9
:10913000200000F0D8F9012801D107250A24641C79
:10914000062CF0D310200021F8F723FC002600E0C5
:10915000761C062E80F0A880DFF80C07EDB26901BE
:109160000844052101FB06F1445C002CF0D03100DD
:10917000EDB2280000F04FF90128E9D1DFF8F00640
:10918000406850F01000DFF8E8164860012C03D169
:109190000020FCF73AFE86E0022C03D10220FCF707
:1091A00034FE80E0032C08D11E20FAF72DFA0728A0
:1091B00003D00120FCF729FE75E0042C08D11E2005
:1091C000FAF722FA072803D00320FCF71EFE6AE014
:1091D000072C08D11E20FAF717FA062803D004201E
:1091E000FCF713FE5FE0082C0DD11E20FAF70CFAF5
:1091F000062808D01E20FAF707FA072803D0052012
:10920000FCF703FE4FE0092C08D11E20FAF7FCF909
:10921000062803D00820FCF7F8FD44E00A2C0DD105
:109220001E20FAF7F1F9062808D01E20FAF7ECF90B
:10923000072803D00920FCF7E8FD34E0052C03D112
:109240000620FCF7E2FD2EE0062C08D11E20FAF7DE
:10925000DBF9072803D00720FCF7D7FD23E00B2C10
:1092600008D11E20FAF7D0F9062803D00B20FCF70E
:10927000CCFD18E00D2C08D11E20FAF7C5F9062800
:1092800003D00D20FCF7C1FD0DE00C2C08D11E20F1
:10929000FAF7BAF9062803D00C20FCF7B6FD02E075
:1092A0000020FCF7B2FD11E0DFF8C4054068C0F310
:1092B000001000280AD00020FCF7A7FDDFF8B00559
:1092C000406830F01000DFF8A815486070BD80B528
:1092D0000C20FAF7B6F9012819D14FF4806006F096
:1092E000E6FB002809D0DFF88405006850F0010093
:1092F000DFF878150860012011E0DFF870050068DC
:1093000040084000DFF864150860002007E0DFF83F
:109310005C050078C00701D5012000E0002002BDF7
:10932000DFF84C054068C0F3400000280BD1DFF89F
:1093300040050068002806D1DFF834054068C0F316
:109340008000002801D0012000E000207047DFF8F5
:109350002005406850F00400DFF81415486070479D
:10936000082807D2202905D2DFF8FC244001104448
:10937000405C00E0002070471C2803D2DFF8EC14AA
:10938000085C00E00020704710B50400082C21D2D2
:1093900020291FD2DFF8E00442541F291AD1DFF838
:1093A000D80400F01AF9002008E0DFF8CC14095CBA
:1093B000DFF8B42463011A441154401C2028F4D36C
:1093C000DFF8AC040068012111FA04F40443DFF86B
:1093D000A004046010BD80B51C281BD2DFF89C24BB
:1093E00011541B2816D1DFF8940400F0C4F90020B2
:1093F00006E0DFF88814095CDFF870241154401C83
:109400001C28F6D3DFF86804006850F08050DFF8BD
:109410006014086001BD2DE9F047824689460120AD
:1094200008F06CF80400022008F068F80500DFF886
:1094300038045FEA4A110844052101FB09F1084498
:109440004678DFF824045FEA4A110844052101FB4D
:1094500009F108448778DFF810045FEA4A110844EC
:10946000052101FB09F1084490F80380DFF8F803B7
:109470005FEA4A110144052000FB09F901EB0900EC
:1094800090F80490464503D14F4501D1002028E0D3
:109490003B0032002100280000F065F9012801D1CD
:1094A00001201EE03B0032002100280000F04DF9B1
:1094B000002801D1002014E04B464246210028003C
:1094C00000F051F9012801D100200AE04B46424644
:1094D0002100280000F039F9012801D1002000E026
:1094E0000120BDE8F08738B50400062C01D3002028
:1094F00072E0032008F002F80500042007F0FEFFE8
:109500000100DFF8680300EB84004079002806D0F2
:10951000DFF8580300EB84000079002801D1002017
:109520005AE0DFF8480300EB8400C079002806D039
:10953000DFF8380300EB84008079002801D1002097
:109540004AE0DFF8280300EB84004079814201D231
:10955000002041E0DFF8140300EB8400C07988426A
:1095600001D2002038E0C14800EB840040798142FC
:1095700021D1BE4800EB84000079854201D2002051
:109580002AE0BA4800EB84000079854201D101202D
:1095900022E0B64800EB8400C079814201D201206C
:1095A0001AE0B24800EB84008079A84201D3012080
:1095B00012E0002010E0AD4800EB8400C079814249
:1095C00009D1AA4800EB84008079A84201D200208A
:1095D00002E0012000E0012032BD70B50400012549
:1095E0000026ADE0052000FB06F020444078182856
:1095F00014DA052000FB06F02044C07818280DDAA4
:10960000052000FB06F0204480783C2806DA05207F
:1096100000FB06F0204400793C281DDB00200521DA
:1096200001FB06F1214448700020052101FB06F1F1
:10963000214488700020052101FB06F12144C870F7
:109640000020052101FB06F12144087100200521BD
:1096500001FB06F1605400250A20052101FB06F1FB
:10966000615C88421DD20020052101FB06F12144E6
:1096700048700020052101FB06F12144887000207C
:10968000052101FB06F12144C8700020052101FBE2
:1096900006F1214408710020052101FB06F1605408
:1096A0000025052000FB06F020448378052000FB00
:1096B00006F020444278052000FB06F020440179A2
:1096C000052000FB06F02044C07800F03EF800289A
:1096D00035D1052000FB06F020448378052000FBEF
:1096E00006F020444278052000FB06F02044017972
:1096F000052000FB06F02044C07800F034F8002874
:109700001DD10020052101FB06F1214448700020F5
:10971000052101FB06F1214488700020052101FB91
:1097200006F12144C8700020052101FB06F1214407
:1097300008710020052101FB06F160540025761C0C
:10974000062EFFF44FAF280070BD824201D20120E7
:1097500008E0904205D18B4201D2012002E00020B6
:1097600000E000207047904203D1994201D10120CE
:1097700000E00020704738B50400002549E004EB04
:109780008500007900282ED004EB85004079002860
:1097900029D004EB85008079002824D004EB8500D3
:1097A000C07900281FD004EB8500037904EB850005
:1097B000427904EB8500817904EB8500C079FFF7DD
:1097C000C4FF012824D004EB8500037904EB850055
:1097D000427904EB8500817904EB8500C079FFF7BD
:1097E000C2FF012814D0002004EB8501087100207D
:1097F00004EB85014871002004EB8501887100208D
:1098000004EB8501C87120780221A94088432070AB
:109810006D1C062DB3D331BD002803D1134909783F
:1098200089071DD4012803D110490978490717D4A5
:10983000022803D10D490978090711D4032803D15F
:109840000A490978C9060BD4042803D107490978C5
:10985000890605D4052805D104480078400601D5BD
:10986000012000E000207047801E0020CC2900204D
:10987000E02A0020FF000010AC290020E829002089
:1098800080B50020DFF89C1608600020DFF89816ED
:1098900008600020DFF89416086000F05BFA0028EA
:1098A00004D10120DFF88816086003E00020DFF80B
:1098B00080160860F6F77AFDDFF87816086001BDBB
:1098C000DFF86C060068704780B5DFF85C0600685A
:1098D000002846D1DFF860060068012825D1DFF8AE
:1098E0005C060068401CDFF8541608600020DFF8B2
:1098F00048160860DFF844060068032802D200F02A
:10990000DCFA2EE0DFF838060078002804D10020C9
:10991000DFF83016096808600120DFF810160860CB
:109920000120DFF80C1608601BE0DFF81406007851
:10993000012816D1DFF810060068012811D1F6F7CA
:1099400035FDDFF808160968401A0A2809D3DFF840
:1099500000060168DFF8FC05006800F071FA00F00D
:1099600047FADFF8C8050068012809D1F6F71EFD9F
:10997000DFF8C0150968401A652801D300F07DFAA8
:1099800001BD38B5DFF8A4452468012C04D0DFF808
:10999000A0452468012C01D1002038E00124DFF823
:1099A0008C552C600024DFF894552C600024DFF8DF
:1099B00090552C700124DFF8A0552C60DFF89445F9
:1099C0002260DFF88C251360DFF890251060DFF847
:1099D0007405016001200860DFF874050168DFF894
:1099E0007405006800F02CFA002004E00021DFF884
:1099F00070251154401C2028F8D300F0ABF9002842
:109A000002D100F03AFA01E000F0F2F9012032BD93
:109A100038B5DFF818351B68012B04D0DFF8103596
:109A20001B68012B01D1002044E00123DFF8FC4436
:109A300023600023DFF8044523600B001B0ADFF8D6
:109A400024452370DFF81C355970931CDFF8184546
:109A500023600123DFF814452360002305E0C45C84
:109A6000DFF800551D44AC705B1C9342F7D3002314
:109A7000DFF8FC4423600123DFF8C4442370012392
:109A8000DFF8D44423600023DFF8BC442360DFF810
:109A9000C4341960DFF8B8140A60DFF8C014086035
:109AA00000F058F9002802D100F0E7F901E000F0D9
:109AB0009FF9012032BDDFF874040068704780B55B
:109AC000DFF8B00407F085FFDFF8A80407F08FFF88
:109AD00000281CD0DFF89804006801280AD0DFF8BD
:109AE00088040068002805D00421DFF8880407F006
:109AF0007BFF09E0DFF880040068002804D004211F
:109B0000DFF8700407F070FF00F0B7F921E1DFF82B
:109B10006004006801286DD0DFF84C04006800285C
:109B20002BD1DFF84C040068022840F0958001201A
:109B3000DFF83C14086001225021DFF8380407F0F8
:109B40004FFFDFF834040068012809D10020DFF856
:109B5000281408600721DFF81C0407F045FFF8E02F
:109B6000DFF814040068401EDFF80C1408600B21B5
:109B7000DFF8000407F038FFEBE0DFF8EC030068E3
:109B800001281CD1DFF8E8030068002817D1002065
:109B9000DFF8D4130860DFF8D4030068411CDFF855
:109BA000CC231160DFF8BC13095CDFF8C80307F0B1
:109BB0002AFF0521DFF8BC0307F016FFC9E0DFF834
:109BC000A8030068401EDFF8A0130860DFF89C03BC
:109BD0000068411CDFF894231160DFF88813095CEA
:109BE000DFF8900307F00FFF0121DFF8880307F08B
:109BF000FBFEAEE0DFF87C0308300068DFF87C1382
:109C0000DFF87C2312688854DFF874030068401C76
:109C1000DFF86C130860DFF86003006800281BD0D1
:109C2000DFF854030068012809D10020DFF8481349
:109C300008600521DFF83C0307F0D6FE89E0DFF875
:109C400038030068401EDFF8301308600921DFF890
:109C5000240307F0C9FE7CE0DFF8FC02006801285D
:109C60002DD10020DFF8F0120860B54800780128F7
:109C70000AD1F6F79BFBB54908600120B24908609C
:109C80000020A949086064E0AD480078002813D19D
:109C9000002004E0B949095CB14A1154401CB8499C
:109CA00009688842F6D3AA480168AA48006800F00B
:109CB000C7F800F09DF84CE000F0DFF849E0AD484F
:109CC00007F083FE9E480078002827D1002100205D
:109CD00000E0401CAA4A1268904206D2A04A125CD8
:109CE000A64B1B5C9A42F4D00121012902D100F05D
:109CF000C4F82BE0002005E09949095C974A1268F6
:109D00001154401C9E4909688842F5D300208D49B2
:109D10000968086000208549086017E000210020DC
:109D200000E0401C964A1268904207D28D4A0244D5
:109D30009278924B1B5C9A42F3D00121012902D107
:109D400000F09BF802E00020784908600020764986
:109D5000086001BD10B573480068002846D1042191
:109D60008848F6F769FA08218648F6F75BFA002476
:109D700000E0641C0A2C0FD2002083490860FA20FE
:109D8000FBF7ECFB042080490860FA20FBF7E6FBB8
:109D90007E4800680028ECD07C480068002801D18B
:109DA000002024E07A48FBF79DFB7A48F6F796FA04
:109DB0007948F6F793FA04217248F6F755FA082124
:109DC0007048F6F747FAE0211820FBF740FDFBF753
:109DD0003DFC01000122674807F0C8FD1820FBF791
:109DE00047FD01204F490860012000E0012010BD1F
:109DF00080B5F6F7DBFA4F49086000205249086049
:109E00000120494908605B4807F0E3FD594807F025
:109E1000DAFD00225021574807F0E2FD01205349A6
:109E2000086051480068401E4F4908604D4801785D
:109E3000504807F0E8FD03214E4807F0D5FD01BD6D
:109E40000022414B1A600222474B1A600200120A9C
:109E5000444B1A70434A50700220454A106000205B
:109E600003E00022454B1A54401C2028F9D34248F5
:109E70000160002042490860704780B501202E49EA
:109E800008603C4807F0A1FD00213A4807F0BBFDFF
:109E90000721384807F0A8FD41F21850FBF75EFB98
:109EA000002029490860334807F087FD00201E493B
:109EB000086000201B49086001BD80B500201E49D4
:109EC0000860FFF747FF002801D1012000E00020D3
:109ED000012802D1FFF7D1FF22E001201E490860CE
:109EE0000020194908601648007800280ED100208B
:109EF00003E000211A4A1154401C2028F9D31448C9
:109F0000016814480068FFF79BFF07E010480068ED
:109F1000801C15490860012014490860FFF768FF9C
:109F200001BD00007C2B0020842B0020882B00200A
:109F3000802B0020AC2B0020942B0020C42B002071
:109F4000642E0020C02B0020902B0020B02B00207E
:109F5000B82B0020B42B00208C2B0020BC2B002021
:109F60006C290020E0280020A02B0020982B002046
:109F7000A82B002000000240A42B00204C29002028
:109F80009C2B00200050004010500040205000400A
:109F9000002000F003080100030C010080B500F070
:109FA000F2F9DFF83C0A0078C00701D400F081F92B
:109FB000DFF82C0A0068C0F3400000280FD0DFF85B
:109FC000200A0068C0F38000002805D0002007F0B8
:109FD00072FE00F0D3FC02E0012007F06CFE5FF49B
:109FE00080200021F7F7D5FC20200021F7F7D1FCD5
:109FF000F6F7DCF90A38DFF8EC190860DFF8E00959
:10A00000006850F00100DFF8D819086001BD80B584
:10A01000DFF8CC090078C00769D5DFF8C40900680B
:10A02000C0F3400000281ED05FF480200021F7F725
:10A03000B0FCDFF8AC090068C0F38000002802D053
:10A0400000F000FA01E000F060FADFF89C09006817
:10A05000DFF898190968C943884216D05FF4800078
:10A06000F7F7A2FC11E05FF480200021F7F791FCE4
:10A0700020200021F7F78DFC5FF080700021F7F7BA
:10A0800088FC00200821F7F784FC00F0B4F90128CF
:10A0900001D1FFF783FFDFF848090068C0F34010E3
:10A0A000002824D0DFF8400900688DF80000DFF8B0
:10A0B00038090068000A8DF80100DFF830090068EF
:10A0C0008DF80200DFF824090068000A8DF803000B
:10A0D000042220216846FFF79BFC012807D1DFF806
:10A0E0000009006830F02000DFF8F418086001BDB6
:10A0F000002818D0102801D2012100E00021DFF84B
:10A10000E028127812F00602062A01D1012200E0AE
:10A110000022C9B2114206D0DFF8D41801EB80004A
:10A1200050F8080C00E000207047002818D01028D4
:10A1300001D2012100E00021DFF8A428127812F0FA
:10A140000602062A01D1012200E00022C9B2114212
:10A1500006D0DFF8A01801EBC00050E9040101E0CF
:10A16000002000217047002817D0102801D20121BB
:10A1700000E00021DFF86828127812F00602062AB3
:10A1800001D1012200E00022C9B2114205D0DFF85E
:10A190006818084410F8020C00E00020C0B27047B4
:10A1A000002818D0102801D2012100E00021DFF89A
:10A1B0003028127812F00602062A01D1012200E0AE
:10A1C0000022C9B2114206D0DFF8301801EB80003E
:10A1D00050F8080C00E000207047DFF80408006821
:10A1E00050F04000DFF8F81708607047DFF8F0071C
:10A1F000007810F00600062803D1DFF8EC0C0068A8
:10A2000000E000207047DFF8D807007810F0060063
:10A21000062803D1DFF8D40C006800E00020704766
:10A22000DFF8CC0C00687047DFF8C80C0068704796
:10A23000DFF8BC1C08607047DFF8B81C0860704786
:10A24000DFF89C07007810F0060006280CD1DFF834
:10A250009007006850F01000DFF8841708600020B5
:10A26000DFF89C17086007E0DFF87407006830F03B
:10A270001000DFF86C1708607047DFF864070068AB
:10A28000C0F38000002801D1002004E0DFF850076F
:10A290000068C0F300107047DFF84407007810F042
:10A2A0000600062803D1DFF8500C006800E000200B
:10A2B00070471CB50423202201A96846FFF761FB03
:10A2C0000028F7D0FFF7F7FB01280AD1F6F76EF860
:10A2D0000400F6F76BF8001B0228FAD3FFF7F4FA34
:10A2E000F0E79DF80000DFF800170860DFF8F806D7
:10A2F00000689DF8011050EA0120DFF8EC160860B4
:10A30000DFF8E406006880B2DFF8DC1608609DF82C
:10A310000200DFF8D8160860DFF8D00600689DF864
:10A32000031050EA0120DFF8C4160860DFF8BC060D
:10A33000006840F07F4050F47F00DFF8B0160860FE
:10A3400004216846F7F794FC012808D0DFF8980646
:10A350000068DFF898160968C943884212D00020C7
:10A36000DFF884160860DFF880060068C043DFF875
:10A370007C160860DFF86806006850F02000DFF8FF
:10A380006016086013BD80B55720F9F73DF9012824
:10A390000CD1DFF84C06006850F00400DFF84016DE
:10A3A00008600120DFF8541B08600DE0DFF830067C
:10A3B000006830F00400DFF8281608605720F9F72D
:10A3C00023F9DFF8381B08605620F9F71DF900283B
:10A3D00008D0DFF80C06006850F00200DFF8001625
:10A3E000086007E0DFF8F805006830F00200DFF8E9
:10A3F000F015086001BD70B5DFF8E4050068C0F332
:10A400004004DFF8DC050068C0F38005DFF8EC0AE3
:10A410000668FFF7B8FFDFF8C8050068C0F3400022
:10A4200084420BD1DFF8B8050068C0F38000854294
:10A4300004D1DFF8C80A0068864201D0012000E09C
:10A44000002070BD80B520200021F7F7A2FA00207F
:10A450000821F7F79EFADFF8F80B0078012804D0FE
:10A46000022805D100F0CEFA02E000F049FDFFE736
:10A47000DFF86C050068C0F38010002837D0DFF8E3
:10A48000D00B0078012832D00120DFF8C41B0870FF
:10A490000020DFF86C150860DFF84405006830F034
:10A4A0000800DFF83C1508600020DFF83C15086064
:10A4B0005FF0FF30DFF834150860DFF8240500682E
:10A4C00030F04000DFF8181508600020DFF8841B2A
:10A4D00008605FF080700021F7F783FA0020DFF852
:10A4E000101A08600020DFF80C1A08600CE0DFF892
:10A4F000F8040068DFF8601B0968884204D05FF444
:10A5000080200021F7F76DFA01BD1CB52020002145
:10A51000F7F767FA5720F9F777F80400684607F06D
:10A52000FAFBA04240F08480F5F740FFDFF82C1BD7
:10A5300008609DF8021009029DF801000143B1F581
:10A54000805F11D121004FF4805000F002F9DFF854
:10A550009004006830F08000DFF884140860142054
:10A56000DFF8F01A086071E0B1F5905F56D19DF800
:10A5700004009DF8071071F0FF01C943884201D122
:10A58000FBF7C3FC9DF80500FF2801D1F5F716FF86
:10A590009DF80500012804D100200821F7F721FAD1
:10A5A00003E000200821F7F7F4F9DFF8A80A0068B3
:10A5B000401CDFF8A01A0860DFF8980A0068142829
:10A5C00009DB0020DFF88C1A0860210041F204004A
:10A5D00000F0BFF83AE0DFF808040068C0F3C010EC
:10A5E00000280DD0210041F2050000F0B2F8DFF89C
:10A5F000F003006830F08000DFF8E413086025E025
:10A60000210041F2030000F0A4F8DFF8D403006851
:10A6100050F08000DFF8C813086017E041F2010035
:10A62000814213D1210041F2010000F092F80DE0C7
:10A63000F5F7BCFEDFF8241A0968401AB0F5FA6F86
:10A6400004D35FF480200021F7F7CBF913BD401C41
:10A65000002803D0012801D010280AD3102807D3DE
:10A66000DFF87C03006830F01000DFF87413086036
:10A670000220704730B583B00C0040218DF80010E7
:10A6800001008DF8011000B20100090A8DF80210D6
:10A6900000218DF8031000B2B0F5905F2FD120009B
:10A6A000F7F797FDDFF848180968084201D002253E
:10A6B00002E0FBF74EFA050028008DF80400C848B8
:10A6C0000068C0F30010002803D0FF208DF80500BB
:10A6D0000EE02000F7F77DFDDFF818180968084242
:10A6E00003D001208DF8050002E000208DF8050060
:10A6F00000208DF80600ED438DF8075022E000B2EF
:10A7000041F2010188420ED1FBF723FA01008DF8D6
:10A710000410000A8DF8050000208DF806000020C6
:10A720008DF807000EE04FF4A05080B200218DF8A4
:10A73000041000218DF805100100090A8DF806109B
:10A740008DF807002200D2B26946002007F000FB16
:10A7500037BD7CB50E0040218DF8001001008DF84A
:10A76000011000B20100090A8DF8021000218DF8D5
:10A77000031000B2B0F5905F19D1FBF7EAF90100C0
:10A7800008008DF8040096480068C0F30010002807
:10A7900003D0FF208DF8050002E000208DF80500B1
:10A7A00000208DF80600090A8DF80710A9E000B214
:10A7B00041F20101884212D15FF0FF30F7F70DF945
:10A7C0000100090E8DF804100100090C8DF8051028
:10A7D0000100090A8DF806108DF8070091E000B21B
:10A7E00041F20301884222D15FF0FF300F21F7F7D9
:10A7F00001F930F0200431F000055FF0FF30F7F789
:10A80000ECF8002803D054F0200455F00005200097
:10A81000000E8DF804002000000C8DF805002000CB
:10A8200080B2000A8DF806008DF8074069E000B29A
:10A8300041F20501884227D15FF0FF300F21F7F781
:10A84000D9F830F0200431F000055FF0FF30F7F761
:10A85000C4F8002803D054F0200455F0000520006F
:10A860002900080E00218DF8040020002900080CA2
:10A8700000218DF8050020002900080A00218DF82C
:10A8800006008DF807503CE000B241F20401884216
:10A8900010D1FEF762FA0100090E8DF804100100D4
:10A8A000090C8DF805100100090A8DF806108DF8C5
:10A8B000070026E01E20F8F7A7FE092802D14FF472
:10A8C000805011E01E20F8F79FFE042802D14FF4BB
:10A8D000A05009E01E20F8F797FE072802D141F2A8
:10A8E000024001E041F2034080B200218DF80410E3
:10A8F00000218DF805100100090A8DF806108DF869
:10A9000007003200D2B26946012007F021FA73BD78
:10A9100001794279120412EB0162817912EB012272
:10A92000C0791018B0F5A05F01D1042025E041F2F4
:10A930000141884201D106201FE041F202418842D4
:10A9400001D1072019E041F20341884201D10820DA
:10A9500013E0B0F5805F01D109200EE040F65111FF
:10A96000884207D040F65A11884203D040F65B1166
:10A97000884201D1052000E00020704700202049D6
:10A9800008601748006830F0080015490860022088
:10A99000DFF8BC160870002012E00021164A11549E
:10A9A0000021134A42F8201000220023114901EB34
:10A9B000C001C1E900230021104A42F82010401CC8
:10A9C0000E28EAD30020DFF8201508600020DFF809
:10A9D000201508600020DFF8881608607047000026
:10A9E000302C0020402C0020582C00205C2C002013
:10A9F00010280020D82500206C2A0020482800209C
:10AA0000542C002030B583B0DFF858060068C0F33E
:10AA1000C000002800F0F381684607F07CF90028A8
:10AA200000F0C681DFF840160968884240F0B38123
:10AA3000DFF834060068F7F7CCFBDFF8AC140968E0
:10AA40000843DFF8A41408609DF8021009029DF87D
:10AA50000100014341F20300814240F09D80DFF894
:10AA600008060468A41EDFF8040600EBC400D0E961
:10AA7000000130F0FF3031F00001DFF8F02502EB8B
:10AA8000C402C2E90001DFF8E40500EBC400D0E92C
:10AA900000239DF804000021090641EA1021000668
:10AAA00010431943DFF8C42502EBC402C2E90001D8
:10AAB000DFF8B80500EBC400D0E900239DF80500DD
:10AAC0000021090441EA1041000410431943DFF852
:10AAD0009C2502EBC402C2E90001DFF8900500EBFF
:10AAE000C400D0E900239DF806000021090241EAD4
:10AAF0001061000210431943DFF8702502EBC40215
:10AB0000C2E90001DFF8640500EBC400D0E90023CE
:10AB10009DF80700002110431943DFF8502502EB90
:10AB2000C402C2E90001DFF8440510F834008006D1
:10AB30001CD5DFF834050068F7F74BFBDFF8B813D6
:10AB400009680843DFF8B0130860DFF8200500EB60
:10AB5000C400D0E9000110F0200011F00001DFF87E
:10AB60000C2502EBC402C2E900011AE1DFF8F80487
:10AB70000068F7F72EFBDFF88013096831EA000060
:10AB8000DFF874130860DFF8E0040068FFF75FFD8A
:10AB9000DFF8D414086004E141F20500814268D175
:10ABA000DFF8C4040268921EDFF8C00400EBC200A4
:10ABB000D0E9000130F0000031F0FF31DFF8AC34B3
:10ABC00003EBC203C3E90001DFF8A00400EBC200FD
:10ABD000D0E900459DF80400002101060020204333
:10ABE0002943DFF8883403EBC203C3E90001DFF82F
:10ABF0007C0400EBC200D0E900459DF8050000216F
:10AC00000104002020432943DFF8603403EBC20332
:10AC1000C3E90001DFF8540400EBC200D0E90045AD
:10AC20009DF8060000210102002020432943DFF89F
:10AC30003C3403EBC203C3E90001DFF8300400EB4E
:10AC4000C200D0E900459DF8070000210100002066
:10AC500020432943DFF8143403EBC202C2E90001A8
:10AC6000DFF804040068FFF7F2FCDFF8FC1308606B
:10AC700097E041F20100814236D1DFF8EC03016830
:10AC8000891E9DF804000006DFF8E42342F8210045
:10AC9000DFF8DC0350F821009DF8052050EA02405F
:10ACA000DFF8CC2342F82100DFF8C40350F821007C
:10ACB0009DF8062050EA0220DFF8B42342F8210074
:10ACC000DFF8AC0350F821209DF807000243DFF8BD
:10ACD000A00340F82120DFF890030068FFF7B7FCDD
:10ACE000DFF8841308605CE041F20400814236D151
:10ACF000DFF874030168891E9DF804000006DFF880
:10AD0000742342F82100DFF86C0350F821009DF80D
:10AD1000052050EA0240DFF85C2342F82100DFF80A
:10AD2000540350F821009DF8062050EA0220DFF875
:10AD3000442342F82100DFF83C0350F821209DF81D
:10AD400007000243DFF82C0340F82120DFF8180346
:10AD50000068FFF77CFCDFF81013086021E0B1F514
:10AD6000805F11D1DFF800030468A41E6846FFF776
:10AD7000CFFDDFF804130855DFF8EC020068FFF799
:10AD800066FCB94908600CE0B7480068FFF75FFC53
:10AD9000B549086005E0B4480068FFF758FCB249BF
:10ADA0000860B048006830F00800AE49086099E0DB
:10ADB000F5F7FCFAA9490968401AB0F5FA6FC0F036
:10ADC0009180A9480068F7F704FA4749096831EA11
:10ADD0000000454908600020A749A34A12681144B1
:10ADE00001F8020CA0480068FFF731FC9E4908609A
:10ADF0009C48006830F008009A49086072E03B48BF
:10AE000000684FF6FC7108426CD0F5F7CFFA9B4909
:10AE10000968401A0A2865D3F5F7C8FA9749086007
:10AE2000002406E090480068FFF711FC8E49086096
:10AE3000641C0F2C56D28C480068F7F7CAF92B49CE
:10AE400009680842EED087480068C0F30010002867
:10AE500006D0854801684FF49050FFF70BFC37E0AF
:10AE6000854881490968084410F8020C002806D179
:10AE70007D4801684FF48050FFF7FCFB28E07A48DA
:10AE80000068F7F7A6F91C49096801421AD07C4806
:10AE9000006875490968884209D10020784908602E
:10AEA000714801684FF49050FFF7E4FB10E06E48E2
:10AEB000016841F20100FFF7DDFB6B480068704953
:10AEC000086005E0684801684FF49050FFF7D2FB36
:10AED0006448006850F0080062490860F5F766FAB7
:10AEE0005E49086037BD0000442C0020582C00202B
:10AEF0004C2C0020502C0020482C0020342C00200A
:10AF000000B583B057480068C0F3C000002877D070
:10AF1000684606F000FF002860D09DF8022012026B
:10AF20009DF801100A43B2F5805F42D14E4909688D
:10AF300088423ED19DF804009DF80510090411EBEC
:10AF400000619DF8060011EB00219DF8070051FA01
:10AF500080F040F65111884219D040F65A118842CB
:10AF600015D040F65B11884211D0B0F5A05F0ED02D
:10AF700041F2014188420AD0B0F5805F07D041F22A
:10AF80000241884203D041F2034188420DD1364844
:10AF90000068F7F71EF93B4909680843394908601A
:10AFA00038480068C04338490860002029490860D3
:10AFB0000DE028480068401C2649086025480068C4
:10AFC000032804DA28480068401E274908602548FD
:10AFD000006830F008002349086038E0F5F7E6F92A
:10AFE0001E490968401AB0F5FA7F30D3002019498C
:10AFF00008601C48006830F008001A49086026E024
:10B00000194800680F2815D217480068401C1649D7
:10B010000860154801684FF48050FFF72BFB11487A
:10B02000006850F008000F490860F5F7BFF90B49B8
:10B0300008600CE00B48006850F0200009490860E7
:10B04000FFF79CFC5FF080700021F6F7A2FC07BDC3
:10B050006A2E00203C2C0020442C0020382C00209C
:10B06000482C0020302C0020542C0020D825002013
:10B0700010280020482800206C2A0020402C0020A6
:10B08000602C0020582C00205C2C002080B5DFF8BC
:10B09000800A006840084000DFF8741A0860DFF892
:10B0A000700A006830F00800DFF8641A0860DFF802
:10B0B000600A006830F00400DFF8541A0860DFF816
:10B0C000500A006830F01000DFF8441A0860802150
:10B0D000DFF8400AF5F7B0F80020DFF83C1A086006
:10B0E000DFF82C0A006850F02000DFF8241A08600E
:10B0F0008021DFF8280AF5F79FF80020DFF8201AF2
:10B1000008604021DFF8140AF5F796F80020DFF810
:10B11000141A0860DFF8100AFAF7E4F941F605009E
:10B12000F5F7DCF841F60540F5F7D8F880215FF037
:10B130004020F5F7A3F840215FF04020F5F79EF896
:10B1400000228021DFF8E409FAF734F94FF47A623B
:10B150008021DFF8D809FAF743F98021DFF8CC091C
:10B16000FAF748F901220C21DFF8C009FAF770F963
:10B170004FF400728021DFF8B409FAF784F900F087
:10B1800017FC1021DFF8A809F5F72EF80321DFF8E6
:10B19000A409F6F763FC0321DFF89809F6F771FCC0
:10B1A000012300220321DFF88C09F6F772FC6C23DF
:10B1B00000220321DFF87C09F6F795FC0321DFF874
:10B1C0007409F6F759FC40212120FAF740FB0321CE
:10B1D000DFF86009F6F74CFC0321DFF85809F6F7B1
:10B1E00040FC2120FAF744FB0321DFF84809F6F779
:10B1F000DAFCDFF84409FAF775F9DFF83C09FAF7E9
:10B200008BF93221DFF83409F5F729FF0122FF21FC
:10B21000DFF82809F5F760FFDFF82429FF21DFF8C0
:10B220001C09F5F765FFA0215620FAF710FB012154
:10B23000DFF80809F5F778FF0121DFF80009F5F7D5
:10B2400078FF5620FAF714FBFF21DFF8F008F5F736
:10B25000F7FE0020DFF8EC1808700020DFF8E8188F
:10B260000870F5F7A3F8DFF8E4180860F5F79EF822
:10B27000DFF8DC180860DFF89808006850F001007B
:10B28000DFF88C18086001BD80B5DFF8840800780D
:10B29000C00757D5DFF8AC080078002812D0022884
:10B2A00007D003D304280AD006D30EE000F085F9B6
:10B2B00010E000F0F5F80DE000F0F4F90AE000F01D
:10B2C00035FA07E000F0CAF804E00820F6F778FB4A
:10B2D00000F06EFB4D20F8F797F910F00F0F0ED12C
:10B2E0005FF40000F6F73FFB4FF480500021F6F7C3
:10B2F00050FB4FF400600021F6F74BFB22E0DFF833
:10B300001008007810F00C0F05D04FF400600021F9
:10B31000F6F767FB04E04FF400600021F6F739FB15
:10B32000DFF8EC070068C0F30010002805D04FF4E8
:10B3300080500021F6F755FB04E04FF480500021C7
:10B34000F6F727FB01BDDFF800180870704780B5DD
:10B35000DFF8F407007801281FD1DFF8E80700784C
:10B36000012809D1DFF8A807007810F01C0F01D0E0
:10B37000012046E0002044E0DFF8C80700780028FC
:10B3800009D14D20F8F740F910F00F0F01D100203E
:10B3900037E0022035E0022033E0DFF8AC07007828
:10B3A00002281FD1DFF89C070078022809D1DFF8B6
:10B3B0006007007810F01C0F01D0012021E0002070
:10B3C0001FE0DFF880070078002809D14D20F8F74A
:10B3D0001BF910F00F0F01D1002012E0022010E045
:10B3E00002200EE0DFF860070078032801D1022078
:10B3F00007E0DFF850070078002801D1002000E0C6
:10B400000220C0B202BD80B50321DFF82807F6F79D
:10B410002FFBDFF840270321DFF81807F6F7B0FB12
:10B42000DFF83007006840F6A171884209D3DFF8E1
:10B43000E006006850F00400DFF8D416086000F061
:10B44000B7FA01BD80B50121DFF8F006F5F771FE0E
:10B450000321DFF8E006F6F7A6FB01BD80B500F09A
:10B46000A7FA4D20F8F7D0F810F00F0F17D0DFF83B
:10B47000D8060078012804D0DFF8CC06007803282D
:10B4800004D10220DFF8BC16087008E0DFF8B80627
:10B490000078022803D10120DFF8A816087001BD4A
:10B4A00080B500F0BAFA012840F08680DFF89806EF
:10B4B0000078012804D0DFF890060078032821D115
:10B4C0000120DFF884160870DFF84406006830F0C9
:10B4D0000800DFF83C160860DFF83406006830F03A
:10B4E0001000DFF82C16086000F062FA4D20F8F723
:10B4F0008BF8000601D400F0EDF90320DFF84416C4
:10B50000087059E0DFF840060078002806D100F006
:10B510004FFA0020DFF82C1608704DE000F05CF9BF
:10B520004D20F8F771F8000644D54D20F8F76CF877
:10B5300010F00F0F3ED04FF480400021F6F75AFA7A
:10B5400000220023994201D190420AD05FF080404E
:10B550000021F6F74FFA0022002399422AD19042A7
:10B5600028D1DFF8AC050068C0F3C000002821D165
:10B57000DFF8E005006840F26D2188420AD300F050
:10B5800017FADFF88C05006850F00800DFF8801526
:10B59000086011E0DFF878050068C0F3400000287B
:10B5A00002D100F0CEF907E0F4F700FFDFF8A015B4
:10B5B000086001E000F0FCF901BD80B500F02DFA53
:10B5C00001286ED14D20F8F71FF810F00F0F03D1AE
:10B5D0000020DFF874150870DFF86C050078022889
:10B5E00038D1DFF82C05006830F00800DFF82015AE
:10B5F0000860DFF81C05006830F01000DFF8101557
:10B60000086000F0D5F94FF480400021F6F7F2F918
:10B6100000220023994201D1904214D05FF0804073
:10B620000021F6F7E7F900220023994201D1904268
:10B6300009D04D20F7F7E8FF000604D40220DFF818
:10B64000041508702DE00420DFF8F814087000F0ED
:10B6500078F926E0DFF8F0040078032811D1012002
:10B66000DFF8E414087000F0A3F94D20F7F7CCFFE1
:10B67000000616D400F02EF90320DFF8C814087075
:10B680000FE0DFF8C4040078002806D10020DFF8BE
:10B69000B414087000F08CF903E000F0DDF800F05D
:10B6A00087F901BD80B5DFF868040068C0F3401079
:10B6B00000280AD04FF480400021F6F79BF90022C1
:10B6C0000023994201D1904211D0DFF84404006870
:10B6D000C0F3401000281FD14FF480400021F6F73E
:10B6E00089F900220023994201D1904214D000F040
:10B6F0005FF9F4F75BFEDFF8541408604D20F7F7AC
:10B7000083FF10F00F0F03D1012000F0F9F90CE0D6
:10B71000022000F0F5F908E000F047F8012804D114
:10B7200000F046F9012000F0EBF901BD80B5DFF82B
:10B73000E0030068C0F3401000280AD04FF48040B6
:10B740000021F6F757F900220023994201D19042D7
:10B7500011D0DFF8BC030068C0F34010002815D1F9
:10B760004FF480400021F6F745F90022002399426A
:10B7700001D190420AD000F01BF9F4F717FEDFF870
:10B78000CC130860012000F0BBF90DE000F00DF8CB
:10B79000012809D14D20F7F737FF000601D400F04A
:10B7A00007F9022000F0ACF901BD10B54D20F7F704
:10B7B0002BFF000602D54FF47A7401E04FF41674A3
:10B7C000F4F7F4FDDFF888130968401AA04201D3AA
:10B7D000012000E0002010BD80B52020F7F7DCFE3E
:10B7E00000280FD04D20F7F70FFF10F00F0F09D0F2
:10B7F000F9F76EF8002805D04FF4804004F04DF9B9
:10B80000002801D0012008E04FF4004004F045F981
:10B81000002801D1012000E0002001280BD1F4F71D
:10B82000C5FDDFF834130860B948006830F0100037
:10B83000B74908600FE0F4F7B9FDDFF81C13096899
:10B84000401A40F2E931884205D3B148006850F00F
:10B850001000AF49086001BD80B52020F7F79CFEBD
:10B8600000280FD04D20F7F7CFFE10F00F0F09D0B2
:10B87000F9F72EF8002805D04FF4804004F00DF9B8
:10B88000002801D0012008E04FF4004004F005F941
:10B89000002801D1002000E0012001280AD1F4F79E
:10B8A00085FDAD4908609A48006830F0100098495D
:10B8B00008600EE0F4F77AFDA7490968401A40F2E3
:10B8C000E931884205D39248006850F01000904951
:10B8D000086001BD80B500209249086000209049B1
:10B8E0000860002208219148F9F7A9FD4FF4804033
:10B8F0000021F6F77FF800220023994201D19042FF
:10B9000006D04FF47A6282218848F9F776FD05E087
:10B910004FF4486282218548F9F76FFD0122042126
:10B920008248F9F78CFD40207E490860F4F73EFD1F
:10B93000874908607648006850F002007449086042
:10B9400001BD80B500207749086000207449086077
:10B95000002204217548F9F772FD4FF48040002160
:10B96000F6F748F800220023994201D1904206D010
:10B970004FF47A6283216D48F9F73FFD05E04FF4FB
:10B98000486283216948F9F738FD01220821674898
:10B99000F9F755FD802062490860F4F707FD6C490E
:10B9A00008605B48006850F002005949086001BD1A
:10B9B00080B500205B490860002059490860544860
:10B9C0000068C0F38000002805D14D20F7F71CFE69
:10B9D00010F00F0F05D100220C215448F9F72FFD6C
:10B9E00010E04FF47A6282215048F9F706FD4FF4D7
:10B9F0007A6283214D48F9F700FD01220C214B4862
:10BA0000F9F71DFD4248006830F002004049086027
:10BA1000F4F7CCFC4E49086001BD80B53C48006895
:10BA2000C0F3401000280AD04FF480400021F5F701
:10BA3000E1FF00220023994201D1904210D0344806
:10BA40000068C0F34010002854D14FF4804000211A
:10BA5000F5F7D0FF00220023994201D1904249D04E
:10BA60002B480068C0F38000002801D0012046E088
:10BA700027480068C0F34000002812D14FF48040EE
:10BA80000021F5F7B7FF00220023994201D190422F
:10BA900003D000202049086007E080201E4908608C
:10BAA00003E0F4F783FC29490860FFF781FFF4F70E
:10BAB0007DFC26490968401A192819D34FF48040A3
:10BAC0000021F5F797FF00220023994201D190420F
:10BAD00006D00F48006850F020000D49086005E0CE
:10BAE0000B48006830F0200009490860012006E09A
:10BAF000002004E0F4F75AFC14490860012002BD5C
:10BB000080B510490870F4F751FC1349086001BD75
:10BB1000642C0020004006400042064000C0054062
:10BB200000C2054000C10540014000F00090024005
:10BB30000070004000800340040400F00040034017
:10BB4000400D03006B2E00206C2E0020742C002072
:10BB5000682C0020702C00206C2C002080B5B3488D
:10BB6000006840084000B1490860B048006850F0E3
:10BB70000400AE490860F4F719FCAD4908604FF4C1
:10BB80008040F5F72AFF00280CD00920A74948700B
:10BB9000802000F0ABFEA548006830F00400A34907
:10BBA000086005E00020A1494870072000F09EFED3
:10BBB0004FF480600021F5F7ECFE4FF40070002197
:10BBC000F5F7E7FE00209949C8610020974908620F
:10BBD0009648006850F001009449086001BD80B5A6
:10BBE00092480078C00740F1FC8000F023F98F49AB
:10BBF00088708E488078022803D18C48C07802284B
:10BC00000FD18A488078032803D18848C078032858
:10BC100007D186488078012810D18448C07801284F
:10BC20000CD05FF0FF30F5F79EFE00207F490862E0
:10BC300000207E49C86100207C4988617B4880786B
:10BC4000022803D0F4F7B2FB78494860774880783F
:10BC500001280DD180200021F5F7C3FE40200021EE
:10BC6000F5F797FE4FF480700021F5F792FE29E07A
:10BC70006E48807802280DD180200021F5F789FEDA
:10BC800040200021F5F7ADFE4FF480700021F5F75C
:10BC900080FE17E080200021F5F77BFE4020002188
:10BCA000F5F777FE1420F9F75FFF002805D14FF470
:10BCB00080700021F5F76DFE04E04FF480700021E4
:10BCC000F5F78FFEF0F703FC002805D15FF4803014
:10BCD0000021F5F786FE04E05FF480300021F5F7DF
:10BCE00058FEF0F7F8FB002805D14FF40040002182
:10BCF000F5F777FE04E04FF400400021F5F749FE28
:10BD00004A480068C0F38000002813D000230022B6
:10BD100000210020F0F781FBF4F748FB4449096853
:10BD2000401AC8285DD34148006830F004003F49FC
:10BD3000086056E03D48407809284EDAF4F758FB91
:10BD4000012807D139484078012803D0374806F048
:10BD5000A9FA42E0F4F78AFF012803D1334806F03C
:10BD6000DBFA3AE05FF400000021F5F712FE2F48FD
:10BD70004078032803D12D4806F056FB2DE02B48D0
:10BD80004078022803D1294806F0D0FD25E0274855
:10BD90004078082803D1254807F0E0F81DE0234843
:10BDA0004078072803D1214807F03CFB15E01F48E5
:10BDB0004078002803D11D4807F057FD0DE01B48CF
:10BDC0004078012803D1194806F09AF805E00220CE
:10BDD000F5F7EAFD154806F065FA1448807813492E
:10BDE000C87001BD1148407870471048807870478E
:10BDF0000E480068C0F34000704780B5FFF7F5FFBC
:10BE0000012803D1094807F07FFD0DE05FF0FF3006
:10BE1000F5F7E3FD002803D0044806F043FA03E0F9
:10BE20006421024807F072F801BD0000802800205C
:10BE3000882C002080B50A20F9F796FE012801D150
:10BE4000012015E01120F9F78FFE012801D1002013
:10BE50000EE01220F9F788FE012801D1022007E048
:10BE60001320F9F781FE012801D1032000E0002012
:10BE7000C0B202BD80B50020DFF858160870082156
:10BE8000DFF85406F4F7D8F90820DFF850160860F8
:10BE9000DFF84C06006850F00100DFF84416086037
:10BEA000DFF83C06006830F00200DFF83416086066
:10BEB0000020DFF83016087001BD80B5DFF82006DD
:10BEC0000078C00740F1B680DFF808060078002847
:10BED00002D100F021F91FE0DFF8F8050078012811
:10BEE00002D100F041F917E0DFF8E80500780228F8
:10BEF00002D100F01AFA0FE00020DFF8D815087020
:10BF00000820DFF8D8150860DFF8D405006850F085
:10BF10000200DFF8CC1508602020F7F775FB30F041
:10BF20008000482805D04E2803D04FF48060F5F7F4
:10BF30001AFD2620F7F768FB30F08000482805D06E
:10BF40004E2803D04FF40060F5F70DFD2820F7F7D9
:10BF50005BFB30F0800048286CD02820F7F754FBBA
:10BF600030F080004E2865D02A20F7F74DFB30F0E6
:10BF7000800048285ED02A20F7F746FB30F080008A
:10BF80004E2857D02C20F7F73FFB30F08000482890
:10BF900050D02C20F7F738FB30F080004E2849D0E5
:10BFA0002E20F7F731FB30F08000482842D02E20B9
:10BFB000F7F72AFB30F080004E283BD03420F7F70B
:10BFC00023FB30F08000482834D03420F7F71CFBE6
:10BFD00030F080004E282DD03620F7F715FB30F0DA
:10BFE0008000482826D03620F7F70EFB30F080007E
:10BFF0004E281FD03020F7F707FB30F0800048288C
:10C0000018D03020F7F700FB30F080004E2811D018
:10C010003220F7F7F9FA30F0800048280AD03220B1
:10C02000F7F7F2FA30F080004E2803D05FF40020DA
:10C03000F5F799FC01BDDFF8A8040078C00701D42A
:10C0400000200CE0DFF88C040078002806D1DFF82F
:10C0500094040078012801D0002000E001207047FE
:10C06000DFF87C040078C00701D4002007E0DFF887
:10C0700064040078012801D1012000E0002070470D
:10C0800010B504005FF080600021F5F782FC01200C
:10C09000DFF850140870E4B2DFF84C04046010BDFF
:10C0A0000220DFF8401408707047DFF83C04006895
:10C0B000012809D14E20DFF8341408605FF0FF300A
:10C0C000DFF82C14086026E0DFF81C040068002864
:10C0D00009D14820DFF8181408605FF0FF30DFF85E
:10C0E0000C14086017E0DFF800040068022808D18B
:10C0F0004E20DFF8F81308604820DFF8F4130860DA
:10C1000009E05FF0FF30DFF8E41308605FF0FF3014
:10C11000DFF8DC130860704780B50820DFF8BC1337
:10C120000860DFF8C003007801281CD15FF00070C0
:10C130000021F5F75FFC00220023994211D19042C3
:10C140000FD10020DFF89C1308700120DFF8841362
:10C150000870F4F72BF9DFF89C130860FFF7A5FFD0
:10C1600001E0F8F750FB01BD10B50020DFF86C13BB
:10C17000086000242021012000F067F9012801D186
:10C1800054F001042221022000F05FF9012801D1BE
:10C1900054F002042421042000F057F9012801D1B1
:10C1A00054F004042621082000F04FF9012801D1A1
:10C1B00054F008042821102000F047F9012801D18B
:10C1C00054F010042A21202000F03FF9012801D169
:10C1D00054F020042C21402000F037F9012801D12F
:10C1E00054F040042E21802000F02FF9012801D1C5
:10C1F00054F0800430214FF4807000F026F90128BB
:10C2000001D154F4807432214FF4007000F01DF914
:10C21000012801D154F4007434214FF4805000F00F
:10C2200014F9012801D154F4806436214FF40050F0
:10C2300000F00BF9012801D154F40064A9480078FA
:10C24000012809D1F4F7B2F8AA490860FFF72DFFD9
:10C250000020A449087067E040F6FF70844203D0D4
:10C26000A048007802280FD102209A490870F4F7FC
:10C270009DF8A04908600820984908605FF0806038
:10C280000021F5F786FB4FE0F4F790F8994909682B
:10C29000401A40F6A171884246D302208D490870A9
:10C2A000F4F784F8934908608020F7F775F90028BF
:10C2B00004D04FF48060F5F783FB35E0E0070ED43F
:10C2C0008020F7F769F9002804D14FF48060F5F772
:10C2D00077FB04E05FF080600021F5F782FB200728
:10C2E0000ED48020F7F758F9002804D14FF40060ED
:10C2F000F5F766FB04E05FF080600021F5F771FB65
:10C3000014F47F64B4F57F6F0ED08020F7F744F902
:10C31000002804D15FF40020F5F752FB04E05FF041
:10C3200080600021F5F75DFB10BD10B508206B495A
:10C33000086000242021012000F0A9F8012801D183
:10C3400054F001042221022000F0A1F8012801D1BB
:10C3500054F002042421042000F099F8012801D1AE
:10C3600054F004042621082000F091F8012801D19E
:10C3700054F008042821102000F089F8012801D188
:10C3800054F010042A21202000F081F8012801D166
:10C3900054F020042C21402000F079F8012801D12C
:10C3A00054F040042E21802000F071F8012801D1C2
:10C3B00054F0800430214FF4807000F068F80128B8
:10C3C00001D154F4807432214FF4007000F05FF812
:10C3D000012801D154F4007434214FF4805000F04E
:10C3E00056F8012801D154F4806436214FF40050EE
:10C3F00000F04DF8012801D154F400643948007868
:10C40000022803D10020374908700FE03548007832
:10C4100001280BD100203349087001202D490870F4
:10C42000F3F7C4FF33490860FFF73FFEF3F7BEFFA1
:10C4300030490968401AC92803D240F6FF70844287
:10C4400002D100202349087010BD38B504000D004A
:10C450002800C0B2F7F7D8F830F080002349096807
:10C46000884209D02800C0B2F7F7CEF830F080003B
:10C470001F490968884208D1200003F00EFB0028FC
:10C4800001D0012002E0002000E0012032BD38B5DB
:10C4900004000D002800C0B2F7F7B6F830F08000B5
:10C4A00012490968884209D02800C0B2F7F7ACF8F1
:10C4B00030F080000E490968884208D1200003F05E
:10C4C000ECFA002801D0002002E0012000E0012069
:10C4D00032BD0000662E00200030064020300640AD
:10C4E000D82B0020652E0020E02B0020E42B00201C
:10C4F000E82B0020DC2B002080B5F3F757FFDFF896
:10C50000841B0860DFF8280C006830F00200DFF8B8
:10C51000201C08600020DFF8701B08600020DFF896
:10C520006C1B0870DFF8080C006850F00100DFF8A1
:10C53000001C086001BD80B5DFF8F40B0078C0076F
:10C5400040F1CB815FF0E04003F0A7FADFF8E41B95
:10C5500008605FF0E04003F0A5FADFF8DC1B08603C
:10C560000121032004F001FADFF8C80B006810F085
:10C57000E04F04D0F3F71AFFDFF8C01B0860F3F7B1
:10C5800015FFDFF8B81B0968401ADFF8B41B8842B2
:10C5900003D36420DFF8F01A0860DFF8EC0A0068C3
:10C5A000642802D100F0FEF997E1DFF8DC0A0068A8
:10C5B000012802D100F05BFA8FE1DFF8CC0A0068B5
:10C5C000652802D100F0B5FB87E1DFF8BC0A0068FE
:10C5D000662802D100F09FFC7FE1DFF8AC0A00681A
:10C5E000672802D100F0A2FA77E1DFF89C0A006820
:10C5F000682802D100F0F6FA6FE1DFF88C0A0068D3
:10C60000692802D100F040FB67E1DFF87C0A00688E
:10C610006B2802D100F0F4FC5FE1DFF86C0A0068DF
:10C620006C2802D100F034FD57E1DFF85C0A0068A5
:10C630006D2802D100F086FD4FE1DFF84C0A00685A
:10C640006E2802D100F037FE47E1DFF83C0A0068AF
:10C650006F2802D100F074FE3FE1DFF82C0A006879
:10C66000702802D100F0B1FE37E1DFF81C0A006843
:10C67000712802D100F0EEFE2FE1DFF80C0A00680D
:10C68000722802D100F0EEFF27E1DFF8FC09006814
:10C69000CF2803D1092001F049F91EE1DFF8E809AC
:10C6A0000068D02803D1092001F0A0FB15E1DFF8D4
:10C6B000D8090068D12803D10A2001F037F90CE12C
:10C6C000DFF8C4090068D22803D10A2001F08EFBEC
:10C6D00003E1DFF8B4090068C92803D1052001F09F
:10C6E00025F9FAE0DFF8A0090068CA2803D105207F
:10C6F00001F07CFBF1E0DFF890090068CB2803D162
:10C70000082001F013F9E8E0DFF87C090068CC2884
:10C7100003D1082001F06AFBDFE0DFF86C09006854
:10C72000CD2802D101F000F8D7E0DFF85C090068FD
:10C73000CE2802D101F0A8F8CFE0DFF84C0900685C
:10C740006A2802D101F0F2FBC7E0DFF83C0900687B
:10C750007D2802D101F01EFDBFE0DFF82C09006842
:10C76000D42802D101F0E8FDB7E0DFF81C09006829
:10C77000D52802D101F03EFEAFE0DFF80C090068D9
:10C78000D62802D101F0DAFEA7E0DFF8FC08006845
:10C79000D82802D101F032FF9FE0DFF8EC080068F2
:10C7A000D92803D1012001F0D7FF96E0DFF8D8089F
:10C7B0000068DA2803D1022001F0CEFF8DE0DFF817
:10C7C000C8080068732802D100F084FE85E0DFF815
:10C7D000B8080068742802D100F0E2FE7DE0DFF8BE
:10C7E000A8080068752803D1012001F09FF874E0C3
:10C7F000DFF894080068772803D1022001F096F84A
:10C800006BE0DFF884080068792803D1032001F089
:10C810008DF862E0DFF8700800687B2803D10420FF
:10C8200001F084F859E0DFF860080068762803D149
:10C83000012001F0DBFA50E0DFF84C0800687828AE
:10C8400003D1022001F0D2FA47E0DFF83C0800688B
:10C850007A2803D1032001F0C9FA3EE0DFF8280866
:10C8600000687C2803D1042001F0C0FA35E0DFF82D
:10C8700018080068D32802D101F0FEFC2DE0DFF893
:10C8800008080068D72802D100F09CFF25E0DFF8F7
:10C89000F8070068DB2802D101F0C0FB1DE0DFF8DB
:10C8A000E8070068B0F5967F02D102F01CF814E0AA
:10C8B000DFF8D4070068002802D100F01FF80CE070
:10C8C000DFF8C4070068B0F5C87F02D102F05EF857
:10C8D00003E06420DFF8B017086001BDDFF8AC07A3
:10C8E00000787047DFF8AC0C00687047DFF8A81CD0
:10C8F00008707047DFF8A00C0078704780B5002002
:10C90000DFF888170870DFF828080068C0F34000D7
:10C91000002804D1F3F74AFDDFF8801C0860DFF837
:10C920001408006810F0E040B0F1E04F17D1DFF8D4
:10C930000008006850F00200DFF8F4170860F3F711
:10C9400035FDDFF8581C0968401A41F288318842E9
:10C950000DD34FF4C870DFF83017086007E0DFF838
:10C96000D007006830F00200DFF8C4170860DFF875
:10C97000C0070068C0F3400000280DD1F3F716FD92
:10C98000DFF800170968401A41F28831884203D362
:10C990006420DFF8F416086002F098FEDFF8F41B5C
:10C9A000086001BD80B50220DFF8E0160870DFF8EE
:10C9B00088070068C0000AD54020F6F7EDFD002882
:10C9C00054D102F015F8DFF8C01608604EE0DFF829
:10C9D0006407006810F0C040B0F1C04F13D10120CF
:10C9E000DFF8A4160860F3F7E1FCB0F51670DFF885
:10C9F00094160860DFF83807006850F00400DFF88C
:10CA00003017086032E04FF40070F4F7E6FF0028BA
:10CA100027D04FF480400021F4F7ECFF00220023E0
:10CA2000994201D190421CD0F3F7C0FCDFF85416B4
:10CA30000968401AB0F5FA7F18D3F3F7B7FCDFF8AE
:10CA400044160860DFF84C0B0068802804D10020F1
:10CA5000DFF8401B086009E08020DFF8381B086021
:10CA600004E002F0A7FDDFF82C1B086001BD80B5D3
:10CA70000220DFF818160870F3F798FCDFF80416A8
:10CA80000968401AB0F5167F43D3F3F78FFCDFF83F
:10CA9000F4150860DFF898060068C0F380000028ED
:10CAA0001ED1DFF88C06006850F00400DFF8801615
:10CAB00008605FF0FF30F4F790FF002807D15FF0C7
:10CAC000FF300F21F4F796FF02F0C5FD01E002F000
:10CAD000A1FD012102F0BFF8DFF8B81A086018E0E4
:10CAE000DFF84C06006830F00400DFF844160860F8
:10CAF0005FF0FF30F4F771FF002805D047F65010C3
:10CB0000DFF8901A086004E047F23870DFF8841A02
:10CB10000860DFF82006006810F0C040B0F1C04F98
:10CB200003D06420DFF86015086001BD80B51E20C9
:10CB3000F6F76AFD072805D001F05AFFDFF848151F
:10CB400008604EE0DFF8F0050068C00005D501F090
:10CB50004FFFDFF83415086043E0DFF8D8050068C0
:10CB6000C0000AD543F65400DFF8281A086001F027
:10CB70006DFFDFF81415086033E00520DFF80C15B1
:10CB800008700220F6F708FDDFF8341C0860DFF8B3
:10CB9000A805006810F0C04F0DD0DFF8240C006825
:10CBA000002804D00020DFF8181C086003E00120F2
:10CBB000DFF80C1C0860DFF8080C0068002808D0BB
:10CBC0000620DFF8D019086000210220F6F7E9FC02
:10CBD00007E05B20DFF8BC19086000210220F6F7AF
:10CBE000F9FC01BD00B583B01E20F6F70DFD072846
:10CBF00005D001F0FDFEDFF89014086043E0DFF897
:10CC000038050068C00005D501F0F2FEDFF87814A1
:10CC1000086038E0DFF81C050068C0000AD543F65C
:10CC20007800DFF87019086001F010FFDFF8581481
:10CC3000086028E00620DFF8541408705E20F6F73C
:10CC4000E3FCDFF87C1B08600120019000200090CD
:10CC5000012302220021DFF8680B006801F021FFA8
:10CC6000DFF85C1B08600121DFF8540B006801F05D
:10CC7000F2FFDFF8201908600022DFF8440B01689A
:10CC80005E20F6F75AFD07BD80B5DFF8AC040068FA
:10CC9000C00005D501F0ACFEDFF8EC13086047E0FA
:10CCA000DFF890040068C0000AD545F23700DFF8CD
:10CCB000E418086001F0CAFEDFF8CC13086037E022
:10CCC0000720DFF8C81308705FF00040F6F764FC37
:10CCD000DFF8EC1A0860DFF86004006810F0C04F5D
:10CCE0000DD0DFF8DC0A0068002804D00020DFF84F
:10CCF000D01A086003E00120DFF8C41A0860DFF8EA
:10CD0000C00A006800280AD044F20600DFF8841840
:10CD1000086000215FF00040F6F743FC08E00620C1
:10CD2000DFF87018086000215FF00040F6F752FC51
:10CD300001BD00B583B0DFF800040068C0003ED537
:10CD4000DFF87C0A0068DFF83C1C0968884223D0C1
:10CD5000DFF86C0A0068012801D1092115E0DFF82D
:10CD6000600A0068022801D104210EE0DFF8500AB1
:10CD70000068032801D1082107E0DFF8440A0068B1
:10CD8000042801D1072100E0002100221E20F6F72F
:10CD9000D4FC0020F6F7AAFBDFF8240A0068642818
:10CDA00008D14FF49670B84908600020DFF8101AD7
:10CDB0000860AFE001F01CFEB3490860AAE0DFF8AC
:10CDC00074030068C00040D543F67110DFF8C41743
:10CDD00008601E20F6F718FC092804D10120DFF8AE
:10CDE000E019086021E01E20F6F70EFC042804D1AB
:10CDF0000220DFF8CC19086017E01E20F6F704FCCB
:10CE0000082804D10320DFF8B81908600DE01E20BF
:10CE1000F6F7FAFB072804D10420DFF8A41908600C
:10CE200003E06420DFF898190860DFF894090068CF
:10CE3000DFF8501B0860DFF888090068642869D0B3
:10CE400001F004FE9049086064E004208F490870F6
:10CE5000DFF86C090068642819D145F25C40DFF8FE
:10CE600034170860B4480068800003D5B1480068F2
:10CE7000400007D5AF48006880004BD4AE4800683A
:10CE8000400047D50120DFF83819086042E0012052
:10CE9000019000200090012304220121DFF82009E5
:10CEA000006801F0FEFDDFF818190860DFF81009CE
:10CEB0000068012805D1002209211E20F6F73DFC5B
:10CEC0001FE0DFF8FC080068022805D100220421D9
:10CED0001E20F6F732FC14E0DFF8E40800680328AF
:10CEE00005D1002208211E20F6F727FC09E0DFF813
:10CEF000D0080068042804D1002207211E20F6F77C
:10CF00001CFC0121DFF8B808006801F0A4FEDFF87E
:10CF10008416086007BD80B587480068C0000CD53E
:10CF2000DFF89C080068012802D10020F6F7DEFA3D
:10CF300001F05EFD5449086061E07E480068C00071
:10CF40001DD545F67160DFF84C1608605FF00040B3
:10CF50000021F4F74FFD00220023994201D19042B5
:10CF600004D00020DFF85818086003E00120DFF843
:10CF70005018086001F06AFD434908603FE0032053
:10CF8000424908705FF000400021F4F733FD0022B1
:10CF90000023994206D1904204D10120DFF82018E5
:10CFA00008601DE064480068800003D5614800689F
:10CFB000400007D55F480068800011D45E480068D3
:10CFC00040000DD5DFF8F8070068002804D10120E3
:10CFD000DFF8EC17086003E00020DFF8E4170860D2
:10CFE000DFF8DC070068002805D145F25C40DFF877
:10CFF000A415086003E06E20DFF89815086001BDF5
:10D0000000B583B04C480068C00004D501F0F0FCC6
:10D010001D49086035E047480068C00009D547F25F
:10D020007730DFF87015086001F010FD16490860D0
:10D0300027E00920154908703820F6F7E5FADFF8EF
:10D0400080170860002001900120009001231E221B
:10D050000021DFF86C07006801F023FDDFF860179E
:10D0600008600121DFF85807006801F0F4FDDFF8DF
:10D07000241508600022DFF8480701683820F6F719
:10D080005CFB07BD502B0020402B0020622E0020AF
:10D0900080B529480068C00005D501F0A9FCDFF87B
:10D0A000D819086042E023480068C0000AD547F656
:10D0B0006D10DFF8E014086001F0C8FCDFF8B81963
:10D0C000086033E00A20DFF85C1808701020F6F7DB
:10D0D00063FADFF8EC1608601748006810F0C04FDC
:10D0E0000DD0DFF8DC060068002804D00020DFF84F
:10D0F000D016086003E00120DFF8C4160860DFF8EE
:10D10000C0060068002808D06E20DFF88814086088
:10D1100000211020F6F745FA08E045F25C40DFF800
:10D120007414086000211020F6F754FA01BD0000C5
:10D130003C2B0020542B0020582B00204C2B00208F
:10D14000C027090030B583B0DFF8DC070068C000F5
:10D1500005D501F04DFCDFF820190860AAE0DFF8E2
:10D16000880C0068C0000AD547F25430DFF8241458
:10D17000086001F06BFCDFF8001908609AE00B20F2
:10D18000DFF8A01708703920F6F73EFADFF83016FE
:10D190000860DFF82C0600683C2835D2DFF820064E
:10D1A0000078C0071DD400200190012000900223C8
:10D1B0003C220021DFF80806006801F072FCDFF86D
:10D1C00000160860DFF8F80500683C284BD2012102
:10D1D000DFF8EC05006801F03EFDDFF8B8130860E9
:10D1E00061E0DFF84407006810F0C04F06D0392036
:10D1F000F5F77CFADFF8C8150860E3E747F6731027
:10D20000DFF89013086055E00A20DFF8B4150968CC
:10D21000DFF8AC251268B2FBF0F200FB1210002818
:10D220000FD100200190012000900A23F02232212A
:10D23000DFF88C05006801F034FCDFF88415086025
:10D24000C0E7DFF8E406006810F0C04F06D03920D0
:10D25000F5F74CFADFF868150860B3E747F6731086
:10D26000CC49086026E0DFF8580500683C21B0FB97
:10D27000F1F03C21DFF848251268DFF844351B68DF
:10D28000B3FBF1F301FB13210A22B1FBF2F401F02D
:10D29000BBFC0500200001F0B7FC50EA052050F06F
:10D2A0008000BC4908600022DFF8140501683920BD
:10D2B000F6F743FA37BD00B583B0DFF86C060068B7
:10D2C000C00005D501F094FBDFF8AC17086036E02C
:10D2D000DFF8140B0068C00009D543F66D10AD49A6
:10D2E000086001F0B3FBDFF89017086027E00C201E
:10D2F000DFF8301608701820F6F786F9DFF8C0144A
:10D300000860012001900020009001230A220121E1
:10D31000DFF8AC04006801F0C4FBDFF8A414086077
:10D320000121DFF89C04006801F095FC9949086030
:10D330000022DFF88C0401681820F6F7FEF907BD1B
:10D3400000B583B0DFF8E0050068C00005D501F046
:10D350004FFBDFF82417086036E0DFF88C0A00681E
:10D36000C00009D543F66D708A49086001F06EFB74
:10D37000DFF80417086027E00D20DFF8A815087013
:10D380001620F6F741F9DFF8381408600120019003
:10D390000020009001230A220121DFF82404006804
:10D3A00001F07FFBDFF8181408600121DFF810049A
:10D3B000006801F050FC774908600022DFF80004A3
:10D3C00001681620F6F7B9F907BD00B583B0DFF89C
:10D3D00058050068C00005D501F00AFBDFF8981673
:10D3E000086036E0DFF8000A0068C00009D543F69F
:10D3F00071106849086001F029FBDFF87C160860AD
:10D4000027E00E20DFF81C1508700C20F6F7FCF85A
:10D41000DFF8AC1308600120019000200090012388
:10D420000A220121DFF89803006801F03AFBDFF8D7
:10D43000901308600121DFF88803006801F00BFCFD
:10D44000544908600022DFF8780301680C20F6F7E1
:10D4500074F907BD00B583B0DFF8CC040068C000E4
:10D4600005D501F0C5FADFF81016086031E0DFF8E5
:10D4700078090068C00009D543F671704549086015
:10D4800001F0E4FADFF8F015086022E00F20DFF881
:10D49000941408700E20F6F7B7F8C9490860012007
:10D4A00001900020009001230A220121C448006855
:10D4B00001F0F7FAC24908600121C148006801F093
:10D4C000CAFB344908600022BD4801680E20F6F707
:10D4D00034F907BD00B583B0DFF84C040068C00024
:10D4E00005D501F085FADFF89015086051E0DFF806
:10D4F000F8080068C00009D545F650602549086065
:10D5000001F0A4FADFF87015086042E01020DFF89F
:10D51000141408700620F6F777F8A94908600A2065
:10D52000F6F772F8A6490968814212D047F67310DF
:10D5300018490860DFF8F003006810F0C04F28D0E9
:10D5400000210A20F5F73CFB00210620F5F738FB07
:10D550001FE0012001900020009001230A220121F8
:10D560009748006801F09DFA9549086001219448A8
:10D57000006801F070FB07490860002290480168CC
:10D580000620F6F7DAF800228D4801680A20F6F73F
:10D59000D4F807BD682B0020632E00206C2B0020E0
:10D5A00000B583B0DFF880030068C00005D501F046
:10D5B0001FFADFF8C414086053E0DFF82C08006895
:10D5C000C0000AD547F25070DFF8C41B086001F0B4
:10D5D0003DFADFF8A414086043E01120DFF844139B
:10D5E00008700820F6F710F8754908600420F6F76F
:10D5F0000BF873490968814212D047F67310DFF8BF
:10D60000901B0860C848006810F0C04F29D0002166
:10D610000820F5F7D5FA00210420F5F7D1FA20E02B
:10D62000012001900020009001230A22012164487A
:10D63000006801F036FA624908600121604800681C
:10D6400001F009FBDFF8481B086000225C48016814
:10D650000420F6F772F80022594801680820F6F70E
:10D660006CF807BD00B583B0AF480068C00005D5B1
:10D6700001F0BEF9DFF80014086054E0DFF8680735
:10D680000068C0000AD547F67100DFF8041B086087
:10D6900001F0DCF9DFF8E013086044E01220A14952
:10D6A00008701A20F5F7B0FF454908601C20F5F70F
:10D6B000ABFF43490968814223D10120019000203A
:10D6C000009001231E2201213D48006801F0E9F984
:10D6D0003B49086000213A48006801F0BCFA50F06C
:10D6E0008000DFF8AC1A08600022354801681A2073
:10D6F000F6F723F80022324801681C20F6F71DF8DF
:10D7000011E047F67310DFF8881A08608648006851
:10D7100010F0C04F07D000211A20F5F751FA002170
:10D720001C20F5F74DFA07BD80B57F480068C000A2
:10D7300005D501F05DF9DFF8401308603FE0DFF840
:10D74000A8060068C0000AD543F67870DFF8401AD2
:10D75000086001F07BF9DFF8201308602FE0132048
:10D76000704908704FF48060F5F716FF144908609F
:10D770006D48006810F0C04F0AD0114800680028BA
:10D7800003D000200E49086002E001200C49086027
:10D790000B480068002809D05B20DFF8F419086006
:10D7A00000214FF48060F5F7FCFE08E00620DFF86A
:10D7B000E019086000214FF48060F5F70BFF01BD10
:10D7C0005C2B002080B51E20F5F71EFF092804D130
:10D7D00001F00EF9A849086055E053480068C00000
:10D7E00004D501F005F9A44908604CE0DFF8F8051C
:10D7F0000068C00009D545F63760DFF89419086065
:10D8000001F024F99C4908603DE014204549087066
:10D810004FF40070F5F7C0FEDFF8D41B0860FEF788
:10D82000E1FA4149096811F0C04F13D0C0B207288E
:10D8300010D0C0B208280DD0DFF8B40B0068002863
:10D8400004D00020DFF8A81B086003E00120DFF807
:10D85000A01B0860DFF8980B0068002809D06E2034
:10D86000DFF82C19086000214FF40070F5F799FEDD
:10D8700009E045F25C40DFF81819086000214FF418
:10D880000070F5F7A7FE01BD00B583B0264800681B
:10D89000C00004D501F0ACF87749086041E0DFF83A
:10D8A00048050068C00009D547F67340DFF8E01866
:10D8B000086001F0CBF87049086032E01520194982
:10D8C00008703B20F5F7A0FEDFF8241B086001205C
:10D8D000019000200090012302220021DFF8100BAC
:10D8E000006801F0DEF8DFF8081B0860DFF8000BC5
:10D8F0000068002805D145F25C40DFF89418086004
:10D9000008E00121DFF8E80A006801F0A4F9DFF877
:10D91000801808600022DFF8D80A01683B20F5F77C
:10D920000CFF07BD622E0020582B00201CB5040000
:10D93000DFF8000A0068C00012D5DFF8B40A0068FA
:10D9400010490968884206D02100C9B2DFF8A00A50
:10D95000006801F0DDFA01F04BF84749086041E248
:10D96000DFF884040068C00040F188802000C0B265
:10D9700001F099F9DFF8781A0860DFF8740A006896
:10D98000004901E0602B00200860E4B2012C05D1C1
:10D9900043F60610DFF8F817086067E0E4B2022CDF
:10D9A00005D143F65B10DFF8E81708605EE0E4B2EB
:10D9B000032C05D143F64F10DFF8D417086055E06B
:10D9C000E4B2042C05D143F66610DFF8C4170860F2
:10D9D0004CE0E4B2052C05D147F20630DFF8B01771
:10D9E000086043E0E4B2062C05D147F25B30DFF873
:10D9F000A01708603AE0E4B2072C05D147F24F3097
:10DA0000DFF88C17086031E0E4B2082C05D147F24A
:10DA10005B30DFF87C17086028E0E4B20B2C05D1FE
:10DA200040F25E60DFF8681708601FE0E4B20C2C7B
:10DA300005D147F65E10DFF85817086016E0E4B22B
:10DA4000092C05D147F60610DFF8441708600DE0F1
:10DA5000E4B20A2C05D147F65B10DFF834170860F2
:10DA600004E047F65010DFF82817086000F0EEFFDA
:10DA700001490860B6E100BF402B00201620DFF806
:10DA8000781B0870DFF868090068642880F09481CA
:10DA9000012001900020009001231C220021DFF8CA
:10DAA0005009006800F0FDFFDFF8441908601E20EF
:10DAB000F5F7AAFD07282ED1DFF8340900680928F8
:10DAC00019D0DFF82C090068192814D0DFF82009D4
:10DAD000006805280FD0DFF81809006806280AD06A
:10DAE000DFF80C090068022805D0DFF80409006897
:10DAF000032840F05881012001900020009001236C
:10DB00001C220021DFF8E808006800F0CAFFDFF8F7
:10DB1000E0180860D0E71E20F5F776FD062840F0F3
:10DB20002E81E4B20B2C2ED1DFF8C4080068122835
:10DB300019D0DFF8BC080068132814D0DFF8B0084B
:10DB4000006810280FD0DFF8A808006811280AD054
:10DB5000DFF89C080068162805D0DFF894080068F4
:10DB60001A2840F02081012001900020009001231C
:10DB70001C220021DFF87808006800F092FFDFF82F
:10DB800070180860D0E7E4B20C2C42D1DFF86008CE
:10DB900000680E282DD0DFF8580800680F2828D01C
:10DBA000DFF84C080068172823D0DFF84408006825
:10DBB00018281ED0DFF838080068122819D0DFF8BE
:10DBC00030080068132814D0DFF8240800681028F3
:10DBD0000FD0DFF81C08006811280AD0DFF8100801
:10DBE0000068162805D0DFF8080800681A2840F0F9
:10DBF000DA80012001900020009001231C220021E6
:10DC0000DFF8EC07006800F04CFFDFF8E41708606D
